:020000022000DC
:1060000000F0032059620200896202008B620200E4
:106010008D6202008F6202009162020000000000A7
:106020000000000000000000000000009362020079
:10603000956202000000000097620200996202006F
:106040009D6202009F620200A1620200A362020040
:10605000A5620200A7620200916F0200AB6202001B
:10606000AD620200AF620200B15E0300B3620200E3
:10607000B5620200B7620200B9620200BB620200B0
:10608000BD6202000D97030079B90200C3620200ED
:1060900035970300C7620200BD8C0300CB6202008B
:1060A000CD620200CF620200D1620200D362020020
:1060B000D5620200D76202009B6202009B6202006E
:1060C000D9620200DB620200DD620200DF620200D0
:1060D000E1620200E3620200E5620200E7620200A0
:1060E000E9620200EB620200ED6202009B620200C4
:1060F0009B620200F16202009B620200EF620200FA
:10610000354936480A1A02D0072291438D46344950
:1061100034480A1A06D00722914381F309880222E3
:1061200082F3148830483149314A00F043F831484D
:106130003149324A00F03EF831483249324A00F0E3
:1061400039F832483249334A00F034F8324833499A
:10615000334A00F02FF833483349344A00F02AF824
:1061600033483449344A00F025F834483449002291
:1061700000F02BF833483449002200F026F8334869
:106180003349091A082903DB002202600430016048
:106190001F482049884205D00268043003B4904764
:1061A00003BCF7E700208646EC4600200021294A80
:1061B0009047FEE7884207D0521A05D00378013095
:1061C0000B700131013AF9D17047884202D0027058
:1061D0000130FAE77047000000F0032000E80320D8
:1061E00000F0032000F003200C090400C832002056
:1061F00028340020F4620200F462020004F4030078
:106200000C090400C8320020C832002034F4030016
:1062100034F4030034F4030034F4030034F40300D2
:1062200034F4030034F4030034F403000C090400D4
:106230006C0A040028340020283400202834002070
:10624000A96A0020AC6A0020AC6A0020AC6A002079
:10625000AC6E0020FD6A020008484FF00701884339
:106260008546074880470748016841F4700101608E
:10627000BFF34F8FBFF36F8FFFF742BF00F00320D4
:10628000E598030088ED00E0FEE7FEE7FEE7FEE7A5
:10629000FEE7FEE7FEE7FEE7FEE7FEE7FEE7FEE7D6
:1062A000FEE7FEE7FEE7FEE7FEE7FEE7FEE7FEE7C6
:1062B000FEE7FEE7FEE7FEE7FEE7FEE7FEE7FEE7B6
:1062C000FEE7FEE7FEE7FEE7FEE7FEE7FEE7FEE7A6
:1062D000FEE7FEE7FEE7FEE7FEE7FEE7FEE7FEE796
:1062E000FEE7FEE7FEE7FEE7FEE7FEE7FEE7FEE786
:0462F000FEE700BF06
:1062F40041DF704776DF70477ADF70477CDF704795
:1063040008B504F0BFF908BD00B583B09DF80430AA
:10631400012262F3030362F3071302A800F8043DA9
:1063240011220549FFF7EAFF10B903B05DF804FB39
:1063340012F077F8F9E700BF4CF5030008B512F046
:1063440070F808BD00B583B0037823B1012B0BD0DE
:1063540003B05DF804FB3B214088FFF7CBFF002826
:10636400F6D012F05EF8F3E70A4B1B6813F4804F83
:10637400EED0094B1B68032BEADD084BD3F8043538
:10638400074A00924FF4B9720649042006F038FB1C
:10639400DEE700BF383300203433002000B0004073
:1063A40024F603001CF603000C4B1B6813F4804F07
:1063B40012D00B4B1B68002B0EDD00B583B0094BCC
:1063C400D3F80435084A0092AA220849012006F0AD
:1063D40017FB03B05DF804FB704700BF383300209F
:1063E4003433002000B00040A4F403001CF6030082
:1063F4002DE9F04188B004AF6421334800F0CAFCB1
:1064040008F052FEA0B9314B1B78BBB100F078FF05
:106414002F4B1B6813F4804F46D02E4B1B68032B65
:1064240042DDE8468AB00DF1100C6646002326E0F2
:10643400294A40F2D11113F03DFBE4E7274A3B1D02
:1064440007CA83E80700184600F03EFC0028DDD0A8
:10645400214A4FF4EE7113F02DFBD7E7C25C4FEAEB
:10646400121E59001E4C256815F80EE006F813E0BC
:1064740002F00F0201312468A25C725401330F2B25
:10648400ECD900238CF82030164BD3F80435CDF822
:1064940008C0154A0192154A00924FF4F07214494B
:1064A400042006F0ADFAC54600214FF4F03000F0A8
:1064B400E6FC0222C8214FF4F03000F0EBFC103768
:1064C400BD46BDE8F08100BF496702006834002082
:1064D4003833002034330020DCF5030034F40300A7
:1064E4003C33002000B0004084F6030094F603001F
:1064F4001CF6030000B58BB00023ADF80830102360
:10650400ADF804301423ADF806304FF4C873ADF879
:106514000A3001A8FFF7F0FEC0B9002306930793E1
:1065240001AB039340F6CD4304934FF480330593BA
:1065340003238DF81830084B0893084B099303A8DC
:1065440012F0D0FD28B90BB05DF804FB11F069FF1F
:10655400E3E711F066FFF6E74963020041630200D6
:1065640000B585B01F4B1B6813F4804F03D01E4B3E
:106574001B68032B1DDCFFF7C7FEFFF7BBFF03A857
:106584000DF0B0FE174B1B6813F4804F03D0164B6D
:106594001B68032B18DC00214FF4F03000F06FFC73
:1065A4000422C8214FF4F03000F074FC05B05DF80B
:1065B40004FB0E4BD3F804350D4A009293220D4987
:1065C400042006F01DFAD6E7084BD3F80435BDF8CD
:1065D4000C200192084A00929B220649042006F0EE
:1065E4000FFAD8E7383300203433002000B00040DD
:1065F40050F603001CF603006CF6030070B582B07D
:106604000446474B1B6813F4804F03D0454B1B686B
:10661400032B05DC032C54D8DFE804F00F0F2A2ADF
:10662400414BD3F804350190404A00924FF48E72E6
:106634003F49042006F0E4F9ECE73E4D05EB041570
:1066440004F10D0000F0FEFB80F00101C9B2284600
:1066540018F0AAFC0546112D58D8DFE805F032578A
:106664005757235757412357575757575757572368
:10667400304D05EB041504F10D06304600F0E2FB45
:1066840080F001010222C9B2284618F0AFFC054689
:10669400304600F0D7FB80F00101C9B2304600F06B
:1066A400DDFBD8E71E4B1B6813F4804F03D01D4B52
:1066B4001B68032B07DC062232214FF4F03000F074
:1066C400E9FB02B070BD184BD3F8043501941A4AA3
:1066D40000924FF49E721649042006F091F9EAE7FD
:1066E4000F4B1B6813F4804FEBD00E4B1B68032B2E
:1066F400E7DD0D4BD3F804350194104A00924FF4B2
:10670400A4720B49042006F07BF9DAE7002DD8D0F7
:106714000B4A4FF4A671284613F0CCF9D1E700BF19
:10672400383300203433002000B0004040F403002C
:106734001CF603002834002054F4030078F403000A
:10674400DCF503003038032800D9704708B5FFF79B
:1067540055FF08BD00B58BB02022002101A818F018
:10676400EAFD01238DF8043007238DF807308DF8F6
:106774000C300A4B04930A4B05930A4B09930A49BC
:1067840001A808F057FC10B90BB05DF804FB074AE8
:1067940040F2851113F08EF9F6E700BF90F503007F
:1067A400ED6A02007D68020068340020DCF5030015
:1067B40000B585B0284A04214FF4C04006F004F91E
:1067C400264B1B6813F4804F03D0254B1B68032B07
:1067D40020DC12F0B1FF48BB00F08CFB214800F034
:1067E400A9FB48BB12F0DCF960BB04A9002341F803
:1067F400043D012012F0C0FA38BB03A812F00EFBCE
:1068040030BBFFF781FDFFF775FEFFF7A3FF05B06F
:106814005DF804FB144BD3F80435144A009240F29B
:10682400B5121349042006F0EBF8D2E7114A40F2FE
:10683400B71113F03FF9CFE70E4A40F2BB1113F042
:1068440039F9CFE711F0EDFDCFE711F0EAFDD4E718
:1068540011F0E7FDD5E700BFA1C9020038330020DD
:10686400343300200166020000B0004060F50300EC
:106874001CF60300DCF5030010B582B01D4B1B6849
:1068840013F4804F03D01C4B1B68032B01DC002442
:1068940012E01A4BD3F80435194A00924FF4AE7241
:1068A4001849042006F0ACF8F1E7174A4FF4B17127
:1068B40013F000F90FE00134032C19D8134800EB4E
:1068C4000410134B4360134B8360611C89B218F0AE
:1068D40047FB0028E9D123010C4AD05A0BF0A2FB54
:1068E4000028E8D0084A40F2631113F0E3F8E2E725
:1068F40002B010BD383300203433002000B0004013
:10690400A0F503001CF60300DCF503002834002086
:1069140039690200AD63020010B5054C041B241153
:106924001D2C01D8204610BD784600F0B7FCF9E7CD
:106934002834002030B583B00D46FFF7EDFF044640
:10694400032D7CD8DFE805F026024B6601210D30CB
:1069540000F084FA444B1B6813F4804F03D0434B7C
:106964001B68032B0ADCE20804F00704802323419C
:106974003F498C5C1C438C5403B030BD3D4BD3F871
:10698400043501943C4A0092B4223C49042006F0A8
:1069940037F8E8E700210D3000F060FA324B1B684D
:1069A40013F4804F03D0314B1B68032B0BDCE2083C
:1069B40004F0070480232341DB435BB22C49885C49
:1069C40003408B54D8E72B4BD3F8043501942C4A5D
:1069D4000092BC222949042006F012F8E7E70622B7
:1069E40032214FF4F03000F055FA1F4B1B6813F4BA
:1069F400804FC1D01D4B1B68032BBDDD1D4BD3F84D
:106A0400043501941F4A0092C4221C49042005F055
:106A1400F7FFB1E7144B1B6813F4804FACD0134B52
:106A24001B68012BA8DD134BD3F804350190164ADB
:106A34000092C8221149022005F0E2FF9CE70A4BAC
:106A44001B6813F4804F97D0084B1B68002B93DD11
:106A5400084BD3F804350D4A0092CB220749012094
:106A640005F0CEFF88E700BF383300203433002020
:106A74006C34002000B00040C0F403001CF6030096
:106A8400DCF40300F8F4030018F5030038F5030000
:106A940000B583B00F4B1B6813F4804F03D00E4B2B
:106AA4001B68032B0ADC0322C8214FF4F03000F0EA
:106AB400F1F908F003FB03B05DF804FB074BD3F8CE
:106AC4000435074A0092D2220649042005F098FFB3
:106AD400E9E700BF383300203433002000B0004021
:106AE400C0F503001CF6030008B503781C2B00D086
:106AF40008BDFFF7CDFFFBE738B5FFF759FEEFF30D
:106B0400108572B6174B9B689BB9164A0123936094
:106B1400154BD3F88010154801401160C3F880006C
:106B2400D3F8841051604FF0FF32C3F8842000245E
:106B340000E0012405B962B6FFF75AFC094B9B68D3
:106B44006BB164B9EFF3108372B6064A1068064954
:106B54000860506848600021916003B962B6FFF78D
:106B6400C7FBFCE7C868002000E100E0FC06FFBDAD
:106B74002A4B1B78002B4FD000B585B0012804D0D8
:106B8400032842D005B05DF804FB04A9002341F8B2
:106B9400083D012012F0F0F840BB02A812F03EF9C3
:106BA40038BB04A9012341F8043D0DF106000EF0A1
:106BB400C7F808BBBDF806000DF05CFD0DF105013A
:106BC4000DF0AEFED8B909F0BFFC9DF80510002009
:106BD40009F07CFD03F0ECFCA0B9104B00221A7004
:106BE4000F4B1B68002BCDD09847CBE711F019FC55
:106BF400D3E711F016FCD4E711F013FCDAE711F037
:106C040010FCE0E711F00DFCE7E711F0C9FF0028E4
:106C1400B8D011F006FCB5E7704700BFED34002092
:106C2400F034002008B5084B01221A7003F0E2FC8E
:106C340018B911F0F9FF18B908BD11F0F2FBF8E723
:106C440011F0EFFBF8E700BFED34002008B5032393
:106C5400002203494968034813F006FD08BD00BF3C
:106C6400F03400203437002008B50378052B0DD00C
:106C7400082B16D0022B00D008BD104B1B7813B97B
:106C8400FFF7E4FFF8E7FFF7CDFFF5E710220C4B21
:106C940099680C4813F072FD0028EDD011F0C1FB87
:106CA400EAE78168C06808F074F918B9034B012257
:106CB4001A70E1E711F0B5FBF8E700BFEC340020EF
:106CC400F03400203437002010B586B00446214A41
:106CD40003AB07CA03C323F8022B120C1A701E4B12
:106CE40094E8070083E80700002A31D01B491C48B8
:106CF40013F09EFC034610B1184606B010BD194BA4
:106D0400009303AB154A1649174813F04DFC03468C
:106D14000028F1D1154815F005F80146124813F082
:106D24006FFC03460028E7D1114813F027F8034607
:106D34000028E1D10E4813F057F801460A4813F031
:106D44005FFC03460028D7D1FFF780FF0346D3E753
:106D54000723D1E7ACF60300F0340020FC34002014
:106D6400683800206D6C0200343700201C35002088
:106D7400E436002008B5064B1B683BB110F094F9CB
:106D8400002803DB024B1B689847F7E708BD00BFE8
:106D9400A838002010B50C46144B1860144A012181
:106DA400144812F0F9FCA0B9610CE00341F26F72CF
:106DB40000238B4208BF824210D24FF47A72002320
:106DC40018F044F9014600220B4812F0FBFC38B9D4
:106DD40010BD0A4A462112F06DFEE5E70521F2E7EF
:106DE400064A472112F066FEF2E700BFA8380020E9
:106DF400796D0200B8F60300AC380020BCF603003D
:106E040008B50D4B1B6873B14FF0A042D2F804359E
:106E14000A4909684B40C2F80435074A1368013B24
:106E2400136023B108BD002011F0FBFAECE704481D
:106E340012F0E6FCF6E700BFCC380020D038002082
:106E4400D43800204FF0A043D3F80425012303FADB
:106E540000F002420CBF18460020704739B90123E4
:106E640003FA00F04FF0A043C3F80805704701236C
:106E740003FA00F04FF0A043C3F80C05704721B9A2
:106E84004FF0A043C3F8080570474FF0A043C3F880
:106E94000C05704712B11346132900D8704770B51A
:106EA400114A10605B00013B104A136000264D0C30
:106EB400CC034FF47A72002314F5FA7045F1000103
:106EC40018F0C4F832460146094812F07BFC48B970
:106ED4004FF0A042D2F804350349096823EA0103BC
:106EE400C2F8043570BD00BFD0380020CC38002073
:106EF400D438002008B50D230BE04FF0A04103F572
:106F0400E072032041F8220001229A40C1F80825CA
:106F14000133102BF1D9054A0121054812F03CFC3C
:106F240000B908BD11F07DFAFBE700BF056E020051
:106F3400F8F60300F0B1104A1060002309E00F4A8C
:106F4400D25C02F5E0724FF0A0410D4841F82200F6
:106F54000133032BF3D90B4B4FF00042C3F8042346
:106F64000020C3F87C01084BE02283F8062340226A
:106F74001A6070470E207047F4380020FCF60300B6
:106F84000C0003000060004000E100E010B50024A4
:106F9400144BC3F87C410EE043F23333994208D9D1
:106FA400114BD3F80425114B1A60114B1B68204672
:106FB40098470134E4B2032C12D84FF0A043D3F81D
:106FC40010250C4B195D01238B409343F1D0074BE3
:106FD4001B68054AD2F80425991ADDD5D11ADBE7D6
:106FE40010BD00BF0060004000B00040F838002031
:106FF400F4380020FCF6030072DF704773DF70473B
:1070040074DF70472DE9F047A2B0074688469146E1
:10701400314C0026C4F80660E68130490B78C3EB96
:1070240043102F4D054425602E4A0244A2601F22BE
:10703400A280A281013303F001030B704FF03C0ADC
:107044005246314613A818F076F906238DF84F30CE
:10705400ADF8487001238DF84A30ADF85C3012AABF
:107064001892ADF83C70ADF84090CDF844800DEB2B
:107074000A021D928DF8783052463146684618F05F
:107084005AF902238DF80030221D294613A811F065
:1070940071FC90B9104B03F10C029968684611F029
:1070A40069FC68B9104A0C491048FFF7A5FF082885
:1070B40009D070B922B0BDE8F08711F0B2F9E9E760
:1070C40011F0AFF9EEE7002203490848FFF794FFF7
:1070D400EFE711F0A6F9EDE740390020FC38002075
:1070E4000039002050390020CC320020C832002062
:1070F400034B00EB800042009A819960704700BF07
:10710400CC32002008B50121054B1878FFF776FF33
:1071140010B904F069FA08BD11F083F9F9E700BF6A
:10712400C832002008B5044B1878FFF769FF00B98E
:1071340008BD11F076F9FBE7C8320020062070473D
:1071440000B587B041F20103984245D020D944F2FA
:107154000103984256D044F2020398426DD1454B44
:107164001B6813F4804F1ED0434B1B68002B1ADDA1
:10717400424BD3F80435108803905268029201916F
:107184003F4A00925F223F49012005F039FC0AE0A2
:10719400012852D1374B1B6813F4804F03D0364B70
:1071A4001B68002B0BDC4FF0A0434FF4F032C3F804
:1071B4001825C3F80C25EFF3108372B653E02F4B58
:1071C400D3F80435029201912F4A009254222D499A
:1071D400012005F015FCE6E7264B1B6813F4804FED
:1071E400E1D0254B1B68002BDDDD244BD3F804359F
:1071F40002920191254A009257222249012005F06A
:10720400FFFBD0E71B4B1B6813F4804FCBD01A4B0A
:107214001B68002BC7DD194BD3F8043510680490A4
:1072240050680390029192680192194A009269226F
:107234001449012005F0E4FBB5E70E4B1B6813F479
:10724400804FB0D00C4B1B68002BACDD0B4BD3F83C
:10725400043501910F4A00926D220A49012005F07C
:10726400CFFBA0E730BF0C4B1B78002BFAD107B043
:107274005DF804FB383300203433002000B00040B4
:1072840080F703002DF7030040F703005CF70300C9
:10729400A0F70300C4F70300E432002000B583B074
:1072A4000023ADF80030054B01936A46014644F2D1
:1072B4000200FFF745FF03B05DF804FB48F5030047
:1072C40010B40346044C006859689A68DB680FC41C
:1072D4005DF8044B704700BF90390020064B074A05
:1072E40092E8030083E803000833443292E8030081
:1072F40083E80300704700BF90390020600000104D
:107304000048704790390020002308E0074901EB4A
:10731400C30000224280426001F8332001331F2B56
:10732400F4D9034B00221A60704700BFA039002033
:10733400A03A002030B405460F4B1B6800240AE035
:107344001F230E4A12F83300A0B102EBC302528885
:10735400AA4207D001341F2C0BD85A1E002BEFD0A1
:107364001346EEE7054A02EBC30252688A42F1D1A2
:1073740000E0002030BC7047A03A0020A039002073
:1073840030B40A4A13680A4C04EBC3056880696088
:10739400012104F833100B441360202B01D030BCBE
:1073A4007047134600221A60F9E700BFA03A002094
:1073B400A0390020C0F30C038B4202D3C91A08443D
:1073C4007047C91A0844A0F500507047C37D002BCC
:1073D40042D083780A7802F0800203F07F031343DB
:1073E4000B7002780B7803F07F0343EAC2130B702F
:1073F4000378002B41D030B44378082B14BF00220B
:1074040001224B7803F07F0343EAC2134B70858853
:1074140003F08003C5F3861423434B708A7802F08B
:10742400030242EA8502D2B28A70857902F0FC0234
:10743400C5F3C10422438A70CB7803F01F0343EAE7
:107444004513DBB2CB70C27903F0E00302F01F02F4
:107454001343CB7030BC704783780A7802F0BF02C4
:107464009B0103F0400313430B70C27803F0C00385
:1074740002F03F0213430B70B3E770470023032B62
:1074840022DC10B402E00133032B19DC0F4C6C2214
:1074940002FB034292F84420012AF4D16C2202FB3D
:1074A4000342948AC2899442EDD1084C6C2202FBB7
:1074B400034292888A42E6D16C2202FB034000E038
:1074C40000205DF8044B704700207047183B0020F3
:1074D400002300E00133032B13DC0B496C2202FB75
:1074E400031292F84420022AF4D16C2202FB031204
:1074F400918A828A9142EDD103486C2202FB0300F7
:1075040070470020704700BF183B002008B10820D6
:10751400704704207047000038B505460C46CB6917
:107524005B78C370CB691B7883F001038370CB69EC
:107534004362087B022814D0FFF7E8FF6870E27A00
:1075440032B9A18AC0F10F03994201DC082831D075
:10755400A18A0346C0F10F00814207DC42B3012235
:1075640005E0154B987DFFF7D1FFE7E701222A706C
:1075740062B1A28A13440B33104A82FB0312DB1755
:10758400C3EB6203013BEB710023AB710023EB758A
:1075940005F10C0294E8030082E80300A2692A6260
:1075A4002289AA82A27AAA75226AAA62184638BDDA
:1075B4000022DCE70720FAE7003B0020ABAAAA2A56
:1075C40030B403460C460978817000214162A168F9
:1075D4000B2903D8217BF1B1012100E001211970AD
:1075E4000020587029B1A1680731C9080139D9713F
:1075F40098710121D97503F10C0504F1100103C937
:1076040085E80300E1899982A1691962217F99754E
:107614009A6230BC70470021E1E700000021164B5C
:107624001B688B4226D90023144A02EBC10252681C
:107634009A421DD910B4114A52F8312002EBC30406
:1076440012F8332082420DD001330C4A02EBC102FE
:1076540052689A42EFD80131074B1B688B4205D917
:107664000023F2E760685DF8044B70470020FAE7F6
:107674000131D4E700207047A43A0020A83A002042
:1076840070B58CB006460D4614462C22002101A884
:1076940017F051FE0E238DF80430ADF808604FF05A
:1076A400000365F300038DF80A308DF80B4001A840
:1076B40001F0B0F90CB070BD30B58DB005460C4684
:1076C4002C22002101A817F036FE0F238DF8043078
:1076D40002958DF80C4001A801F09CF90DB030BD65
:1076E40000B58DB048B913F1020F06D001228DF810
:1076F4000420029301A801F08DF9034B186804F0EB
:1077040069F80DB05DF804FBB43A00202DE9F041AE
:10771400054688460378BBB10D4B1C68621C1A6091
:1077240004F00704AB8A0B4F07EBC4067380A988E7
:10773400A869FFF73FFE7060EB6903F00103737003
:1077440007F83480BDE8F0817846FFF7A7FDE3E74A
:10775400FC3A0020BC3A002070B5064603784BB1D1
:10776400B58A347F04F00104B188B069FFF722FEC2
:10777400002304E07846FFF791FDF1E70133072B7E
:1077840015D80C4A02EBC30252688242F6D1094A68
:1077940002EBC3025288AA42F0D1064A02EBC302AA
:1077A4005278A242EAD1034800EBC30000E0002073
:1077B40070BD00BFBC3A0020F0B40D684C688F68FF
:1077C400CE68D5601461576196610D694C69D561C5
:1077D40014620378DB091370D17DF9B1037803F0E7
:1077E4007F0393700023537013789BB143789B01FC
:1077F40003F4FE53817843EA910393808378DB009A
:1078040003F01803C17843EA51139371C37803F06A
:107814001F03D37100235362F0BC70470178C1F396
:1078240080119170017801F03F01D17043B190F95A
:107834000130002B02DB04235370D5E70823FBE758
:1078440004235370D0E770B50C461E4603788BB101
:1078540004252A44A26000F10C032360836A636058
:10786400204604F05DFB024610B923691D443560CF
:10787400104670BD0125ECE72DE9F0418EB00D46B0
:1078840016461C46804600282DD0002D2FD0002CF3
:1078940031D0636A0233059304F10C00A378002B02
:1078A4002DD00121627801AF3B46082A14BF002283
:1078B400012204F08CF80697CDF81C80B2B2ADF822
:1078C40020200B9515440C9563788DF83430237B78
:1078D400022B16D00023ADF8283005A804F06FF869
:1078E4000EB0BDE8F0817846FFF7D8FCCDE77846C6
:1078F400FFF7D4FCCBE77846FFF7D0FCC9E70221B9
:10790400D0E723692BB1236909931023ADF82830FC
:10791400E3E77846FFF7C2FCF5E72DE9F04186B0CE
:1079240004460D46C37D002B3ED0082605FB06F811
:10793400E379AB423AD0A5716B46324601A92046A1
:10794400FFF781FF074648BB4DB994F84F3033B970
:10795400A369C3F30C03A380012384F84F30E37DB0
:107964007BB994F84E3063B92DBBB4F846106278F5
:1079740023468A1AA16E0846FFF77EFF012384F886
:107984004E3005992046FFF721FDA16E3246414451
:10799400009817F0A7FC01A804F0DCFAB7FA87F006
:1079A400400906B0BDE8F0810C26BFE7B4F8466094
:1079B400A6EB0806BFE77846FFF770FCD5E770B57D
:1079C400054690F84C40002605E00136631C85F816
:1079D4004C300134E4B2EB79A3420AD3AA6C0123FC
:1079E400A3401A42F5D121462846FFF796FF002806
:1079F400EBD1304670BDF0B587B045781544C37DF2
:107A0400DBB10B239D4221D816460F4604466B4634
:107A14002A4601A9FFF717FF0546C0B90599204674
:107A2400FFF7D4FCE37D53B132463946009817F092
:107A340059FC01A804F08EFA09E00F23E2E723467B
:107A4400324600993846FFF717FFF2E70925284622
:107A540007B0F0BD10B5044690F84430012B0ED1A8
:107A6400237B012B0FD00C4BDB68A36303F0AEF92F
:107A7400A16B014404F12C0003F00CF910BD78460D
:107A8400FFF70CFCECE7A37D034AD168126902FB03
:107A94000313A363EAE700BF003B002038B50024CA
:107AA40000E00134032C13D80A4A6C2303FB04239B
:107AB40093F84430012BF4D16C2505FB04252846AA
:107AC400FFF77DFF0028ECD02846FFF7C3FFE8E767
:107AD40038BD00BF183B002038B5044690F8443048
:107AE400022B02D07846FFF7D9FB054B1D6803F043
:107AF4006DF9411904F12C0003F0CCF838BD00BF36
:107B0400003B002038B5044690F84430022B02D0E4
:107B14007846FFF7C3FB084B5D7D5A689B6803FBFF
:107B2400052503F053F9411904F14C0003F0B2F8B0
:107B3400012384F8643038BD003B002010B50446AE
:107B44000C4B1B68806E98470023A36604F12C003D
:107B540003F070F894F84430022B05D0002084F828
:107B6400440002F00BF910BD04F14C0003F062F87C
:107B7400F4E700BFB83A002010B504460121FFF72E
:107B8400C5FD2046FFF7DAFF10BD10B58CB00446E2
:107B940090F84430012B02D07846FFF77FFB012395
:107BA4008DF80430236D029301A800F033FF2046C2
:107BB400FFF7C4FF0CB010BD2DE9F04104460E469A
:107BC40015461F46531EDBB2012B46D8A36E13B1D4
:107BD4007846FFF763FB2E4B1B6838469847A06630
:107BE400002852D03346224606F12001D3F8008003
:107BF400D3F804E0D3F808C0D868C2F80080C2F80B
:107C040004E0C2F808C0D060103310328B42EDD1CA
:107C1400186859689B681060516093600023A364DE
:107C2400A4F84670B188B069FFF7C4FBA061012DC8
:107C340017D06FF00103A362002384F86430154B5E
:107C44006365E465144B6363E463012002F096F812
:107C540084F844500120BDE8F0817846FFF71EFB0C
:107C6400B4E70E4B1B7D84F84D30002384F84E306E
:107C740084F84F3084F84C30B36A23656FF0010305
:107C8400A362074B6363E463DFE70020E3E700BF1D
:107C9400B03A0020E7870200CD7D0200003B0020BF
:107CA400D97D020030B583B0C3790133C27D92B16E
:107CB400082505FB03F582B14FF48073AB422AD249
:107CC4001E4B1B6813F0040F36D01D4B1B68002B92
:107CD40006DC00242DE00C25EBE74FF4C073EDE740
:107CE400184BD3F804350195174A00924FF41772D4
:107CF4001649012004F084FE00241AE0144C6C237D
:107D040003FB02442B46022201462046FFF754FFA0
:107D140078B900240DE00022032A09DC0C4B6C2402
:107D240004FB023494F84430002BE7D00132F3E72B
:107D34000024204603B030BD0024FAE73833002085
:107D44003433002000B0004038F803002BF803005F
:107D5400183B002030B585B00D460446A8B100217B
:107D64002046FFF7D3FC2946206DFFF7A5FC2046EB
:107D7400FFF7E4FE0F4B1B6813F0040F03D00E4B08
:107D84001B68032B05DC05B030BD7846FFF786FA87
:107D9400E5E70A4BD3F8043594F8442002950192A0
:107DA400074A00924FF4D2720649042004F028FED8
:107DB400E9E700BF383300203433002000B000402E
:107DC400E0F703002BF8030008B508460021FFF78D
:107DD400C1FF08BD10B50C4691F84430012B09D100
:107DE40094F84D307BB9237B012B07D02046FFF755
:107DF400CCFE10BD7846FFF751FAF1E7002120468A
:107E0400FFF7A8FFF5E7013B84F84D30002384F821
:107E14004C302046FFF7D3FDEBE70000062900D0E5
:107E2400704770B582B003460178890101F4FE51B0
:107E340040789D78DC78240444EA05641D7944EA9A
:107E440005245B791C4341EA90011046FFF716FBB9
:107E54000546B8B1866C2643866444B3037853B3AD
:107E6400EB795A1C01239340013B9E4227D0002307
:107E740085F84C302846FFF7A2FD2846FFF7EAFDB7
:107E840002B070BD104B1B6813F0040FF8D00F4BF9
:107E94001B68012BF4DD0E4BD3F804350D4A009218
:107EA40040F2B2420C49022004F0AAFDE8E70321A3
:107EB400FFF750FFE4E77846FFF7F0F9D0E72846EC
:107EC400FFF763FEDCE700BF3833002034330020C3
:107ED40000B000404CF803002BF803002DE9F043F8
:107EE40089B080460F4614461E4695780DB3284641
:107EF400FFF794FB8146C8B18DF80050236A0693BE
:107F0400A38AADF80E3004AB04F10C0292E803002E
:107F140083E80300A37D8DF81C30CDF8048002971C
:107F240023788DF80C3031466846C84709B0BDE85F
:107F3400F083FFF773FFF9E700B585B000238DF8F0
:107F44000F3098B10346084602330B600DF10F0160
:107F540003F039FD9DF80F3043B10D4B1B6813F04E
:107F6400040F03D00B4B1B68032B04DC9DF80F009C
:107F740005B05DF804FB084BD3F80435074A0092BA
:107F84004FF439720649042004F03AFDEEE700BFCD
:107F9400383300203433002000B000408CF8030054
:107FA4002BF803002DE9F0438FB004460E46154626
:107FB4001F46D0F81890037823B181884846FFF70C
:107FC400F9F9A06104F10C00A378002B3AD0012147
:107FD40062780DF128084346082A14BF00220122C2
:107FE40003F0F5FCC4F81890CDF808800396637884
:107FF400EA1A92B2ADF810203244089207978DF82D
:1080040024300023ADF81830237B022B1CD0A37836
:108014006BB3237B022B1BD02546002345F8243F5A
:108024002A46E178206A0DF0BBF9606A98B101A98B
:10803400FFF782FF00283AD12A46E178206A0DF042
:10804400AFF9F2E70221C3E71023ADF81830DEE7F9
:1080540023690593E0E7237B022B2CD104F10C0167
:10806400E0890DF04BFA0028D3D1052020E000234D
:108074006362237B012B0DD02146002341F8243F6A
:10808400A08A0DF0AAF901A9606AFFF755FFA0B113
:1080940000200DE004F12401E0890DF09EF901A90E
:1080A400606AFFF749FF0028E6D0002000E00020C6
:1080B4000FB0BDE8F0830520FAE70520F8E70000DB
:1080C40070B5F0B00D4614461E4610AB0A46014684
:1080D4002046FFF767FFA0B11F4B1B6813F0040F86
:1080E40037D01E4B1B68052B33DD1D4BD3F80435ED
:1080F4001C4A009240F221521B49062004F080FCE5
:1081040027E003AB01228DF80C20A28AADF80E20E3
:10811400002204928DF8142010AA06926278AD1AF7
:10812400ADF81C5008AA93E8030082E803000AABE8
:1081340004F10C0292E8030083E80300A37D8DF8A8
:108144003830236A0C93636A0D930F9605A800F0E8
:1081540061FC70B070BD00BF3833002034330020A0
:1081640000B00040B0F803002BF8030010B5D47D34
:1081740014B9FFF7A5FF10BDFFF7B0FEFBE7000041
:108184002DE9F04385B004AF43781344C47D94B122
:108194004FF480749C4273D3EFF3108C72B60024B6
:1081A400032C10DC3B4E6C2505FB046595F844500C
:1081B40025B10134F4E74FF4C074EBE735466C267F
:1081C40006FB045400E00024BCF1000F00D162B6A9
:1081D400002C5AD015460E46014601222046FFF7D0
:1081E400EBFC002853D02A463146A06E17F07AF8EB
:1081F400294B1B6813F0040F3AD0284B1B68032B40
:1082040036DD6D46B4F846E04FEA4E030833DB082A
:10821400A5EBC3039D460DF11008C446002312E0EC
:10822400A26ED25C4FEA121959001D48066816F86E
:1082340009600CF8136002F00F0201310068825CDF
:108244000CF8012001337345EAD3002308F81E30EB
:10825400144BD3F80435CDF80880134A0192134A1D
:1082640000924FF47C721249042004F0C9FBAD461D
:108274002046FFF7A4FB2046FFF7ECFB002000E0BC
:1082840009200437BD46BDE8F0830420F9E7042043
:10829400F7E700BF183B00203833002034330020B8
:1082A4003C33002000B000407CF8030094F6030047
:1082B4002BF8030070B504460D461646808A02F07A
:1082C40023F801281AD1237BD3B1022B0BD094F9C4
:1082D4001630002B16DB237853B932462946204644
:1082E400FFF789FB0BE02369002BF0D1102006E097
:1082F400324629462046FFF743FF00E0102070BDB8
:108304001020FCE70720FAE708B50549054800F006
:108314004FF800B908BD7846FEF7C0FFFAE700BF82
:10832400B5F1030021F1030010B5FFF7EDFF4FF4A1
:10833400D8720021134816F0FEFF05F0F1FC00246A
:10834400114B1C6040222146104816F0F4FF104BDC
:10835400104A1A60104A5A604CF250329A600F491F
:10836400D9601A6104221A759C7508225A750C4842
:1083740003F010FA0B4B18600B4B1C600B4805F014
:10838400D5FD10BD183B0020FC3A0020BC3A00206B
:10839400003B002080969800F049020020A10700CD
:1083A4009D850200B43A0020A43A0020E57602003C
:1083B40008B50346B0FA80F040090A46B1FA81F1E3
:1083C4004909884210D14BB1EFF3108072B60849C5
:1083D4000B60084B1A6048B962B606E0002AF3D174
:1083E400FFF792FF002000E00E2008BD0020FCE70C
:1083F400B03A0020B83A0020C0B110B58CB00446A1
:108404000369B3B1C369B3B18369B3B1014601A8C8
:10841400FFF782F8034610B118460CB010BDA28ACB
:10842400216901A8FFF746FF0346F5E70E23184626
:1084340070470E23F0E70E23EEE70E23ECE7D0B1EE
:1084440010B58CB004464068B8B1A269BAB1207CBA
:10845400022816D0B8B194F90020002A15DB0A4688
:10846400214601A8FFF7ACF8A268616801A8FFF7EC
:1084740021FF0CB010BD0E2070470E20F9E70E202E
:10848400F7E71020F5E71020F3E70720F1E70000F5
:10849400037B012B01D00020704710B58AB0002265
:1084A4008388C3F386148DF800409B008DF8013057
:1084B4000B0E8DF802300B0C8DF803300B0A8DF87F
:1084C40004308DF805100623049301238DF8183029
:1084D400838AADF81A3007928DF80820CDF80CD0B5
:1084E400036A08938DF81420C389ADF81630837D90
:1084F40043B98DF824206FF0010102A8FFF79FFF14
:108504000AB010BD024B5B7D8DF82430F3E700BF49
:10851400003B002038B500240BE01E4A6C2303FB0B
:108524000423DB795A1C01239340013B9D4228D04C
:108534000134032C2CD8174A6C2303FB042393F82F
:108544004430022BF4D16C2303FB042393F86430EE
:10855400022BEDD16C2000FB0420816CFFF798FF07
:108564000028E5D10B4A6C2303FB04F3D11881F8EE
:1085740064008D6CD35C002BCFD17846FEF78EFE61
:10858400CBE7044B6C2000FB0430FFF7F5FACFE790
:1085940038BD00BF183B002008B5FFF77FFAFFF78E
:1085A400B9FF012008BD00002DE9F04182B0074663
:1085B4000E46144698461046FEF78AFF054620B13B
:1085C400A28883889A4210D312D82046FFF7C4F8B1
:1085D400B8B103784BB123787BB1E1794B1C01210D
:1085E400994001392046FFF753FF02B0BDE8F081FE
:1085F4000521FFF7AFFB0025E7E77846FEF74EFEBF
:10860400EBE7002D4FD0464B1B6813F0040F03D04B
:10861400444B1B68032B55DC2846FFF75DFA2B7B84
:10862400012B5DD0AA6CA17901238B401A42DCD1C5
:108634001343AB64A279EB799A4259D0E37D002BC2
:1086440061D00823B34260D1AB6EA079E27D002AE9
:1086540060D008243246394604FB003016F042FE4E
:10866400AC6C2B78002B57D0EB795A1C0123934028
:10867400013B9C42B9D1022385F86430A96C284699
:10868400FFF706FF044643462A46B5F84610A86E8F
:10869400FFF76CFD002CA8D1002385F86430284630
:1086A400FFF76AFAA1E72046FFF7FCFA054600281F
:1086B400A9D100212046FFF7EBFE02210020FEF79E
:1086C400FBFF92E7184BD3F80435A2790192174ABD
:1086D40000924FF428721649042004F091F99BE7A4
:1086E40095F86430002B9DD12846FFF70BFA99E7E3
:1086F4009BB2E27D2AB1082203FB0263A5F846304F
:10870400A2E70C22F8E70C239CE704212846FFF794
:1087140021FB6AE70C249DE77846FEF7BFFDA3E73B
:10872400383300203433002000B00040A0F80300A8
:108734002BF803002DE9F0418EB000284DD00546FA
:10874400002A4CD0984614460F4600220C920D92F3
:108754000CA960880CF0D2FE20B9002630460EB079
:10876400BDE8F081226902F00102E168208905F088
:10877400A5FA08B10026F1E7226902F00102E168D6
:10878400208905F06BFA0646C0B901AA214628469D
:10879400FFF712F804AB0EAA12E9030083E8030002
:1087A40002F0B6FF9DF8043083B1434601AA391F95
:1087B400281DFFF7F9FE02F0CBFFCFE72169002265
:1087C40001F001012089FEF75BFFC7E7434601AAD8
:1087D400791E681CFFF7CAFCEDE70E26BEE70E26DD
:1087E400BCE710B50C4691F84430022B0BD10223A0
:1087F40084F86430A16C2046FFF74AFE10B90023C8
:1088040084F8643010BD7846FEF748FDEFE70000B9
:10881400002959D0A0F59670072857D8DFE800F052
:10882400040E1A25313D454D4A68314B13443149F4
:108834008B424DD8304B1A60002070474A68A2F52D
:108844001233A3F5F8732D498B4243D82A4B5A604F
:10885400002070474A68A2F54343503B28498B42A5
:108864003AD8254B9A60002070474A68A2F54333F2
:10887400A3F5A07323498B4230D81F4BDA60002044
:1088840070474A68A2F54333A3F5A0731D498B4290
:1088940026D8194B1A61002070474B689A1EFD2A8E
:1088A40020D8154A1375002070474B685A1E7E2A3B
:1088B4001AD8114A5375002070474B68012B15D8FC
:1088C4000D4A9375002070470E20704705207047AD
:1088D400072070470720704707207047072070471C
:1088E400072070470720704707207047072070470C
:1088F400806967FF80778E06003B0020904C9600CD
:1089040030D3970040899500002934D000220A60B2
:108914004A60A0F5967007282FD8DFE800F0040914
:108924000E13181D2227164A12684A600020704749
:10893400134A52684A6000207047114A92684A609C
:10894400002070470E4AD2684A60002070470C4AE3
:1089540012694A6000207047094A127D4A6000206B
:108964007047074A527D4A6000207047044A927D4E
:108974004A60002070470E2070470520704700BFF2
:10898400003B0020F8B500B30546164B1F68F7B945
:108994000E463C46B4420ED205EBC4035B68CBB131
:1089A40015F8340010F0800F16D1B8B1FEF736FE7A
:1089B400B0B90134EEE70C4B43F8375003EBC7036F
:1089C4005E607B1C074A136002E00E2700E0042768
:1089D4003846F8BD0E27FBE70B27F9E70F27F7E723
:1089E4000F27F5E7A43A0020A83A0020084B19689D
:1089F40061B110B501E021463CB10C680B79002B44
:108A0400F9D0034803F065FFF5E710BD704700BFD8
:108A1400CC3C002038B5054630B1104B1C68ACB1D5
:108A24000F4B01221A7004E07846FEF737FCF4E796
:108A340024683CB12379002BFAD154F8043C28462D
:108A44009847F5E7064B1B78022B00D038BDFFF79B
:108A5400CDFF034B00221A70F8E700BFCC3C002086
:108A6400C83C002010B5044630B100232372211DF8
:108A7400034803F003FF10BD7846FEF70FFCF4E74C
:108A8400CC3C002010B5044650B10A4B1B78013B86
:108A9400DBB2012B08D9211D074803F01AFF10BDD2
:108AA4007846FEF7FBFBF0E7024B02221A70012323
:108AB4002372F4E7C83C0020CC3C00200A88836879
:108AC4009B5A07339BB223F0030313449BB20288DF
:108AD400043A934200D900230B80704710B582B04A
:108AE40004468368CB1A02A921F8023DFFF7E6FF8A
:108AF400BDF80630A068184402B010BD00880438E0
:108B040080B2704743888268D018D15201238370A1
:108B140070478268002393704380838070470731D5
:108B240089B221F0030189B2428883889A4204D22F
:108B34009B1A99421CDC0020704710B59A420FD949
:108B44000488A41AA14215D98B4215D3032C03D946
:108B54008368134404229A7000234380184606E075
:108B6400826813449B784BB9FFF7D3FF002010BDF4
:108B7400042070470020FAE70420F8E70420F6E711
:108B840038B504460D468368828813448B4202D06C
:108B94007846FEF783FB0023AB70211D2046FFF7C8
:108BA4008DFFA288A36813449B78042B00D038BDA2
:108BB4000023A380FBE710B50C4683684288134466
:108BC4008B4202D07846FEF769FB0023A37010BDE8
:108BD40070B5064615460C46002944D0002E46D0F2
:108BE400B4F1005F08D94FF08053D3F80C3103F58A
:108BF4000023B4EB832F0ED3B4F5000F08D94FF044
:108C04008053D3F80C3103F50053B4EB832F02D314
:108C14007846FEF743FB6B1E2344B3F1005F08D98B
:108C24004FF08052D2F80C2102F50022B3EB822FD0
:108C34000ED3B3F5000F08D94FF08052D2F80C21AF
:108C440002F50052B3EB822F02D37846FEF726FBDF
:108C5400042D10D9358000237380B380B460043DA3
:108C64002580A37070BD7846FEF718FBB6E77846FA
:108C7400FEF714FBB4E77846FEF710FBEAE738B5D5
:108C84000446A0B16288A36813449B78012B12D0D8
:108C9400A388A1681944EFF3108572B68B78032B6F
:108CA4000DD02046FFF735FF05B962B638BD7846CA
:108CB400FEF7F4FAE6E77846FEF7F0FAE8E720462E
:108CC400FFF70CFFA368C31A638000238370EBE7EC
:108CD400F8B50E4615460446C0B1DEB16288A368F5
:108CE40013449B78012B19D0E5B12046FFF706FF0A
:108CF400A84219D329462046FFF711FF0746A0B919
:108D040029462046FFF7FEFE30600EE07846FEF767
:108D1400C5FAE2E77846FEF7C1FADFE77846FEF7E0
:108D2400BDFAE1E7092700E009273846F8BD70B528
:108D34000C4616460546B8B1D4B1A378012B1BD115
:108D44002388B3421CD3FEB126800223A370E91802
:108D54002846FFF7B3FE6A88AB889A4203D0AB6813
:108D6400134400229A7070BD7846FEF797FAE3E741
:108D74007846FEF793FAE0E77846FEF78FFADFE7E6
:108D84007846FEF78BFADEE77846FEF787FADBE7EC
:108D940038B50D46044650B16DB1A288A36813449A
:108DA4009A78022A0BD0032A0ED005200BE07846CD
:108DB400FEF774FAF0E77846FEF770FAEDE703225F
:108DC4009A702B60002038BD7846FEF767FA0020C1
:108DD400F9E710B5044640B1A288A3681344987813
:108DE400022814BF0020012010BD7846FEF756FA71
:108DF400F2E710B5044618B1A088A168014407E061
:108E04007846FEF74BFAF7E72046FFF767FE014680
:108E140088780328F8D0022814BF0020012010BD50
:108E240038B50C46054650B16CB1A378012B0ED071
:108E3400032B11D121462846FFF7A2FE38BD784600
:108E4400FEF72CFAF0E77846FEF728FAEDE721461C
:108E54002846FFF7B0FEF1E77846FEF71FFAEDE784
:108E640008B5064B986800221A605A609A60DA6066
:108E74001A615A619A6104F047FD08BDD03C002094
:108E840000B585B00A4BDB6802228DF800200193FF
:108E94004FF480530293074A6946012001F098F980
:108EA40018B1002005B05DF804FB0120FAE700BF0B
:108EB400D03C0020EC3C002000B585B00A4B1B6878
:108EC40002228DF8002001934FF480530293074A45
:108ED4006946012001F07CF918B1002005B05DF865
:108EE40004FB0120FAE700BFF03C0020EC3C00202A
:108EF400164BDA68137951795B1A03F57F2303F66D
:108F0400FF7302EB03339A4205D002F580520F4BF4
:108F1400DA600320704700B585B00D4B1B68012053
:108F24008DF8000001930B4B0393042302930A4A28
:108F3400694601F04DF918B1002005B05DF804FB55
:108F4400024B01221A760220F7E700BFD03C002032
:108F5400F03C0020F43C0020EC3C002000B585B03F
:108F64000C4BDA680C4B1B68043301208DF80000AD
:108F74000192039340F6FC730293084A694601F098
:108F840027F928B90120034B187605B05DF804FBD6
:108F94000020FAE7D03C0020F03C0020EC3C00200C
:108FA40000B585B00A4B1B6801208DF800000193C1
:108FB400084B039304230293074A694601F008F916
:108FC40018B1002005B05DF804FB0120FAE700BFEA
:108FD400F03C0020DC3C0020EC3C002010B584B0C8
:108FE400114BDA681478114B1B68043301208DF897
:108FF40000000193039202940D4A694601F0E8F8D7
:1090040080B90A4B1B6804F0FC041C440434064B6E
:109014005C61D9680A780A441A6100225A760120F0
:1090240004B010BD0020FBE7D03C0020F03C002041
:10903400EC3C002008B50023092B09D8064A52F855
:109044002320824201D00133F6E7044A536002E050
:109054007846FEF723F908BDDCF80300D03C002075
:1090640010B5214BDB6853B11F4B1B7E5BB91E4B04
:109074005B68092B15D97846FEF710F911E078469C
:10908400FEF70CF9F0E77846FEF708F9EFE7164B20
:1090940000225A60012C01D0032C23D1124B1B7ED9
:1090A40003BB114B5A68114B53F8223098470446BE
:1090B40002280DD00328EAD00128EBD10A4A5368CC
:1090C40001335360092BE5D97846FEF7E7F8E1E769
:1090D400054B1B7E1BB1044B02221A70DAE7FFF723
:1090E400BFFED7E710BD00BFD03C0020DCF8030072
:1090F400104B1B681B685A1E12F1030F18D8C3F3D8
:109104000B020AB10020704710B50B4AD36000234C
:10911400137653760124147093600848FFF78AFF8E
:109124000749204601F042F8FFF79AFF204610BD98
:1091340000207047F03C0020D03C0020858E0200C7
:109144004991020008B50B78032B06D00B4B1B7812
:10915400012B06D0022B0BD008BD084B00221A7637
:10916400F4E7064B1B7E002BF6D1FFF779FFF3E7FC
:109174000B78032BF0D1FFF773FEEDE7D03C002012
:1091840000B585B0174BDB6818784FF6FF7203F50E
:109194008051184404F080FEF0B10246114BD968A6
:1091A4000B780B44984219D00E4B5B7E93B10E4B57
:1091B40001208DF8000001920393042302930B4ACB
:1091C400694601F005F858B90120064B187605B038
:1091D4005DF804FB064BEBE70120F8E70120F6E716
:1091E4000020F4E7D03C0020BCFA0300EC3C002053
:1091F400B8FA030008B5104BDB681878002203F5B1
:109204008051184404F048FE08B1012008BD0A4BFF
:10921400DA68137951795B1A03F57F2303F6FF7338
:1092240002EB03339A4205D002F58052024BDA6016
:109234000320EBE70220E9E7D03C0020F0B585B03D
:10924400524BDE6872793379591E8A4200F0968057
:1092540006F580510D780D444D490968081D0F79B4
:1092640007449B1A03F57F2303F6FF731B0303F5DF
:1092740080531E446B88013B9BB247F6FE629342C7
:109284005CD92C4616E07846FEF708F815E024F47D
:109294007F6424F00F0404F5805423781C44A64210
:1092A40047D9A54247D26388013B9BB247F6FE6289
:1092B400934211D92388002BE5D0238804EB830340
:1092C40023F47F6222F00F029342E0D06288B2F569
:1092D400FE4FDCD01C46E2E725462FE07846FDF73A
:1092E400DDFF15E024F47F6424F00F0404F58054BA
:1092F40023781C44A64220D9A5423BD26388013B73
:109304009BB247F6FE62934211D92388002BE5D025
:10931400238804EB830323F47F6222F00F02934239
:10932400E0D06288B2F5FE4FDCD01C46E2E7254669
:1093340004E0002502E0002500E00025E5B1144B1F
:1093440019686A8801F58051384604F0A5FD07467E
:10935400B8B101200D4B18768DF8000001950D4B26
:109364000393042302930C4A694600F031FF50B979
:109374002C46CAE70025E1E7012000E0012005B002
:10938400F0BD0120FBE70020F9E700BFD03C00203E
:10939400F03C0020B4FA0300EC3C00202DE9F0413D
:1093A40086B06A4B1B692BB1684B5B6933B14FF0D4
:1093B400000848E07846FDF771FFF5E77846FDF7C9
:1093C4006DFFF4E77846FDF769FF15E025F47F6546
:1093D40025F00F0505F580552B781D44AE421CD9A8
:1093E400AC421ED26B88013B9BB247F6FE629342AD
:1093F40011D92B88002BE5D02B8805EB830323F4AC
:109404007F6222F00F029342E0D06A88B2F5FE4FE9
:10941400DCD01D46E2E72C4600E000241CB1009499
:1094240045E00024FAE700230093019B002B68D158
:109434004FF0010824B1628847F6FF739A4202D1C3
:10944400424B01225A76414B5B7E002B7AD1B8F114
:10945400000F75D13D4B5A6922F47F6727F00F073F
:10946400BF1A07F580571C69DE68337972799B1A35
:1094740003F57F2303F6FF731B0303F580531E4498
:10948400002301936388013B9BB247F6FE6293423B
:10949400C5D92546ADE77846FDF700FF22E024F460
:1094A4007F6424F00F0404F5805423781C44A642FE
:1094B400BBD92388019A02EB83029742B5D9009B5A
:1094C400634023F47F6323F00F03002BADD1638843
:1094D400013B9BB247F6FE618B42A6D801922388DA
:1094E400002BD8D0238804EB830323F47F6222F07B
:1094F4000F029342D3D06288B2F5FE4FCFD01C4600
:10950400D5E7124A526901208DF808000392009AA7
:10951400059204930E4A02A900F05AFE70B90B4951
:10952400019B23F003024B6913444B6114B1074BB5
:109534001C617FE77846FDF7B1FEF8E7002002E002
:10954400012000E0012006B0BDE8F081D03C0020FD
:10955400EC3C002008B54FF010235B69B3F1FF3FEA
:1095640003D04FF010235B6963B94FF08052516907
:10957400136903FB01F3A3F58053054A1360FFF756
:10958400B7FD08BD4FF010235B69A3F58053F2E7E4
:10959400F03C0020024B1878003018BF01207047BF
:1095A400D03C002010B504460E4B1B78ABB9237891
:1095B400032B02D07846FDF771FE0A4B9C60E268EB
:1095C400DA6000225A601A76012018705A76064929
:1095D40000F0ECFDFFF744FD10BD7846FDF75EFE9C
:1095E400E5E700BFD03C002049910200014B186818
:1095F400704700BFF03C002010B5044680B163689A
:109604001BB123680BB1A36813B97846FDF746FE76
:10961400A3685A1E134207D10023E360236110BDDF
:109624007846FDF73BFEEAE77846FDF737FEF3E7B9
:10963400F8B5F8B10446F9B18268FAB1EFF31085D0
:1096440072B6026980680244E668B24203D1C5B9C1
:1096540062B6042513E027686368013830401A466F
:1096640000FB037015F03EFEE3680133E36055B977
:1096740062B604E00E2502E00E2500E00925284626
:10968400F8BD0425FBE70025F9E770B5F0B1044601
:109694008268EAB1EFF3108572B60669C268964231
:1096A40010D0084621686268A368013B1E4006FB8F
:1096B400021108B115F016FE23690133236165B95F
:1096C40062B606E03DB962B6052502E00E2500E06B
:1096D4000925284670BD0525FBE70025F9E70000AC
:1096E400C0F30B0333BB39B301F6FF71090B134B02
:1096F4000222C3F80425114BD3F80034002BFAD00E
:1097040000220AE00D4BC3F808050C4BD3F80034D3
:10971400002BFAD000F5805001328A42F2D3074B75
:109724000022C3F80425054BD3F80034002BFAD0EB
:1097340000207047102070470920704700E0014066
:1097440010F0030F2FD111F0030F2FD182B312F0B9
:10975400030F2FD110B49208174B0124C3F804450A
:10976400154BD3F80034002BFAD002E00430043156
:109774002246541E52B10B68B3F1FF3FF6D003608A
:109784000D4BD3F80034002BFAD0EFE70A4B00213D
:10979400C3F80415084BD3F80034002BFAD0104654
:1097A4005DF8044B70471022104670471022FBE707
:1097B4000922F9E70922F7E700E0014001800023CC
:1097C400438042607047000038B5124C4FF4805516
:1097D4002A460021204615F0AEFD0F4B1C600AE01E
:1097E400002228212046FFF7E9FF23880833234479
:1097F4006360303D1C46502DF2D8083D05D0002250
:10980400A9B22046FFF7DAFF38BD7846FDF746FDDA
:10981400F5E700BFF83C0020F84C002008B508220A
:109824000221084803F0F1FE38B1074A916841600B
:10983400127B027203F022FF08BD044804F03CF8D6
:10984400FAE700BF044D00204C4D0020F832002000
:109854000E4B1B78CBB910B50D4B5C6804F5005466
:10986400B4F1807F00D910BD04220121094803F01E
:10987400CCFE30B14460054A0121117003F0FEFEB4
:10988400F1E7054804F018F8EDE77047604D002053
:109894004C4D0020044D0020E832002010B5044651
:1098A40008B1A04710BD7846FDF7F8FCF9E70000C1
:1098B40008B501210B4803F009FF20B9022109482A
:1098C40003F004FF28B1084803F0F6FFFFF7C0FFD8
:1098D40008BD064B00221A605A609A60DA601A6169
:1098E400F4E700BF044D0020183300204C4D002045
:1098F40000B58DB004918DF8082003900CA80223C4
:1099040000F82C3DFFF786F80DB05DF804FB00006D
:1099140010B58CB00C4682B94B88012B20D1134B67
:109924001B7833B16268124B5A60104B00221A70D4
:1099340016E07846FDF7B2FCF4E7032A12D12C2294
:10994400002101A815F0F7FC10238DF804300394CE
:10995400084BDA6805921B69069301A8FFF75AF8C9
:109964000CB010BD7846FDF799FCE8E7604D002087
:109974004C4D0020044D002038B503F0B5FF28B944
:1099840001F090FF0028F8D020BFF6E701F0C0FEF8
:10999400002211461A4803F092FD00252C4605E0EA
:1099A400051D02460021164803F089FD30B14388A5
:1099B400012BF5D0022BF4D1041DF2E7A4B19DB123
:1099C4002268104B9A6022791A73AC4201D9237928
:1099D40093B12A680B4B1A600A4B1A685A60FFF756
:1099E40037FF01F0B5FE38BD064B00221A609A60BD
:1099F4001A73FFF713FFEFE7024B00221A60EBE73D
:109A0400044D00204C4D002008B503F0AFFFA0F535
:109A1400805008BD00B587B00023009301930293E2
:109A2400039304930593FFF7EFFF00900123019341
:109A3400064B03936946064803F0F8FE10B907B0D5
:109A44005DF804FB034803F037FFF8E715990200BB
:109A5400044D00200833002038B50F4B00241C604F
:109A64005C609C60DC601C6101F0B0F90B4D6860C7
:109A74000B4BAB600B4BEB602C616C610A4B1C70A5
:109A84000A480B4B036000F0F9FD284601F0A0F8EA
:109A9400FFF7C0FF38BD00BF4C4D0020284D00200B
:109AA400819C020000879303614D0020404D0020FB
:109AB400559C020038B501F02BFE174B1B7B13BBE2
:109AC400154B9B7B23BB144B1A8A41F282639A4247
:109AD40004D8124B1B78A3B1012300E00123CBB1BE
:109AE4000D4D01232B7300242C82AB680133AB6032
:109AF400FFF794FEA9682A7B01392046FFF7F8FE98
:109B040002E00023EBE7082401F022FE204638BDE2
:109B14000824F9E70824F7E74C4D0020614D0020A4
:109B240010B501F0F5FD214B5B7B9BB11F4B9B7B7B
:109B3400F3B91E4B1A8A41F282639A4204D81C4B31
:109B44001B782BB1012300E001239BB1012302E028
:109B54000023FAE700231C461BB3144B00225A735C
:109B64001B7B4BB1012B0ED07846FDF797FB18E019
:109B74000023F0E70023EEE7FFF79CFF88B1784667
:109B8400FDF78CFB0DE0094B00201860586018733A
:109B9400188202469968FFF7ABFEFFF73FFEFFF716
:109BA40057FE01F0D5FD204610BD00BF4C4D0020EE
:109BB400614D002038B5254B1B7B002B36D1044664
:109BC400224B5B8A33BB1AB9204B9B688B4205D36B
:109BD40002B31E4B9B6801338B421BD21B4B9B6809
:109BE4002A338B4224D3194B9B7B0BBB174DA960A3
:109BF4002B606B602B8242F606526A826B732B7366
:109C0400FFF70CFEFFF724FE2A7BA9682046FFF726
:109C14006FFE0DE062B10D4B9B6801338B4207D19F
:109C24000A4B01225A73FFF77BFF01E0012B00D09E
:109C340038BD002AFCD1054B9B688B42F8D1034BFD
:109C440001225A73FFF76CFFF2E700BF4C4D00206E
:109C54000378042B00D0704743681B78002BFAD09C
:109C640010B58468027E437E012A14BF00220122BB
:109C7400416904F11000FFF79DFF10BD08B5214BA9
:109C84001B7B7BB1012B20D07846FDF707FB1D4AD7
:109C9400138A013313821B4B5B8A13B1013B194AAC
:109CA400538208BD174B1A8A41F282639A4204D840
:109CB400154B1B783BB1012300E00123002BE6D0B8
:109CC400FFF72EFFE7E70023F8E70E4B1B8A41F26C
:109CD4008262934204D80C4A127872B1012200E0E5
:109CE4000122002AD3D042F2B012934207D9054B85
:109CF40001225A73FFF714FFCDE70022F1E7FFF7C3
:109D04000FFFC4E74C4D0020614D002010B5184BE7
:109D14001A685B689A4225D20446154B1B7B012BBB
:109D240013D0144B9A4212D2114B1A685B68403B11
:109D34009A4214D2EFF3108072B60D4A1368591C7C
:109D44001160236090B962B610BD0B4BEAE7084B73
:109D540001225A73FFF7E4FE0028EBD1E4E7FFF792
:109D640077FDE7E7FFF774FD0F20EDE70020EBE751
:109D74004C4D0020FFFF7F0000E0FF0008B568B9EC
:109D84000C4B1B6893B10B4A1368013B136063B916
:109D9400094B00229A73FFF7C3FE06E0064B01222B
:109DA4009A73044A13680133136008BD7846FDF7BB
:109DB40075FAE8E7004D00204C4D002000B58DB049
:109DC400ADF808008DF8102003910CA8032300F8C7
:109DD4002C3DFEF71FFE0DB05DF804FB014B9868A7
:109DE400704700BF4C4D0020054B1B7B012B02D05C
:109DF400034B98687047024B98680138704700BF5E
:109E04004C4D0020044B9B68584010F0010F00D0CB
:109E1400013B1846704700BF4C4D0020014B187B96
:109E2400704700BF4C4D002038B50A4B1B7873B9FE
:109E3400084B01221A70084DA8602973FFF7EEFC45
:109E440000242C606C60FFF703FD204638BD082019
:109E5400FCE700BFFC4C00204C4D00202DE9F041F4
:109E6400002724E02449BC2303FB04F3CA5A01322B
:109E7400CA520221284602F073FB01360221284609
:109E840002F03EFB80B11C4ABC2303FB0423D3F83D
:109E94000880B8F1000FE5D0BC2303FB04F3D25AC9
:109EA40001463846C047DDE78EB90137FFB2022FBD
:109EB4001FD83C46BC2303FB07F308330E4D1D4457
:109EC40004350221284602F01BFB0026DAE70021B4
:109ED400284602F0ADFB0828E7D1074BBC2202FB61
:109EE4000434A368002BE0D0002204493846984784
:109EF400DBE70120BDE8F0816C4D002004F903008C
:109F040008B5082383731023437300F11C034361D2
:109F14000323037300F1180303610C3002F05AFBAE
:109F240008BD000008B50378012B06D0022B07D02A
:109F34007846FDF7B3F9002001E04FF4A97008BD9D
:109F44000048FCE7645E010008B50278012A07D0E6
:109F5400022A13D07846FDF7A1F94FF4FA7308E00A
:109F640083685B1A98084FF4A97303FB00F303F5A5
:109F7400FA730748984228BF184608BD83685B1ADD
:109F8400180B044B03FB00F303F5FA73F1E700BF6E
:109F9400A0860100645E010010B5044601210C3066
:109FA40002F0AEFAA0B10D4AC4F89C200022C4F815
:109FB400A0206168FFF7C8FFC4F8A800C4F8AC404B
:109FC400012384F8B83004F19C000BF0DFFF00B9E2
:109FD40010BD7846FDF762F9FAE700BFE1A0020080
:109FE400F8B506460C46174615680378012B18D1B8
:109FF4001249A1FB0431C9098900B468641B8C426D
:10A0040000D30C468CB1706825F00305F168224634
:10A0140029442844FFF794FB58B93B681C443C602E
:10A02400F8BD7846FDF73AF9E2E77846FDF736F9E8
:10A03400E9E77846FDF732F9EFE700BFEB5DF26040
:10A04400F8B507460C46164615680378022B16D158
:10A05400114BA3FB04231B0C1B03BC68641B9C4215
:10A0640000D31C467CB1786825F0030521462844BA
:10A07400FFF736FB58B933681C443460F8BD7846A2
:10A08400FDF70CF9E4E77846FDF708F9EBE77846C5
:10A09400FDF704F9EFE700BFB77609BB38B505460D
:10A0A4000C4611462378012B06D0022B0FD078469C
:10A0B400FDF7F4F8002304E0021D2046FFF790FFAB
:10A0C400A3686868984214BF0020012038BD021DAF
:10A0D4002046FFF7B5FFA368F3E700002DE9F84336
:10A0E4000F46D1F8A850234B1B7863B90646A5F553
:10A0F400FA7501F10C090121484602F001FA804683
:10A1040040B1002422E00BF07DFF002387F8B83033
:10A11400BDE8F8837846FDF7C1F8F2E70BF072FF6B
:10A124000121484602F01CFA00237B6087F8B8300E
:10A13400114B186801F04EFB3846FFF72DFFE7E797
:10A144004046FFF7EFFE2044A8420CD82A1B4146A4
:10A154003846FFF7A3FF0028E0D100F037FE841B48
:10A16400EED5341AECE70BF04DFF3846FFF714FF39
:10A17400CEE700BF684D0020644D002010B50848AC
:10A1840001F008FB074B1860002406E0064BBC20D6
:10A1940000FB0430FFF7B4FE0134022CF6D910BDE5
:10A1A400619E0200644D00206C4D002038B50446C9
:10A1B4000D46022805D8054BBC2202FB0434A560D9
:10A1C40038BD7846FDF76AF8F5E700BF6C4D00200E
:10A1D4002DE9F84306460C461746022816D8CCB19A
:10A1E4002378012B1AD0022B3ED16368C3F30B03EF
:10A1F400002B31D1A368C3F30B03002B30D1A36828
:10A20400002B34D17846FDF749F830E07846FDF765
:10A2140045F8E4E77846FDF741F8E1E7636813F0B1
:10A22400030F0DD1E36813F0030F0DD1A36813F0EE
:10A23400030F0DD1A368D3B97846FDF72FF816E0C4
:10A244007846FDF72BF8EDE77846FDF727F8EDE7BC
:10A254007846FDF723F8EDE77846FDF71FF8C9E7E0
:10A264007846FDF71BF8CAE77846FDF717F8EFF3D1
:10A27400108872B6BC2505FB06F505F10803204DD0
:10A284001D4404350021284602F03AF9814668B39A
:10A294000021284602F064F920686168A268E36836
:10A2A400C9F80000C9F80410C9F80820C9F80C302E
:10A2B4002FB1134ABC2303FB06235B883B80104A5F
:10A2C400BC2303FB06235A8801325A8093F8B83022
:10A2D40073B90C4B1B780BB100200AE0084BBC206F
:10A2E40000FB0630FFF758FE002002E0042000E0E7
:10A2F4000020B8F1000F00D162B6BDE8F88300BFBA
:10A304006C4D0020684D002018B1830B024AD05CCC
:10A3140070470020704700BF14F9030012DF704734
:10A3240000B583B01378A3B1042B14D1072110F81E
:10A33400013C163B152B31D8DFE803F0593030309F
:10A344003030303030303030303030303030302E0B
:10A354000F3A517DEBE70021E9E7022901D00729F3
:10A364001CD110F8021C013901F05AFEB0B1264B81
:10A374001B6813F0400F11D0244B1B68012B0DDD1B
:10A38400234BD3F804350190224A00928A222249B1
:10A39400022002F035FB01E0022902D003B05DF88F
:10A3A40004FB10F8021C0139C9B211F0DDFCF5E719
:10A3B4000229F3D110F8021C0139C9B203F0DEFC02
:10A3C4000028EBD0104B1B6813F0400FE6D00F4B66
:10A3D4001B68012BE2DD0E4BD3F8043501900F4AC4
:10A3E40000929D220C49022002F00AFBD6E7018864
:10A3F4004FF6E4639942D1D110F8021C03390230BC
:10A40400FCF79CFECAE700BF383300203433002039
:10A4140000B0004064F9030057F9030090F9030009
:10A4240000B58DB02C22002101A814F084FF0D2367
:10A434008DF8043001A8FEF7EDFA0DB05DF804FBC9
:10A4440070B58AB00CF022FB58B3064600238DF891
:10A45400103005AC05460FCD0FC42B682360727D08
:10A46400052A04D9337D03F00F03072B20D1184BA1
:10A474001B689BB104AB0393337DC3F303038DF8D3
:10A484000430737D062B1DD9063B8DF8053006F18B
:10A494001D0302930E4B1B6801A8984730460CF02D
:10A4A400D5FA0CF00DFB80F00100C0B20AB070BD0B
:10A4B400307D04AB063A06F11D0100F00F000BF0ED
:10A4C400C1F8D4E700238DF805300293E2E700BF1A
:10A4D400A44F002070B582B0304B1B78002B55D1AF
:10A4E400002857D0067A0F2E01D0072E54D10446E7
:10A4F400C06870B1FCF7E4FE0DF10700FFF70EFF32
:10A504000546002843D19DF80730012B04D00225CD
:10A514003DE0FCF7E3FEEFE7FCF7F6FE00F044FB5A
:10A52400304601F0BDF8E07800F024F900F0C2FFF5
:10A534000BF0EAFC1A480CF05FFB0BF021FAFFF772
:10A544001DFE02F035FF174803F014FA04F082FCF4
:10A55400204601F041FC2046FDF7E6FE03F08EFFA5
:10A564002046FFF731F9FCF7E9FD18B1062801D0C0
:10A5740005460CE000F048FD0B480BF045F80B4B8A
:10A5840000221A60054B01221A7000E008252846B3
:10A5940002B070BD0E25FAE70725F8E7A14F0020A9
:10A5A40045A4020025A4020028330020A44F002063
:10A5B40010B50E4B1B789BB10D4B1B7893B900F073
:10A5C4009FFF48B90BF0C2FC044660B90CF0FEF9D9
:10A5D400074B01221A7006E07846FCF75FFEF1E7AC
:10A5E400082400E00824204610BD00BFA14F00202D
:10A5F400A04F002010B5094B1B785BB10BF0B6FCE3
:10A60400044640B90CF0F8F900F0E4FF034B0022D3
:10A614001A7000E00824204610BD00BFA04F00209F
:10A6240030B583B004460D460E4B1B6813F4804FBF
:10A6340003D00D4B1B68062B05DC29462046FDF78D
:10A64400DBFE03B030BD094BD3F80435084A019250
:10A65400084A009240F2B1120749072002F0D0F9EB
:10A66400EBE700BF383300203433002000B0004053
:10A6740018F9030098F6030057F9030008B5FEF72C
:10A68400F1F908BD08B500F0EBFE002008BD08B5DF
:10A6940005F0AAFF08BD0000064A136801331360E1
:10A6A400B3F1704F02D0034B186870471346012270
:10A6B4001A60F8E7A84F002010B5044618B100232B
:10A6C4002360636010BD7846FCF7E8FDF7E738B512
:10A6D4000C46054668B184B100236360EFF3108330
:10A6E40072B62A686AB16A6854606C6003B962B66B
:10A6F40038BD7846FCF7D2FDEDE77846FCF7CEFD91
:10A70400EAE72C60F1E710B5044658B1EFF3108383
:10A7140072B6206808B142682260226832B103B977
:10A7240062B610BD7846FCF7B9FDEFE76260F6E764
:10A7340010B5044608B1206810BD7846FCF7AEFD9C
:10A74400F9E735DF7047000008B54FF0FF30FFF739
:10A75400F8FFBFF34F8F0549CA6802F4E062044B67
:10A764001343CB60BFF34F8F00BFFDE700ED00E064
:10A774000400FA05072814D8DFE800F0080C1504D3
:10A78400110F0A066420704714207047FA2070479E
:10A794001E2070474FF4FA707047322070474B20E8
:10A7A4007047FA2070479620704746DF7047F8B527
:10A7B40004460D464B1EDBB2012B09D80022226150
:10A7C4006261A261E2612046FFF7EFFF012616E015
:10A7D4007846FCF763FDF1E7CA5CC8185200D2B2B0
:10A7E400407842EAD012CA5401339BB20E2BF3DDF7
:10A7F400CB7B5B00CB73002F08DB0136F6B2AE4295
:10A804000BD8214611F9207F0023EFE794F82F306D
:10A8140083F0870384F82F30EFE7F8BD2DE9F0418A
:10A8240090B084460C4696461F4602F10F06361138
:10A834001FFA86F804AD0068DCF80410DCF8082080
:10A84400DCF80C300FC50EF00F05B8F1000F02D084
:10A8540085B1002300E0002398466BB1012104A8D0
:10A86400FFF7A5FFB8F1000F1BD0B0B2013800010B
:10A8740010230EE00123EFE70221F0E7013B9BB236
:10A884002218D25C10A9194411F8101C4A400DF882
:10A894000320002BF2D100250C950D950E950F95F4
:10A8A40034E0B1B20139ADB22A4604EB0111684675
:10A8B40014F018FD80230DF805306B1C03E0002212
:10A8C4000DF8032001330F2BF9DD10230AE0013BBF
:10A8D4009BB21DF8032010A9194411F8101C4A401A
:10A8E4000DF80320002BF2D1D5E7013B9BB210AA4F
:10A8F4001A4412F8102C2118C95C4A4008A9CA54F9
:10A90400002BF2D104A8FFF750FF0135B3B2013B8D
:10A91400AB4202DD28011023F2E710230AE0013BD9
:10A924009BB210AAD11811F8402C11F8101C4A40FF
:10A9340008A9CA54002BF2D104A8FFF736FF0CACC7
:10A944000FCC38607960BA60FB6010B0BDE8F0816C
:10A9540070B51E4E10E063693360002363611B4AC7
:10A96400D368591ED160ABB1184A9368013B936018
:10A9740000232370032D11D034682CB3134B9B6830
:10A9840013B32578EDB2EB1EDBB2012BE3D904F14E
:10A994001406F1E77846FCF781FCE5E723781BB160
:10A9A4002378DBB2062B0BD1636913B17846FCF72D
:10A9B40075FC01232370054B5A6862615C60DBE718
:10A9C4007846FCF76BFCEFE770BD00BFB04F00208A
:10A9D40010B50446436913B17846FCF75FFC164B87
:10A9E4001B684BB16068144B1B685B68C31A002B6F
:10A9F40002DB114B19680DE00F4A136863611460A0
:10AA0400D3680133D36003B110BD7846FCF746FC2C
:10AA1400FAE719464B691BB15A68121A002AF8DB87
:10AA240063614C61044AD3680133D360002BEBD1DA
:10AA34007846FCF733FCE7E7B04F0020114B5B6826
:10AA4400FBB110B50AE00023237004E00223237055
:10AA54002046FFF7BDFF0B4B5B688BB1094B5C686D
:10AA640062695A60002363612378DBB2052BEAD064
:10AA74002378DBB2012BE9D07846FCF70FFCE5E73D
:10AA840010BD7047B04F002038B505461BE0626921
:10AA9400234B1A6000226261DA68511ED9602AB31E
:10AAA400A3683BB306232370A3682169284698470B
:10AAB40000F08CF90546FFF74BFFFFF7BFFF237843
:10AAC400DBB2062B1AD0164B1B6843B3144B1B681E
:10AAD4005B685B1B642B22D5114B1C682378DBB2AB
:10AAE400022BD4D07846FCF7D9FBD0E77846FCF7A4
:10AAF400D5FBD5E77846FCF7D1FBD3E7E26812B97A
:10AB040000232370DFE76368134463605B1B642BDB
:10AB1400F9D4022323702046FFF75AFFD3E738BD48
:10AB2400B04F002008B5124B1B6873B1104B1B6863
:10AB34005B68C31A13F1640F08D402230D4A00F1B1
:10AB44006401012000F006F970B908BD084B1968CA
:10AB54000223084A4968012000F0FCF80028F4D0D8
:10AB64007846FCF79BFBF0E77846FCF797FBECE7AD
:10AB7400B04F00209DAB020008B5FFF7E9FEFFF7D8
:10AB84005DFF00F023F9FFF77FFF00F01FF9FFF7E7
:10AB9400C9FF012008BD000008B5024B186800F089
:10ABA40019FE08BDAC4F002008B5064B00221A6000
:10ABB4005A609A60DA60044800F0ECFD034B1860B8
:10ABC40008BD00BFB04F00207DAB0200AC4F002099
:10ABD40038B50446F0B1A36803B3EFF3108572B639
:10ABE4000023636123781BB12378DBB2062B19D1D0
:10ABF400636913B17846FCF751FB012323700B4BB7
:10AC04005A6862615C6005B962B6094B186800F065
:10AC1400E1FD38BD7846FCF741FBDCE77846FCF7FC
:10AC24003DFBDAE77846FCF739FBE1E7B04F00205B
:10AC3400AC4F002038B50446E0B1EFF3108572B68E
:10AC44002378DBB2062B19D02378DBB2012B1AD080
:10AC54002378ABB12378033BDBB2012B03D90B4A36
:10AC640093680133936004232370094B186800F040
:10AC7400B1FD05E07846FCF711FBDEE70023237005
:10AC840005B962B638BD05232370F9E7B04F00203B
:10AC9400AC4F002070B50E460446E0B1EFF31085CA
:10ACA40072B62378DBB12378DBB2062B17D0237876
:10ACB400DBB2012B30D02378DBB2052B2CD02378E8
:10ACC400033BDBB2012B03D9154A9368013393602C
:10ACD4000323237014E07846FCF7E0FADEE72378D8
:10ACE4001BB12378DBB2062B12D1636913B178460A
:10ACF400FCF7D4FA01232370094B5A6862615C6043
:10AD04006660084B186800F065FD05B962B670BD51
:10AD14007846FCF7C3FAE8E701232370F0E700BFA5
:10AD2400B04F0020AC4F002010B4094B00F150028A
:10AD3400002443F8224000F110040122A240C3F889
:10AD4400042300F5A87043F820105DF8044B704705
:10AD540000800040022825D838B533F0030423D1FD
:10AD6400EFF31084124D2C6072B6124C44F820207C
:10AD7400114A42F82010114A1354114B002243F88F
:10AD84002020104B1B7833B10F4B1B68CA1A07D411
:10AD94001146FFF7C9FF064B186838B962B604E0DC
:10ADA4005A1AF5E7072070470A2038BD0020FCE74F
:10ADB400E44F0020C44F0020D84F0020C04F002093
:10ADC400EC4F0020D04F0020D44F0020EFF310832D
:10ADD4000C4A136072B60C4B1B787BB10B4B0022F0
:10ADE400C3F84C210122DA64D3F84C05084B1B68E4
:10ADF4001844044B1B6803B962B67047054B1868C6
:10AE0400F7E700BFE44F0020D04F0020008000404F
:10AE1400D44F0020E84F002070B5002418E01F4BE9
:10AE2400002243F82420012303FA05F51C4BC3F840
:10AE34000853FFF7CBFF1B4B1B5D13F0020F21D010
:10AE4400B04704F15003164A002142F8231001349C
:10AE5400022C21D804F15003114A52F82330002B5C
:10AE6400F5D0D2F8043304F11005EB4013F0010FD0
:10AE7400EDD00A4B53F82460002ED0D17846FCF76D
:10AE84000DFACCE70146304600F02EFC0028D8D05D
:10AE94007846FCF703FAD4E770BD00BFC44F002026
:10AEA40000800040C04F002070B50546002414E027
:10AEB400981A27E05E1A29E02946184600F014FC87
:10AEC400002836D12A4B53F824302BB101221A60C2
:10AED400274B002243F824200134022C3AD8254B76
:10AEE40004F5A872002143F8221004F1500243F83B
:10AEF400221053F82230204B53F824201F4B1B6898
:10AF0400D01AD5D405F17801CE1AD3D4864214D9F7
:10AF14001B4B53F82430002BD4D0194A002142F89B
:10AF24002410184A125D12F0020FC5D02846984723
:10AF3400C8E77846FCF7B2F9C4E7114B53F824305C
:10AF4400002BC9D0E0B2511B02D4FFF7EDFEC3E7DA
:10AF5400A91AFAE70C4B1B681BB90C4B4FF480720F
:10AF64001A60064B1D600A4B01221A7070BD00BFA7
:10AF7400EC4F002000800040D84F0020D44F002028
:10AF8400C44F0020C04F0020E44F002000E100E047
:10AF9400D04F0020002300E00133022B0ED80F4ACB
:10AFA400D25C12F0010FF7D000220C49CA540C49AC
:10AFB40041F823200B4941F82320EDE70A4B1860A0
:10AFC4000A4B00221A700A4B4FF0FF32C3F80823D1
:10AFD400084B4FF48072C3F880217047C04F0020A3
:10AFE400C44F0020EC4F0020E84F0020D04F002039
:10AFF4000080004000E100E0024A1368013313605E
:10B00400704700BFF84F002010B50023084A1360B2
:10B01400084C094AA260094AE2602361FFF7D6FEA0
:10B0240000F5C330A03060602046FFF7D1FD10BDAD
:10B03400F84F0020FC4F0020FDAF0200A086010065
:10B0440030DF704731DF704710B402684368A2EB09
:10B054007312846883EAF4330360C1680C44446067
:10B06400114481601344C36018465DF8044B704773
:10B0740070B582B00D46064608B100240BE0784650
:10B08400FCF70CF9F9E79DF807103019FFF7DAFF20
:10B094009DF807301C44A5420DD90DF10700FFF7B8
:10B0A400CFFF9DF80730002BF7D02A1B9342EAD933
:10B0B4008DF80720E7E702B070BD000030B583B01B
:10B0C4000546002402A840F8044D0421FFF7D0FFF0
:10B0D400074B2B60019B6B60AB60EB6003E0284681
:10B0E400FFF7B2FF0134132CF9D903B030BD00BF10
:10B0F400ED5EEAF108B5A0F1C8039BB2632B0AD94F
:10B10400A0F596739BB2632B08D9B0F5C87F08D31A
:10B1140000F07AFE01E00FF009FD08BDFDF778FBB1
:10B12400FBE70620F9E708B5A0F1C8039BB2632B3F
:10B134000AD9A0F596739BB2632B08D9B0F5C87FE2
:10B1440008D300F0B3FE01E00FF002FD08BDFDF7E7
:10B15400DBFBFBE70620F9E748DF704749DF704770
:10B164004ADF70472DE9F00F1F4BD3F80465002721
:10B17400837AA3BB1D4BD3E90023B41A24F07F4A7E
:10B184004FF0000B4FEA4A124FEA4B13B2EB0A029C
:10B1940063EB0B03590241EAD2514FEA422C0D46AC
:10B1A4001CEB0A0145EB0B024FEA821949EA91694B
:10B1B4004FEA81181346B8EB010269EB03031AEB5B
:10B1C40002044BEB0305E30B43EA45424368134493
:10B1D4004360064BC3E90067BDE8F00F70470023E6
:10B1E40083720268F2E700BF00B0004048500020BC
:10B1F40010B504460023C3600361FFF7B3FF23685F
:10B20400084A926822600121217503B9064B991AF4
:10B21400A161B1F57A7F01D39A4202D94FF47A73CE
:10B22400A36110BD3450002080969800094B03227E
:10B234001A75094A9A611A6840F6D8639A4204D882
:10B24400054B40F6D8629A607047034B43F2B062F4
:10B254009A607047145000203450002008B50B4BFE
:10B264001B78012B05D0022B0BD07846FCF716F87F
:10B2740003E00223037501238372044B00221A7036
:10B2840008BD03230375024B8361F6E74550002094
:10B294003450002038B50546002404750123437258
:10B2A4004068FFF701FE0AF019FF6B682A6813442F
:10B2B4000A490968283101FB02F1094AA2FB01216C
:10B2C400A3EB91410323074A78392046FFF742FD57
:10B2D40000B938BD7846FBF7E1FFFAE730500020AB
:10B2E40083DE1B4331B2020010B50C4631B1036951
:10B2F400013303618269036813440360C368013343
:10B30400C36001220275826952088261012B0DD04B
:10B31400022B19D082690368134417498B4222D83F
:10B3240040F6D7639A4221D800231DE0B2F5FA7F94
:10B3340005D040F6D8639A42ECD88361EAE7002C42
:10B34400F7D100238361E5E70369022B06D0012BC3
:10B35400E0D1002CDED100238361DBE70268064BD9
:10B364009B1A8361D6E7002313B110BD0123FBE7C9
:10B37400FFF790FFF9E700BF80969800437A1BB966
:10B384000E4B00221A70704710B504460AF0C2FE34
:10B394006068226810440A4B1B68283303FB02F3DD
:10B3A400084AA2FB0323A0EB93407838FFF7F2FD91
:10B3B40000236372014B00221A7010BD4450002018
:10B3C4003050002083DE1B4308B5224B01221A7241
:10B3D400214B1B7813B1214B1B781BB31D4B00224F
:10B3E4001A7504281AD8DFE800F00314110C0700BA
:10B3F4001848FFF7FDFE1EE001211648FFF774FF11
:10B4040019E000211348FFF76FFF14E00AF020FE53
:10B4140011E0FFF701FD0AF04FFE0CE07846FBF760
:10B424003DFF08E0FFF7D2FC0A4B5A68801A186007
:10B434001846FFF713FF074B1B7D023BDBB2012BC2
:10B4440004D9044800230372143008BD0148FFF7EF
:10B4540095FFF6E71450002045500020445000208A
:10B4640008B5043803280DD8DFE800F00D190902E7
:10B47400FFF774FE30B17846FBF710FF02E0784620
:10B48400FBF70CFF08BD0A4840F6D8638360FFF75A
:10B4940067FE0028F6D07846FBF700FFF2E7044881
:10B4A400FFF75EFE0028EDD07846FBF7F7FEE9E7EC
:10B4B4003450002010B40D4A00231370137101217D
:10B4C400517143F2B064946043F69824D460084AFE
:10B4D4001060084A1370084A1370084A13725372B2
:10B4E4001360917253605DF8044B70473450002030
:10B4F40030500020445000204550002014500020BB
:10B5040008B50648FFF728FE034608B1184608BDEB
:10B514000348FFF725FE0346F8E700BFCDB302005A
:10B5240034500020084B1B7D032B09D0074B1B789C
:10B53400012B07D0022B01D0002070470120704757
:10B54400012070470120704714500020455000200E
:10B55400014B5868704700BF145000200E4B5B7AB3
:10B564000BB90020704710B50B4B5C681A68144483
:10B574000A4B1B68283303FB02F3094AA2FB03238B
:10B58400A4EB9344783CFFF721FC0346201A00D433
:10B5940010BD181BFCE700BF1450002030500020E1
:10B5A40083DE1B43014B187A704700BF1450002000
:10B5B400EFF3108372B6054A527A22B1044A4FF46B
:10B5C4008071C2F8001103B962B6704714500020AC
:10B5D40000E100E008B5034B01221A70FFF7E8FF11
:10B5E40008BD00BF4550002008B5034B02221A7065
:10B5F400FFF7DEFF08BD00BF4550002008B5094B2A
:10B604001B782BB148B9084B1B7813B1012300E018
:10B614000023044A107013B908BD0023F9E7FFF7AB
:10B62400C7FFF9E7445000204550002008B50378CF
:10B63400012B10D013B1022B06D008BD4368002B98
:10B64400FBD080689847F8E74368002BF5D0C168C1
:10B6540080689847F1E74368002BEED080689847EC
:10B66400EBE70000044B1B780F2B04D0034B4FF483
:10B674008022C3F8002170479451002000E100E0CB
:10B6840010B501460548FDF7D3FF20B90446FFF77E
:10B69400E9FF204610BD0424FBE700BF5050002002
:10B6A40010B50C4C20700C480C4B03601023436005
:10B6B4008360FDF7A1FF0A48FEF7FEFF23780F2BF6
:10B6C40007D05B01DBB2074A82F812334FF48023C0
:10B6D400136010BD9451002050500020645000208D
:10B6E4009851002000E100E030B585B00C460546D5
:10B6F40048B100238DF80030019502946846FFF7A5
:10B70400BFFF05B030BD7846FBF7C8FDF1E7000088
:10B7140010B5EFF3108472B60A490A68531C0B6023
:10B7240042B9094A12780F2A04D0084A4FF48021FA
:10B73400C2F8801013B104B962B610BD7846FBF7A5
:10B74400ADFDF8E7645100209451002000E100E0D1
:10B7540010B5EFF3108472B60B4B1B687BB10A4A29
:10B764001368013B13603BB9084B1B780F2B03D0C4
:10B77400074B4FF480221A6004B962B610BD7846B4
:10B78400FBF78CFDEBE700BF6451002094510020CF
:10B7940000E100E010B5044680B10C4B1B68082B97
:10B7A40010D8EFF3108372B6084A1068411C116078
:10B7B400074A42F8204003B962B610BD7846FBF749
:10B7C4006DFDEAE77846FBF769FDEAE7685100207A
:10B7D4006C51002038B504460D4B1B68834213D9C5
:10B7E400EFF3108572B661090A4A04F01F040123BD
:10B7F40003FA04F452F82130234342F82130FFF7CE
:10B8040031FF05B962B638BD7846FBF747FDE7E777
:10B81400685100209051002070B50D46164604462C
:10B8240058B175B1EFF3108372B6A560E6600022DB
:10B834002274246003B962B670BD7846FBF72EFD0E
:10B84400EFE77846FBF72AFDECE7000038B504463D
:10B8540090B1A368A3B1EFF3108572B6237C9BB9B2
:10B864000123237421460948FEF731FFFFF7FAFE4E
:10B87400002005B962B638BD7846FBF70FFDE8E74E
:10B884007846FBF70BFDE6E71120F2E7985100201C
:10B8940010B5044608B1207C10BD7846FBF7FEFCC9
:10B8A400F9E7000070B584B02C4B1B7823B901254F
:10B8B4002A4B1D7000240AE07846FBF7EFFCF6E7FC
:10B8C400274B53F8243098470646F0B10134254BF2
:10B8D4001B68A3421ED96109234A52F8213004F09F
:10B8E4001F00C34013F0010FF0D0EFF3108372B6C2
:10B8F400012606FA00F052F8216026EA000642F812
:10B904002160002BDCD162B6DAE72046FFF762FF44
:10B914003546DBE71548FEF7F6FE07E0A368E06866
:10B924009847002323741148FEF7EDFE50B10468D4
:10B93400237C002BF2D17846FBF7B0FCEEE7684697
:10B94400FFF774FE69460A48FDF79FFE0028F6D00B
:10B95400024B00221A70284604B070BDA05100208A
:10B964006C51002068510020905100209851002013
:10B974005050002008B5FFF795FF08BD46DF70471B
:10B9840070B58CB003460E4615466C46006859687F
:10B994009A68DB680FC430687168B268F3680FC4D2
:10B9A4006846FFF7EBFF08AC0FCC28606960AA601B
:10B9B400EB600CB070BD08B5FEF730FF08BD08B5EC
:10B9C40002F0ABF808BD08B502F0E1F808BD38B5DF
:10B9D400032900F29380DFE801F00235356719701E
:10B9E400817A5A7861F306025A70C17AD2B261F34D
:10B9F400C7125A70C168C1F3074201F47F4422435D
:10BA0400090401F47F010A4300219A70C2F3072458
:10BA1400DC70120C1A710489220A42EA0422A3F887
:10BA24000520D971197201690A0202F47F0242EAFF
:10BA34000162080A00F47F40024342EA1162C3F83B
:10BA4400092038BD1970597801F0800162F3C711DB
:10BA54005970C168C1F3074201F47F4422430904C9
:10BA640001F47F010A439A70C2F30721D970120CC2
:10BA74001A7101890A0A42EA0122A3F805204188C1
:10BA84000A0A42EA0122A3F8072001690A0202F421
:10BA94007F0242EA0162080A00F47F40024342EA5C
:10BAA4001162C3F80920CCE7197000245C70C168E6
:10BAB400C1F3074201F47F452A43090401F47F01DD
:10BAC4000A439A70C2F30721D970120C1A710189C2
:10BAD4000A0A42EA0122A3F80520DC711C720169FA
:10BAE4000A0202F47F0242EA0162080A00F47F407B
:10BAF400024342EA1162C3F80920A2E77846FBF741
:10BB0400CDFB9EE770B584B00E461446054668B179
:10BB140062B10023009301930293039323463246B8
:10BB240029466846FFF747FF04B070BD7846FBF727
:10BB3400B5FBEEE7F0B585B00F4614461D46064644
:10BB440018B112B10BB10B9B13B97846FBF7A6FBE6
:10BB54006B463A4631462046FFF72DFF0B9B9DF876
:10BB6400282029466846FFF726FF05B0F0BD0000EF
:10BB74002DE9F04786B000AF88461546994604463D
:10BB840008B101B113B97846FBF788FB05F111063A
:10BB940005F1100A05F11803DB086A46A2EBC3039A
:10BBA4009D46254B1B6807F1180040F8043D6A4682
:10BBB4000421FFF7A7FF3B1D102221466846FFF72B
:10BBC400FAFE2A464146684613F08CFB01230DF821
:10BBD4000530EA186B4692B26946381DFFF7EBFE52
:10BBE4009DF80F3003F07F034C4604F8013B2A46CE
:10BBF400414604A813F076FB02230DF80A30B6B2CE
:10BC0400234632466946381DFFF7D5FE2068616831
:10BC1400A268E368009001910292039303230DF854
:10BC24000A3009F1110332466946381DFFF7C3FE95
:10BC34001837BD46BDE8F087BCF9030070B588B07D
:10BC44000D46064600B3F9B1114C6368039304AA88
:10BC5400042103A8FFF756FF04AB1022314618460F
:10BC6400FFF7A9FE083494E8030001908DF808104A
:10BC740004AB052201A91846FFF79DFE06AB03CBD2
:10BC84002860696008B070BD7846FBF707FBDBE706
:10BC9400BCF9030070B586B00D460646F8B1F1B1A3
:10BCA400114C2369019302AA04210DEB0100FFF753
:10BCB40029FF02AB102231461846FFF77CFE636968
:10BCC40006A941F8183D02AB04221846FFF773FE9B
:10BCD4009DF8173003F03F032B7006B070BD784613
:10BCE400FBF7DCFADCE700BFBCF9030010B504463F
:10BCF40058B123787BB1E368B3F1807F0DD294F916
:10BD04000A30002B05DB012006E07846FBF7C6FA73
:10BD1400EFE7002000E0002010BD0020FCE730B574
:10BD240087B00446037B8DF8043002688368D27AB6
:10BD340022B30822134409330293236803936368EC
:10BD4400049305A901A802F0F7F8E0B1237B012BC5
:10BD540009D02568FEF748F8286120680C30FDF703
:10BD6400D5FF054660B92168059800F0B8F9059B30
:10BD7400093323610025284607B030BD0422D9E7E2
:10BD840002F056F9F7E70425F5E7000030B583B073
:10BD94000F4B1D7875B1837A012B16D904460378AD
:10BDA400012B0AD00B4B1B6823B1A27A618820892E
:10BDB40098470546284603B030BD6946408809F0D7
:10BDC4009DFB0028EED00025F4E70025F2E700BF34
:10BDD400A8510020A451002008B560B14268084B66
:10BDE4001A60084B01221A70FDF736FEFDF7C4FDF8
:10BDF40002F014FD08BD024B00221A60F1E700BFF7
:10BE0400A4510020A8510020002945D008B5A0F570
:10BE1400C870062842D8DFE800F00A1B0424302A40
:10BE240039004968012003F069F8002008BD1E4A62
:10BE340012784B689A4201D10020F7E7003318BF0B
:10BE44000123194A1370012002F0F4FA0020EDE7EF
:10BE54004968072924D8C9B2012003F029F8002031
:10BE6400E4E70979012003F073F80020DEE749686C
:10BE7400002003F043F80020D8E74968072911D8C7
:10BE8400C9B2002003F014F80020CFE7097900209C
:10BE940003F05EF80020C9E70E2070470520C5E7CF
:10BEA4000720C3E70720C1E7A8510020002931D0AB
:10BEB40010B50C46A0F5C87005282DD8DFE800F0B1
:10BEC4000B12032C221A012003F02CF860600423C7
:10BED4002360002010BD114B1B784B6004230B60C2
:10BEE4000020F7E7012002F0F9FF606004232360DB
:10BEF4000020EFE7002003F015F8606004232360BE
:10BF04000020E7E7002002F0E9FF606004232360DB
:10BF14000020DFE70E2070470520DBE7A851002052
:10BF240010B5044650B1236863B123685B696BB1F3
:10BF3400002323732046FFF7F2FE10BD7846FBF77B
:10BF4400ADF9F0E77846FBF7A9F9EEE77846FBF799
:10BF5400A5F9EDE710B5044690B12369A3B12368B0
:10BF6400B3B123685B69BBB1206900F01EF90023FB
:10BF74000246A168206800F078FA02F031F810BD9A
:10BF84007846FBF78BF9E8E77846FBF787F9E6E7AD
:10BF94007846FBF783F9E4E77846FBF77FF9E3E7B4
:10BFA40070B588B004460E461546837A013B837209
:10BFB400039005924FF0FF33049301238DF818305A
:10BFC40003A8FFF7ACFE98B1104B1B6813F0020FE7
:10BFD40016D00F4B1B68012B12DD0E4BD3F8043522
:10BFE4000D4A009291220D49022000F009FD07E05C
:10BFF4002A463146079813F075F903A8FFF7AAFFFC
:10C00400A37A0133A37208B070BD00BF3833002097
:10C014003433002000B0004008FA0300FBF90300A9
:10C0240070B590B0002843D0044616460D4600F083
:10C03400C2F8021B214608A813F054F90023009308
:10C0440008AB2246294602A800F0CEF9044610B1F6
:10C05400204610B070BD02A8FFF748FE0028F7D0B4
:10C06400079BD3B1314602A804F0F0FA294602A88E
:10C0740000F093F8C5B2334602AA29460DF129000F
:10C08400FCF758FB044602A8FFF780FE48B905995F
:10C09400BDF81000FBF774F9DAE77846FBF7FEF811
:10C0A400E0E72A460DF1290102A8FFF779FFEEE740
:10C0B4000E24CDE74B78DB09C3724B7803F07F0382
:10C0C40083728A78CB781B0243EA02430A791343CA
:10C0D400C3604A798B7943EA02230381704738B5F8
:10C0E4000D460446002840D0002D42D02889FEF792
:10C0F4000BF9012841D195F90A30002B41DBEB689B
:10C10400B3F1807F41D26B69002B42D02B6903F0DD
:10C114000102237803F07F0343EAC21323706A69A0
:10C12400127803F0800302F07F0213432370EA7A4B
:10C13400637803F07F0343EAC213DBB26370AA7A25
:10C1440003F0800302F07F0213436370EB681A0C60
:10C15400A2701A0AE27023712B891A0A6271A37100
:10C164006B881A0AE271237238BD7846FBF796F899
:10C17400BAE77846FBF792F8B8E77846FBF78EF80B
:10C18400B9E77846FBF78AF8B9E77846FBF786F80B
:10C19400B9E77846FBF782F8B8E7C37A1BB90420FD
:10C1A400081A093870470820FAE709387047073039
:10C1B4007047093070470130704770B588B0044645
:10C1C4000D461646002300938DF8043002691302CD
:10C1D40003F47F0343EA0263110A01F47F410B4332
:10C1E40043EA1263CDF805302846FFF7E0FF036801
:10C1F400CDF8093082888379ADF80D208DF80F30A1
:10C20400606904AA69461130FFF7BAFB3046FFF7AC
:10C21400D2FF04462846FFF7CEFF062308E0013B81
:10C224009BB2C25C08A9194411F8101C4A40E2549C
:10C23400002BF4D108B070BD2DE9F04395B004AFE4
:10C2440004460D4691461E4697F86480002387F8FD
:10C254003F303B84FB6107F130033B611046FFF73D
:10C26400A6FF78613046FFF7A2FF78623B6E6361F8
:10C27400324649462046FFF7A0FF31462046FFF7E5
:10C2840019FF2089FEF740F801281DD04FF000095E
:10C29400B9F1000F4BD0E37A002B33D00823DBB283
:10C2A40087F82C30ED1A073DADB23D837B691D4400
:10C2B400BD62B8F1000F27D0B8F1010F3DD0784628
:10C2C400FAF7ECFF002120E0A5F10902E37A2BB193
:10C2D40008239A4204D24FF00009D9E70423F8E76F
:10C2E400E1682089FBF726F8814610B14FF0000978
:10C2F400CEE7391D208909F001F90028C8D14FF093
:10C304000109C5E70423CAE7002107F1300300222D
:10C314002046FFF75CFB63690133FB6007F13F01D3
:10C3240007F10C00FFF74FFB97F83F303BB997F844
:10C334003F004437BD46BDE8F0830321E5E7F379C8
:10C34400307A40EA03206080FDF7DEFF20701F4B47
:10C354001B6813F0020FEAD01D4B1B68032BE6DDAC
:10C364006C46B7F818C04FEA4C030833DB08A4EB5B
:10C37400C3039D460DF1100E7546002311E07A6A41
:10C38400D25C4FEA121859001248066816F8086081
:10C3940005F8136002F00F0201310068825C6A54F0
:10C3A40001336345EBD300230EF81C300A4BD3F85A
:10C3B4000435CDF808E0094A0192094A0092E622C0
:10C3C4000849042000F01CFBA546B0E738330020E0
:10C3D400343300203C33002000B000406CFA0300EA
:10C3E40094F603005FFA03002DE9F04784B0884611
:10C3F400154699469DF83070064618B112B10BB136
:10C404009A4202D17846FAF749FF2878C009FDF725
:10C41400F9FC30610023736195F800A00AF07F0AEB
:10C424000293039301E0029BCBB103AA02A95046F5
:10C4340008F040FF0024012CF5D804AB03EB84037F
:10C4440053F8083C002BEED0019700934B462A4644
:10C4540041463046FFF7F0FE18B90134EBE70520FA
:10C4640000E0002004B0BDE8F087F0B58FB00C46C2
:10C4740015461F46064650B16DB1012F0FD897B12E
:10C48400012F39D07846FAF709FF00210CE07846ED
:10C49400FAF704FFF0E77846FAF700FFEDE778468D
:10C4A400FAF7FCFEEBE700210AAB00223046FFF767
:10C4B4008EFAF37A13BB04238DF8243073690133A5
:10C4C40001930AAB02932846FFF771FE039007908D
:10C4D400A31C9BB2ADF810300022ADF818200592D1
:10C4E4001844089001A8FFF76AFA2A4629463046FC
:10C4F400FFF763FE0FB0F0BD0321D5E70823DBE7A8
:10C5040038B50D460446C8B12378AB421AD9EDB903
:10C5140062682378134413F8013CA1780B44DBB21E
:10C5240012789B1ADBB2CBB16368585DA378013BE8
:10C534001840A368627802FB003038BD7846FAF7E9
:10C54400ADFEE1E77846FAF7A9FEE0E76268531921
:10C5540013F8013C525D9B1ADBB2E4E70020ECE7E0
:10C5640038B50C460546A0B12B78A34215D9C4B9F9
:10C574006A682B78134413F8013CA9780B44DBB2A6
:10C5840012789B1ADBB21BB16A68135D0133135531
:10C5940038BD7846FAF782FEE6E77846FAF77EFE7B
:10C5A400E5E76A68131913F8013C125D9B1ADBB2C4
:10C5B400E9E710B5044608B1002307E07846FAF726
:10C5C4006DFEF9E762680021D154013322789A4262
:10C5D400F8D810BD10B5044643786BB12378012B0D
:10C5E4000ED9A36883B1636893B1A378A3B15A1E2B
:10C5F400134217D0002310E07846FAF74FFEEDE718
:10C604007846FAF74BFEECE77846FAF747FEEAE796
:10C614007846FAF743FEE8E700232BB12046FFF7FC
:10C62400C8FF10BD0123F8E77846FAF737FEF5E7AF
:10C6340038B50C46054658B12B78A3420CD97CB1C9
:10C644006B681A1912F8010C1B5DC01AC0B238BD10
:10C654007846FAF723FEEFE77846FAF71FFEEEE78F
:10C664006A682B78134413F8010CAB781844C0B2F1
:10C674001378C01AC0B2EAE728B108B529B1FFF7A8
:10C6840009FB002008BD0E2070470E20FAE768B1B0
:10C6940071B110B582B00B46002402A901F8014D16
:10C6A4000122FFF765FA204602B010BD0E20704744
:10C6B4000E20704700B330B58BB00546F1B10C467F
:10C6C4001031FFF7BBFA0E4B09930E4B93E80300AE
:10C6D4000790ADF8201003AA042109A8FFF712FA65
:10C6E40001940623009307AB03AA10212846FFF701
:10C6F40021FA00200BB030BD0E2070470E20F9E760
:10C704006E6B626B80FA0300E8B130B58BB00546FE
:10C71400D9B10C460E4B09930E4B93E803000790D6
:10C72400ADF8201003AA042109A8FFF7EBF901943E
:10C734000623009307AB03AA10212846FFF7FAF952
:10C7440000200BB030BD0E2070470E20F9E700BF6B
:10C754006E6B696B80FA030010B330B587B0044682
:10C7640001B30D46104B019302AA04210DEB010005
:10C77400FFF7C8F902AB102221461846FFF71BF950
:10C784009DF816301B0203F47C536FEA43436FEAAF
:10C7940053439DF8172013432B80002007B030BD6E
:10C7A4000E2070470E20F9E77674616438B50C46A4
:10C7B40083692BB10268406801FB0020984738BDAB
:10C7C400056840680246002104FB005012F0B3FDE6
:10C7D400F5E738B50546002404E021462846FFF76E
:10C7E400E5FF0134AB68A342F7D8013BEB6038BDE9
:10C7F400F8B504460F46C56800260CE02168636856
:10C804001A4605FB0311384612F036FD88B9012398
:10C8140016E001361D46A368B34210D96369002BA4
:10C82400ECD02268616805FB01213846984703462D
:10C8340030B96B1E002DECD1A368013BE9E700235E
:10C844001846F8BD38B5C3680133C36082689342A3
:10C8540008D003694BB10268C468406800FB042037
:10C86400984738BD0023C360F3E70468C56840688F
:10C87400024600FB054012F035FDF2E770B50E46A6
:10C88400044648B141B12368B34209D0256865B96B
:10C8940026600023336017E07846FAF7FFFCF2E7DE
:10C8A4007846FAF7FBFCF1E725462C682CB1B44234
:10C8B400FAD17846FAF7F2FCF6E735B12EB1B54273
:10C8C40002D02B6833602E6070BD7846FAF7E6FC20
:10C8D400F5E738B505460C4649B140B12A68CAB1F6
:10C8E400A24209D123682B60002020600CE0784626
:10C8F400FAF7D4FCF2E71A4613680BB1A342FAD153
:10C9040052B1A34201D0052038BD23681360002032
:10C914002060F9E70520F7E70520F5E72DE9F04168
:10C924000D461746064608B101B112B97846FAF722
:10C93400B5FC3368AB4204D0346834B14FF000081E
:10C9440009E07846FAF7AAFCF6E73560002028608B
:10C954000FE0A046344654B129462046B84730B9C2
:10C964002668B542F5D17846FAF798FCF1E714B198
:10C974000F20BDE8F081B8F1000F09D045B1A845FA
:10C984000AD0D8F800302B60C8F800500020F0E737
:10C994007846FAF783FCF2E70020EAE730B583B083
:10C9A400184606AC54F8045B00920B46024605494F
:10C9B40000200AF077FD2246294600200AF088FC70
:10C9C40003B030BD88FA0300034B1860034B1960B1
:10C9D400034B1A60704700BF383300203433002003
:10C9E4004033002030B583B0044C246824B1079D43
:10C9F4000195069D0095A04703B030BD403300204B
:10CA040030B585B008AC54F8045B039401940095E8
:10CA1400FFF7E8FF05B030BDC268137951795B1A9E
:10CA240003F57F2303F6FF731B0303F580531344BD
:10CA340042699B1A8068181A704770B50579012DF0
:10CA440001D9002070BD044606683046FFF7E4FFB4
:10CA54003DB9A3899B00834207DB73681BB900209F
:10CA6400F0E70023F7E70120ECE70020EAE738B518
:10CA740005460C4610F0030F0DD114F0030F0ED130
:10CA84000023B3EB940F0ED255F82320B2F1FF3FED
:10CA94000BD10133F5E77846FAF700FCEDE7784669
:10CAA400FAF7FCFBECE7012038BD0020FCE770B589
:10CAB400054600240EE0002300E0002318463BB3A3
:10CAC4005379A3421BD1EB681E4432792B699A42F5
:10CAD40019D101342B69A34219D9EB6826039A1999
:10CAE4009B5D083BDBB2F62BE7D85379FF2B04D0D0
:10CAF4001379FF2BDFD00123E0E70023DEE778463C
:10CB0400FAF7CCFBDFE77846FAF7C8FBE1E7012048
:10CB140070BD0000F0B585B004460368DB68187882
:10CB240019795A79891A01F57F2101F6FF710903F0
:10CB340001F58051E2891944184401F0ADF9074622
:10CB440023689E6826F47F6525F00F0505F580555A
:10CB5400A81BA2899200824237D2B51804F10C02B4
:10CB6400A3899B0001208DF8000001960392029393
:10CB740000226946FDF72CFB002852D101208DF8D4
:10CB8400000001952E4B0393042302932D4A69461A
:10CB9400FDF71EFB002848D19FB1226839885368ED
:10CBA40003EB8103536001208DF800000197264BAD
:10CBB400039304230293234A6946FDF709FB0028E3
:10CBC40037D1A660002005B0F0BDD9680B7991F883
:10CBD40005C0A3EB0C0303F57F2303F6FF731B03CC
:10CBE40003F580530B449D4227D0824202D12A7818
:10CBF4001544B3E701208DF800000196134B03930D
:10CC04000423029300226946FDF7E2FA28B92E783C
:10CC14002E44A58906EB8505A0E77846FAF73EFB86
:10CC2400F5E77846FAF73AFBA8E77846FAF736FBD1
:10CC3400B2E77846FAF732FBC3E70120C3E700BF47
:10CC4400BCFA0300D2520020B4FA0300B8FA03007D
:10CC540010B584B004460368DB68187819795A79EA
:10CC6400891A01F57F2101F6FF71090301F580514D
:10CC7400E2891944184401F00FF9E0B10346A060B9
:10CC8400216800884A6802EB80024A6001208DF81E
:10CC940000000193094B039304230293084A694655
:10CCA400FDF796FA10B9002004B010BD7846FAF7E3
:10CCB400F5FA0020F8E70220F6E700BFB4FA030013
:10CCC400D252002070B584B005460368DE68437B09
:10CCD40006EB033608213046FFF7C9FE80B900246D
:10CCE40000E00134072C0BD8335D05F10802125D16
:10CCF4009342F6D0FF2BF4D07846FAF7CFFAF0E758
:10CD0400083501208DF8000001960395082302934D
:10CD1400054A6946FDF75CFA10B9002004B070BDFD
:10CD24007846FAF7BBFAF8E7D252002000B585B08E
:10CD34000368DA681B691B0302218DF80010019255
:10CD44000293074A69460120FDF742FA18B9002008
:10CD540005B05DF804FB7846FAF7A0FAF7E700BFE0
:10CD6400D252002082890379012B0FD010B5920092
:10CD74001BB1022B10D0012007E000F10C018068E8
:10CD840012F07AFAB0FA80F0400910BD836858882E
:10CD9400B0FA80F0400970470368DB68447B0822DE
:10CDA400811803EB043012F067FAB0FA80F04009FE
:10CDB400EBE7000038B501460C48FCF731F80C4BA2
:10CDC4005D6845B938BD2368002222609A68D86836
:10CDD4009047A542F6D00648FDF795FC0446002886
:10CDE400F1D17846FAF75AFAEDE700BFAC510020CA
:10CDF400C05200202DE9F041044617460D4611B9F2
:10CE0400FFF7B0FF58B10DB104F10C072668237980
:10CE1400042B0DD8DFE803F005464E0C5D00032516
:10CE2400F2E7A5B1B3691BB12A46394630469847A3
:10CE34002E4B9C4203D303F582739C4202D978465D
:10CE4400FAF72CFA201FFFF7B5FFBDE8F081D4F8FC
:10CE54000880B8F800300BB3B8F8003008EB83034F
:10CE640023F47F6222F00F02934204D0B8F8022028
:10CE7400B2F5FE4F08D128F47F6828F00F0808F5B2
:10CE8400805898F800304344B3605A8847F6FF73DB
:10CE94009A42C7D07846FAF701FAC3E77846FAF718
:10CEA400FDF9D9E7F369002BC2D02A46E18930465F
:10CEB4009847BDE73378012B07D1627B237B013B85
:10CEC4009A42B5D102233370B2E77846FAF7E6F90D
:10CED400F3E73DB900233370336A002BA8D0304602
:10CEE4009847A5E77846FAF7D9F9F3E7B85100204F
:10CEF40000B583B002A9002341F8043D82B205487D
:10CF0400FBF7E6FE20B90198043003B05DF804FB9A
:10CF14000020FAE7AC51002070B50446002536E045
:10CF24001020FFF7E5FF0646002860D002230371B6
:10CF340008230372042343721023C372837245735C
:10CF4400236903734FF6FF73C3810460294B98422E
:10CF540003D303F58273984202D97846FAF79EF90F
:10CF640036F8042C311F2448FBF7E1FE0EE00023C1
:10CF740000E000234BB3E36833445B79AB4228D130
:10CF8400E3681E44327923699A4226D10135236924
:10CF9400AB4226D9E0682E03304440F6FC710430DD
:10CFA400FFF765FD0028BBD1E3689A199B5D083B38
:10CFB400DBB2F62BDDD85379FF2B04D01379FF2B8A
:10CFC400D5D00123D6E70023D4E77846FAF766F9EB
:10CFD400D1E77846FAF762F9D2E77846FAF75EF9CC
:10CFE400D4E7064B1868FEF7F5FB002070BD04205B
:10CFF400FCE700BFB8510020AC510020C85200200B
:10D0040038B50546C3681C781C4400200DE07846FA
:10D01400FAF744F91FE024F47F6323F00F0303F5C8
:10D0240080531A78134420461C46EA6813795179D0
:10D034005B1A03F57F2303F6FF731B0303F5805389
:10D0440013449C4215D262884FF6FF739A4210D063
:10D054002388002BDBD0238804EB830323F47F6233
:10D0640022F00F029342D6D06288B2F5FE4FDAD195
:10D07400D1E738BD38B50446FFF7C2FFA06010B34E
:10D08400428847F6FF739A4222D00820FFF730FF08
:10D094000546F8B10323037104600F4B984203D390
:10D0A40003F58273984202D97846FAF7F7F835F80F
:10D0B400042C291F0948FBF73AFE094B1868FEF7B0
:10D0C40089FB002005E0E26813781344A36000E0C4
:10D0D400002038BD0420FCE7B8510020AC510020EA
:10D0E400C852002070B505794379ED1A05F57F25FE
:10D0F40005F6FF752D0305F58055054404780444B1
:10D1040000260DE07846FAF7C9F819E024F47F64A4
:10D1140024F00F0404F5805420780444A5421ED959
:10D1240063884FF6FF7293421DD047F6FF72934215
:10D1340019D013B9238806EB83062388002BE1D08A
:10D14400238804EB830323F47F6222F00F029342CB
:10D15400DCD06288B2F5FE4FD8D01C46DEE77846B4
:10D16400FAF79CF8DCE7304670BD000070B584B077
:10D1740005460068FFF744FF044600282FD0638863
:10D18400002B30D12E682388002B3ED0238804EB5B
:10D19400830323F47F6222F00F02934203D0628858
:10D1A400B2F5FE4F07D124F47F6323F00F0303F598
:10D1B40080531A781344B3602B689968DA6813793A
:10D1C40050791B1A03F57F2303F6FF731B0303F542
:10D1D4008053134499421CD3002004B070BD784698
:10D1E400FAF75CF8CBE701208DF8000001941F4B9F
:10D1F4000393042302931E4A6946FCF7E9FF0028BF
:10D20400C0D07846FAF74AF8BCE77846FAF746F809
:10D21400BCE7238833B3238804EB830323F47F62BE
:10D2240022F00F02934203D06288B2F5FE4F07D179
:10D2340024F47F6424F00F0404F5805423782344F9
:10D2440001208DF8000001930A4B039304230293F9
:10D25400074A6946FCF7BCFF0028BDD07846FAF7B8
:10D264001DF8B9E77846FAF719F8D4E7B4FA0300D9
:10D27400D2520020BCFA030008B50379042B13D85A
:10D28400DFE803F00306090C0F00FFF743FC08BDB9
:10D29400FFF7DEFCFBE7FFF715FDF8E7FFF766FF96
:10D2A400F5E7FFF743FDF2E77846F9F7F7FF0020CB
:10D2B400EDE700002E4B1B78022B57D110B582B03E
:10D2C40041E002A9002341F8043D2A48FBF760FD30
:10D2D40090B9019C201D284B1860284B01221A701C
:10D2E400FFF7ABFB58B30323214A13706268137032
:10D2F4006068FCF757F922E0214B1B6803B198479B
:10D30400012002B010BD1C4B1868FFF7B5FF1D4B80
:10D31400187018B9194B02221A7010E0174B032227
:10D324001A700CE0144B1B68E3B1134B1868826845
:10D33400144B1978FFF75EFD104B00221A700C4B4A
:10D344001B78022BDCD10D4B1B78032BF7D801A2E1
:10D3540052F823F0C7D202000BD3020005D3020017
:10D3640029D302007846F9F799FFDEE701207047D8
:10D37400D0520020AC510020D4520020BC520020D6
:10D38400CC520020D852002008B5074B1B8893428A
:10D3940000D008BD054B1B78022BFAD1034B0322A6
:10D3A4001A70FFF787FFF4E7D2520020BC52002026
:10D3B40008B54FF4827210491048FBF709FC104974
:10D3C4000120FCF7F3FE0F48FEF7E4F90E4B18605A
:10D3D40000230E4A13700E4A13800E48FDF76CF9B1
:10D3E400FCF7B8F818B90C4B02221A7008BD0A4BA6
:10D3F40003221A70FAE700BFB8510020AC51002094
:10D404008DD30200B9D20200C8520020BC520020C1
:10D41400D2520020C0520020D052002038B5054618
:10D424000820FFF765FDD0B1044604232B70037177
:10D4340005600C4B984203D303F58273984202D9DA
:10D444007846F9F72BFF34F8042C211F0648FBF724
:10D454006EFC064B1868FEF7BDF9002038BD0420A9
:10D46400FCE700BFB8510020AC510020C852002096
:10D4740038B50C460546D0B1631E9BB247F6FE6232
:10D48400934218D82B78022B17D1EB6818781979A6
:10D494005A79891A01F57F2101F6FF71090301F513
:10D4A400805122461944184400F0F6FC38BD7846F1
:10D4B400F9F7F4FEE0E70020F8E70020F6E7F8B516
:10D4C4000E461546074680B33B78022B40F0938006
:10D4D4007DB3FA68137813449D42C0F08E801379AB
:10D4E40051795B1A03F57F2303F6FF731B0303F5DE
:10D4F400805313449D4200F282802B884BB32C88C6
:10D5040005EB840424F47F6323F00F039C4203D0CF
:10D514006B88B3F5FE4F0FD125F47F6525F00F0519
:10D5240005F580552C782C4406E07846F9F7B6FECC
:10D53400CAE7FC6823781C44FD682B796A799B1A36
:10D5440003F57F2303F6FF731B0303F580531D4488
:10D554000FE07846F9F7A2FED1E77846F9F79EFE88
:10D564001DE024F47F6424F00F0404F58054237830
:10D574001C44AC4226D26288531E9BB247F6FE611D
:10D584008B4207D8D6B1718833884A40134217D0EA
:10D59400002300E00023ABB92388002BDDD02388CF
:10D5A40004EB830323F47F6222F00F029342D8D06A
:10D5B4006288B2F5FE4FD4D01C46DAE70123EAE7CD
:10D5C4000123E8E7AC421CD26288531E9BB247F6A3
:10D5D400FE618B4207D856B1718833884A401342A2
:10D5E40007D0002300E000236BB12046F8BD0123DF
:10D5F400FAE70123F8E70024F7E70024F5E700241D
:10D60400F3E70024F1E70024EFE770B50E46144673
:10D61400054658B1731E9BB247F6FE6293420BD97E
:10D6240047F6FF739E4205D0002306E07846F9F7DB
:10D6340035FEEFE7012300E0012393B1802C14D8D9
:10D644002B78B3B104F11000FFF752FC98B100221B
:10D654000271C6810334A4080134848140F80C5B50
:10D6640070BD7846F9F71AFEE8E77846F9F716FE32
:10D67400E6E70020F4E70020F2E7000010B50446D6
:10D684000F4B984203D303F58273984202D978462C
:10D69400F9F704FE0C3C0A4B9C4203D303F5827356
:10D6A4009C4202D97846F9F7F9FD34F8042C211F7D
:10D6B4000448FBF73CFB044B1868FEF78BF810BDDD
:10D6C400B8510020AC510020C852002070B50D465E
:10D6D400064658B16B1E9BB247F6FE6293420BD9C5
:10D6E40047F6FF739D4205D0002306E07846F9F71C
:10D6F400D5FDEFE7012300E001230BB31020FFF772
:10D70400F7FB044600B301230371C5814FF6FF7391
:10D71400838106600D4B984203D303F582739842CC
:10D7240002D97846F9F7BAFD34F8042C211F0848C9
:10D73400FBF7FDFA074B1868FEF74CF8002070BDA4
:10D744007846F9F7ABFDD9E70420F8E7B851002093
:10D75400AC510020C85200202DE9F041C46894F86F
:10D76400008004EB08068368B34202D80020BDE8B9
:10D77400F0813746054634F80830B3B134F8084030
:10D7840006EB840424F47F6323F00F039C4203D04C
:10D794007388B3F5FE4F1AD126F47F6626F00F0680
:10D7A40006F580563478344411E07846F9F776FD6E
:10D7B400E4E77846F9F772FD0FE024F47F6323F081
:10D7C4000F0303F580531A78134427461C46AB68AD
:10D7D400A34210D02388002BEBD0238804EB8303CF
:10D7E40023F47F6222F00F029342E6D06288B2F5FE
:10D7F400FE4FEAD1E1E77A88531E9BB247F6FE61F9
:10D804008B4201D90020B2E7EB68187839461844F6
:10D8140000F042FB30B1874206D041882846FFF72A
:10D8240055FFA4E70020A2E70020A0E770B5044656
:10D834000D46002303700B68C3F30B030BBB6B682B
:10D84400FE2B22D829686A68AE68E868E160226124
:10D854006661A06129696A69E16122620023A360AB
:10D8640063602046FFF723F9D0B12169E068FFF730
:10D8740039FC60602046FFF7FDFB034648B11846BB
:10D8840070BD7846F9F70AFDD9E77846F9F706FD41
:10D89400D8E7022323702046FFF75EFF0346EEE736
:10D8A400012323702046FFF737FB03460028E6D107
:10D8B400E2680832A260E2E710B5044620B1A3682A
:10D8C40033B1236843B110BD7846F9F7E7FCF6E7B6
:10D8D4007846F9F7E3FCF4E7246021460148FCF7B5
:10D8E400F6FEF0E7C052002008B50648FBF771FACF
:10D8F40008B1002008BDFBF74DFE08B10020F9E790
:10D904000120F7E7AC51002010B5C0B10446C3684C
:10D91400187819795A79891A01F57F2101F6FF716E
:10D92400090301F5805147F6FF721944184400F0C9
:10D93400B3FAA06078B10223237000236360084B1C
:10D9440002221A7007490120FCF730FC064B1868C4
:10D95400FDF740FF10BD7846F9F7A0FCEBE700BFE8
:10D96400D05200208DD30200C852002008B5FBF726
:10D974003DFE08BD50B110B50446064B1B6813B1FB
:10D984007846F9F78BFC034B1C6010BD014B002259
:10D994001A607047CC52002046DF70472DE9F047EB
:10D9A40007460E468589012411E0013B9BB2C1184C
:10D9B40018F801201EF803A082EA0A0209F80120DF
:10D9C400002BF2D1A5EB0C05ADB20134A4B2BDB16C
:10D9D400230A43EA0423F3833046FFF7DDFFAC4612
:10D9E400102D28BF4FF0100CD7F81890601E0001BE
:10D9F400D7F8088006F1200E5FFA8CFC6346DFE757
:10DA0400BDE8F0872DE9F04780460F461646994653
:10DA140000F1100400F1200518E05246394604EBE9
:10DA2400090011F05FFC4E44B6B2103EB6B2574442
:10DA340020E0013B9BB2EA5CE15C4A40E254002BEB
:10DA4400F7D14046FFF7A8FF4FF00009A6B1C9F18E
:10DA5400100A5645E1DA3246394604EB090011F062
:10DA640041FC06EB0900C0F110020021204411F032
:10DA740062FC00261023E2E7BDE8F087F8B504460F
:10DA84000D461646838A002B3BD0402294F8203062
:10DA9400023B03EBD3735B10DB0003F03803134347
:10DAA40043F001032B746268176850689168C5F8E5
:10DAB4001170C5F81500C5F81910127B6A77A28990
:10DAC400130A43EA0223EB832846FFF765FFA38A80
:10DAD4006BB1B3F57F4F16D2A28A130A43EA02232D
:10DAE4002B820223A28A21692846FFF78BFFA28991
:10DAF4006AB994F8202005F12001304611F0F2FBB8
:10DB0400F8BD0022C2E77846F9F7C8FBE4E7002332
:10DB1400A1682846FFF776FFEBE730B58DB00546E0
:10DB240003686C46186859689A68DB680FC4EA6928
:10DB340069462846FFF7A2FFEC696B6801228DF85D
:10DB44001020186859689A68CDF81100CDF815109E
:10DB5400CDF819201B7B8DF81D300023ADF81E3045
:10DB64006846FFF719FF95F8203008E0013B9BB2A7
:10DB7400E25C0CA9194411F8101C4A40E254002B31
:10DB8400F4D169462846FFF709FF0DB030BD2DE9F1
:10DB9400F0418CB000AF04460E4603683D46186859
:10DBA40059689A68DB680FC5A38933BBD4F8088029
:10DBB400A369A36094F82030073303F4FC73ADEB3E
:10DBC400030D6D466A4639462046FFF757FF6368E2
:10DBD40001223A74186859689A68C7F81100C7F89E
:10DBE4001510C7F819201B7B7B770023FB8338466D
:10DBF400FFF7D2FE94F820301EE0636801223A74E5
:10DC0400186859689A68C7F81100C7F81510C7F85A
:10DC140019201B7B7B770023FB8339462046FFF7C3
:10DC2400BDFEC3E7013B9BB2EA5C07F13001194436
:10DC340011F8101C4A40EA54002BF3D1C4F80880B0
:10DC440094F82020E169284611F016FBB0FA80F020
:10DC5400400930703037BD46BDE8F08100231F2BEA
:10DC640028D870B4164603EB4214134D05EBC404D4
:10DC7400A48834B1844212D001331F2BF2D904207A
:10DC84000BE003EB461355F8334061F3170445F8F2
:10DC9400334005EBC3039880002070BC7047064AEC
:10DCA40003EB461352F8330061F3170042F83300D4
:10DCB4000020F2E704207047DC52002000231F2BD1
:10DCC4001AD870B403EB42140C4D05EBC404A488B9
:10DCD400844204D001331F2BF4D9002008E003EB65
:10DCE400421355F83330C3F317038B4202D200209A
:10DCF40070BC70470120FBE700207047DC52002015
:10DD040008B54FF400720021034811F014FB034BD3
:10DD140000221A7008BD00BFDC520020D952002036
:10DD240008B5FFF7EDFF08BD2DE9F041D8B1E2B128
:10DD3400EBB1FF291DD01C2B1DD81E4690460C4666
:10DD44009F1CFFB2791C07F045FE054640B147749D
:10DD54002B238374C47432464146143011F0C2FA42
:10DD64002846BDE8F0810025FAE70025F8E70025FC
:10DD7400F6E70025F4E70025F2E700002DE9F04F6F
:10DD840085B004AF0C461646054630B3002C69D066
:10DD9400611EC9B22A7822B3012A28D0364B1B68E7
:10DDA40013F4807F03D0354B1B68012B25DC324BE9
:10DDB4001B6813F4807F5AD0304B1B68032B58DD4B
:10DDC400EB46A0466300083303F47E73ADEB030D0A
:10DDD4000DF11009CE4600232EE07846F9F75EFADD
:10DDE400D4E73246681C0CF0A7FD00203BE0324625
:10DDF400681C00F0B5FD002035E0214BD3F8043554
:10DE04000192204A00926D221F490220FEF7F8FD7C
:10DE1400CDE76A1CD25C4FEA121A59001B4E3068D7
:10DE240010F80A000EF8130002F00F0201313068F6
:10DE3400825C0EF8012001334345EAD3002309F83C
:10DE440014300F4BD3F80435CDF80890104A0192E2
:10DE5400104A00926E220C490420FEF7D1FDDD46E3
:10DE64000B2000E009200437BD46BDE8F08F0B20ED
:10DE7400F9E70B20F7E700BF3833002034330020E4
:10DE840000B00040F0FA0300E7FA03003C3300203E
:10DE940018FB030094F60300F8B506460D46174632
:10DEA400884201D8344613E07846F9F7F7F9F9E7E0
:10DEB4007846F9F7F3F921E024F47F6424F00F04A1
:10DEC40004F5805423781C44A5422AD9A6422BD2B7
:10DED4006288BA4226D024F47F6323F00F0303F54B
:10DEE4008053AB4207D3B2F5FE4F16D0238804EB20
:10DEF4008303AB4213D22388002BD9D0238804EBAD
:10DF0400830323F47F6222F00F029342D4D0628809
:10DF1400B2F5FE4FD0D01C46D6E7002402E0002420
:10DF240000E000242046F8BD0024FBE7014B186004
:10DF3400704700BF0455002070B50E46054678B101
:10DF440096B12B78012B13D8234B1B6AA3B96B68AA
:10DF54001D2B15D82B78012B16D0204B1C681CE0E8
:10DF64007846F9F79BF9EBE77846F9F797F9E8E78C
:10DF74007846F9F793F9E7E77846F9F78FF9E6E792
:10DF84007846F9F78BF9E5E7EB68B3F1FF3FE4D0A6
:10DF94007846F9F783F9E0E7246894B154F8083C2B
:10DFA4001B682946A4F1080098470028F4D114F806
:10DFB400042C012303FA02F207490B6A13430B6290
:10DFC400EAE7054B1B6A23B16A68034B03F8012B8C
:10DFD4003360014B186A70BDE054002008550020DE
:10DFE40010B5114B1B6A13B1104B1C6804E0784642
:10DFF400F9F754F9F8E724688CB1A4F108000A4B46
:10E004001A6A14F8041C01238B401A42F3D054F802
:10E01400083C5B68044911F8012B9847EBE7024B75
:10E0240000221A6210BD00BFE054002008550020F1
:10E0340010B50F4B1B6A13B10E4B1C6804E07846F5
:10E04400F9F72CF9F8E7246874B1A4F10800084B37
:10E054001A6A14F8041C01238B401A42F3D054F8B2
:10E06400083C9B689847EEE7014B00221A6210BDFA
:10E07400E0540020085500202DE9F0410D461746D4
:10E084009846064648B1074B1C6824B143463A46B5
:10E0940031792846A047BDE8F0817846F9F7FEF8C3
:10E0A400F1E700BF0455002070B50C46164605463E
:10E0B400C0B1DCB1F6B1236803B3636813B3A368DA
:10E0C40023B3164B1B781F2B24D82C60134A1378C8
:10E0D400591C11702B716E7105F108011048FEF77F
:10E0E400CDFB70BD7846F9F7D9F8E2E77846F9F741
:10E0F400D5F8DFE77846F9F7D1F8DCE77846F9F7A1
:10E10400CDF8DAE77846F9F7C9F8D8E77846F9F7A9
:10E11400C5F8D6E77846F9F7C1F8D6E7DC5400200D
:10E1240008550020F8B504460F4616461D469B6860
:10E13400ABB10A23237000232373AB88E3812B68DC
:10E144001B8863822B681888FCF7DEF82074AB68A0
:10E15400A3616760A6602B681B7B2377F8BD7846B4
:10E16400F9F79CF8E5E710B58CB0044603685A68E3
:10E174000AB9DB89EBB12368DB8913F0010F1CD1E9
:10E18400002223681B7B03F07F038DF808300023F3
:10E194008DF809308DF80A202346032202A904A829
:10E1A400FFF7C0FF6FF0020104A8FAF748F90CB0BA
:10E1B40010BD7846F9F772F8DDE769464FF4C87088
:10E1C400FCF7B1FF18B9019A02F00102D9E77846C9
:10E1D400F9F764F8F7E700000378012B00D07047E3
:10E1E40000B585B01E4B1B6873B11D4B1B6801A89D
:10E1F4009847A8B91B4B1B7863B1019B1A883AB1A5
:10E204005B6833B1012304E07846F9F747F8ECE79B
:10E21400002383B9144B1B7813B1019B1B88D3B91A
:10E224001248FAF72FFC00230E4A13700E4A13709B
:10E2340005B05DF804FB01A8FFF795FF0028E9D1BC
:10E244000B4B1B681BB10A4B1B689847E2E77846E7
:10E25400F9F724F8F7E701A8FFF785FFE0E700BF27
:10E264003055002019550020185500200C55002069
:10E274002C5500200B6813B1013B0B60704710B59F
:10E284000C460348FCF7D6FC0023236010BD00BFF6
:10E294005055002010B584B004462C4B1B68EBB1DC
:10E2A4002A4B1B6801A8984700284BD1284B1B68B0
:10E2B400C3B127490A6801988368934228BF13466B
:10E2C400B3F5E16F94BFD31AA2F5E1630B607BB998
:10E2D40003885BB1436853B1012308E07846F8F73B
:10E2E400DDFFDDE77846F8F7D9FFE2E7002383B9DD
:10E2F400019B5B6813B3164B1B68B3F5E16F1BD22C
:10E30400144901FB03F121441348FCF7C3FC04B096
:10E3140010BD01A8FFF727FF28B9104B1B683BB1BC
:10E324000E4B1B689847019B9A68094B1A60DFE7FC
:10E334007846F8F7B3FFF3E70949E4E70648FCF742
:10E3440079FCE4E70448FCF775FCE0E7305500206D
:10E354003455002040420F00385500202C55002031
:10E3640000D2496B03780A2B00D07047C389234A33
:10E3740012889342F9D1418A204A52889142F4D1B9
:10E384008268032AF1D11D4A9268002AEDD000B5B3
:10E394008DB01A4A5268B2F5803F02D20132174951
:10E3A4004A6005228DF8042041680A7802F07F0251
:10E3B4008DF808200A7802F07F02007F121AD2B288
:10E3C4000132D2B28DF80920897801F00F01ADF83D
:10E3D4000A10ADF80C3093B2084A9289934201D2E4
:10E3E400064A9381054AD289934201D9034AD381CB
:10E3F40001A8FAF70FFB0DB05DF804FB1C550020D3
:10E4040038B503689B68094C44F8043B03689D686D
:10E41400B5F5E16F28BF4FF4E165FCF7D7FC04497B
:10E4240001FB05012046FCF735FC38BD34550020BE
:10E4340040420F0010B584B004460D4B1B6863B115
:10E444000B4B1B6801A8984728B9019BDA89224223
:10E4540001D01B882BB904B010BD7846F8F71EFF15
:10E46400EEE70448FAF7FEFA034B01221A70F2E7CA
:10E47400305500200C5500201855002008B5134BCA
:10E484001B78DBB901211248FAF77CFAD0B90022D3
:10E49400104B1A70104B1149D960114B1A605A6015
:10E4A4005A61104A9A60104A1A61104ADA60104B95
:10E4B400104A1A60054B01221A7008BD7846F8F715
:10E4C400EDFEDFE77846F8F7E9FEE0E71A550020AD
:10E4D4002CFB0300195500203455002099E202005A
:10E4E4005055002079E202002455002040420F00DC
:10E4F4000C550020DDE1020070B582B0044630B353
:10E5040001A90DF1060007F03FF8A368B3F5803FB9
:10E514003FD82088FBF7F8FE012804D02088FBF7B9
:10E52400F3FE002838D16088FBF7EEFE98B9A368A3
:10E534001BB122880AB16188C9B9184B00241C8018
:10E544005C809C601648FCF775FB204622E0784608
:10E55400F8F7A4FED4E76088FBF7D6FE0328E6D0DC
:10E564006288BDF806309A42E1D0072012E00B4CD5
:10E5740022806180A3600A4DEE68FCF727FC311805
:10E584002846FCF787FB7F23A3810020E08160609D
:10E5940000E0072002B070BD0720FBE71C550020F7
:10E5A40050550020004870471C55002038B50C46D3
:10E5B400054628B144B1064B1D60064B1C6038BDAE
:10E5C4007846F8F76BFEF5E77846F8F767FEF2E76A
:10E5D400305500202C55002000B585B0114B1B6828
:10E5E4008BB1104B1B6801A8984748B9019B1A8846
:10E5F4001AB15A680AB19B684BB90B48FCF71AFB6D
:10E6040005B05DF804FB7846F8F748FEE9E701A891
:10E61400FFF7F6FE0548FAF725FA054B01221A70B2
:10E62400EEE700BF30550020385500200C5500207F
:10E634001955002030B585B00D4614466B460D22A1
:10E6440001462846FDF7B7F96B4603CB20606160AD
:10E6540005B030BD30B58DB004460DF12F025449DC
:10E66400002006F0C7FE1BE0131B21E030F8131056
:10E674000A440133012BF9D9013202EB8202520020
:10E684000123012B1BD94A4B1B685B6800211980AD
:10E6940095421ED20DF12F024549002006F0AAFE34
:10E6A400434B1B68002B66D058684268A31ADBD41E
:10E6B400404DA5FB03239D0C00231A46DAE73C4991
:10E6C40009684968581E31F8100021F81300013315
:10E6D400D7E7FBF783FB0546FBF7A0FB9DF82F303C
:10E6E400022B4AD0324A11680831022B14BF00228F
:10E6F40001229DF8183062F30003012814BF0022A0
:10E70400012262F341036FF387038DF818300B463F
:10E7140053F8102F5B68CDF81920CDF81D302B026B
:10E7240003F47F0343EA05632A0A02F47F42134396
:10E7340043EA1563CDF821300DF1250206A8FFF751
:10E7440079FF152306AA01211B48FFF7EDFA0146BC
:10E7540088B101230371184807F07AF9174B1B6835
:10E7640013F0020F03D0164B1B68042B09DC104B6B
:10E774001B685B685C600DB030BD0D4A11683031B8
:10E78400B3E7104BD3F80435094A1268117E507E62
:10E79400957ED27E04920395029001910A4A0092DA
:10E7A4004FF4807209490520FEF72AF9DFE700BF1C
:10E7B4006456002083DE1B43685500203833002054
:10E7C4003433002000B0004068FB03005BFB03000F
:10E7D40008B5FCF7FBFAFFF73DFF08BD08B5FFF7E6
:10E7E40039FF08BD30B583B005460C460822013117
:10E7F400103010F041FD10B1002003B030BD6A4666
:10E8040029462046FFF716FF082204F10D01684649
:10E8140010F032FDB0FA80F04009EEE730B583B075
:10E82400194B01221A700023184A1360184C194A14
:10E83400E260194AA260236104210DEB0100FCF798
:10E8440017FCFCF7C3FAE2680199B1FBF2F302FB8F
:10E85400131318446060114D3423114A114928469A
:10E8640007F0D4F94FF47A71284607F04BF928469B
:10E8740007F08EF82046FCF7ABF90B4A04210B484D
:10E88400FDF740F903B030BD48560020645600201F
:10E894004C56002080969800E1E70200685500205D
:10E8A40004560020D5E702003856002080FB030000
:10E8B40010B504460A4B1B7803B920B903B15CB107
:10E8C400074B1C7010BDFCF781FA064BD968014454
:10E8D4001846FCF7DFF9F3E70248FCF7ABF9EFE77A
:10E8E400485600204C560020014B1878704700BF52
:10E8F40048560020F8B5069E70B3074676B30D4619
:10E904003046012100F8011B747863F300048A4245
:10E9140014BF0022012262F341046FF38704747070
:10E924003B4653F8102F5B68C0F80120C0F805304F
:10E934002B0203F47F0343EA0563290A01F47F41B0
:10E944000B4343EA1563C0F8093006F10E02394659
:10E95400FFF770FE0020F8BD0E20FCE70E20FAE75A
:10E96400F0B58FB01746054648B100230C936E1CD2
:10E974000DF137020CA9304606F03CFD30E0784634
:10E98400F8F78CFCF1E77846F8F788FC2DE09DF861
:10E994003730FBB129460C983030FFF723FFC8B15C
:10E9A4000C99303137E004238DF804302A4612F8EC
:10E9B4000D3BC3F340008DF81C00C3F300038DF836
:10E9C4001D3006940C9B029303910497059201A8B1
:10E9D400FAF720F80DF137020CA9304606F00AFDCB
:10E9E4000C9B13B35B68002BCDD0D5F809402302F0
:10E9F40003F47F0343EA0463220A02F47F421343CD
:10EA040043EA146429460C980830FFF7EBFE00280B
:10EA1400BDD00C9908310C9B5A6813884FF6FF70CF
:10EA24008342C0D001331380BDE70FB0F0BD2DE9A0
:10EA3400F041804607683E68FF25002405E016F88B
:10EA44002430FF2B0ED00134E4B23B79A3420BD91E
:10EA5400FF2DF4D016F92430002BF0DA7846F8F7BD
:10EA64001DFCECE72546EEE7FF2D02D0AB4200D8B3
:10EA7400FF2588F80450BDE8F0810000F0B585B0AA
:10EA840005460C4617464B78FF2B27D003689E6833
:10EA940006B339466078B0470646F8B93D4B1B6863
:10EAA40013F4803F3FD03C4B1B68032B3BDD3B4BB7
:10EAB400D3F804352A689169607851F820100291DE
:10EAC40012690192364A0092AB2236490420FDF7BE
:10EAD40097FF28E07846F8F7E1FBDAE7A378FF2B05
:10EAE4000ED02B68DE680EB32A4B1B6813F4803FEC
:10EAF40003D0294B1B68032B1CDC3946A078B04794
:10EB0400E378FF2B44D0AB79DBB2012B25D1214B29
:10EB14001B6813F4803F03D01F4B1B68032B20DCBE
:10EB2400E3786B710126304605B0F0BD7846F8F7FE
:10EB3400B5FBD9E7194BD3F804352A685169A07895
:10EB440051F82010029112690192174A0092BA22D8
:10EB540014490420FDF754FFCFE77846F8F79EFBED
:10EB6400D5E70E4BD3F804352A68116A6879E6783C
:10EB740051F82660039651F820100291126901920F
:10EB84000A4A0092C92207490420FDF739FFC7E762
:10EB94000126C8E7383300203433002000B0004099
:10EBA400D0FB0300C7FB0300DCFB0300E8FB03000E
:10EBB4002DE9F04107460E469046427901680C68FB
:10EBC4000D7904EB8505194613B9D2B203791BB943
:10EBD40004EB8104043410E0AC42FBD2237883F0CC
:10EBE40080039342F6D00434F6E742462146384681
:10EBF400FFF744FF034658B90434AC4207D22378E4
:10EC0400B342F2D013F0800FF6D0002300E00023CB
:10EC14001846BDE8F081000030B583B00D460446C7
:10EC240098B1B5B125606B7963710023A371114B61
:10EC34001B6813F4803F03D00F4B1B68032B0CDCC1
:10EC44002046FFF7F4FE03B030BD7846F8F726FB04
:10EC5400E7E77846F8F722FBE4E7084BD3F80435F6
:10EC64002A690192064A0092DE2206490420FDF731
:10EC7400C7FEE5E7383300203433002000B00040FD
:10EC840094FB0300C7FB030070B584B00D46164621
:10EC9400044608B31B4B1B6813F4803F03D01A4B84
:10ECA4001B68032B1CDCA3790133DBB2A3710023A3
:10ECB400324629462046FFF77BFF38B92379FF2BDC
:10ECC40004D0324629462046FFF772FFA379013B60
:10ECD400DBB2A37104B070BD7846F8F7DFFAD9E768
:10ECE4000A4BD3F804352268D16951F825100291F2
:10ECF40012690192064A0092E92206490420FDF7AE
:10ED04007FFED0E7383300203433002000B00040C9
:10ED140088FB0300C7FB03008079003018BF012083
:10ED24007047000010B50D4B834202D07846F8F7C7
:10ED3400B5FA0B4B5B686BB1094C237803EB830387
:10ED44005A01084810446168043006F0CBFE0023E1
:10ED5400636010BD7846F8F7A1FAEDE76856002025
:10ED6400B457002074560020F8B50F461646134BCE
:10ED7400834202D07846F8F791FA114B5B68C3B12D
:10ED84000F4D6C682A23A374731C6374324639468E
:10ED940004F1130010F0A6FA2B7803EB83035A0155
:10EDA400084810442146043006F052FE00236B60EC
:10EDB400F8BD7846F8F772FAE2E700BF685600201B
:10EDC400B45700207456002010B50C46144B8342EF
:10EDD40002D07846F8F762FA124B5B6813B17846B2
:10EDE400F8F75CFA2378616803EB83035A010E4851
:10EDF40010440231043006F0EDFD0A4B586068B14E
:10EE0400E3680360237803EB83035A01064B9B58A2
:10EE140003712278034B1A70002010BD0220FCE716
:10EE240068560020B45700207456002008B5064BDD
:10EE3400C01A8010054B03FB00F00B46C1B2044816
:10EE4400FFF71AF908BD00BF78560020976FF996AE
:10EE54006856002070B5104C0126254645F8046B11
:10EE64004FF480730D4A0E49284606F0CFFE28461B
:10EE740006F08EFDC4F8A060A4348023094A002162
:10EE8400204606F0C3FE204606F082FD32460649BF
:10EE94000648FFF709F970BD74560020BC570020DE
:10EEA40031EE0200BC580020FCFB03006856002031
:10EEB40038B504460D46012806D84DB104EB840448
:10EEC4006301054AD55038BD7846F8F7E7F9F4E709
:10EED4007846F8F7E3F9F1E77456002010B50446D4
:10EEE400012802D97846F8F7D9F904EB84046301C0
:10EEF400014AD05C10BD00BF7456002038B50446EA
:10EF04000D46012802D97846F8F7C8F904EB8404C1
:10EF14006301034818442946043006F0F3FD38BD64
:10EF24007456002010B50446012802D97846F8F733
:10EF3400B5F904EB84046201034B1344586F034B8B
:10EF4400A3FB0030800910BD74560020D34D62101D
:10EF540038B504460D46012802D97846F8F79EF9DB
:10EF640004EB84046301034818442946043006F082
:10EF74000DFE38BD7456002008B50020FBF7E4FBF5
:10EF840008BD08B503780D2B00D008BDFFF7F4FFCA
:10EF9400FBE770B582B004460E46C38AADF8003074
:10EFA4000523ADF80230684605F05AF9054610B15C
:10EFB400284602B070BD0DF106022146208A05F0F4
:10EFC4004DFC05460028F3D101AB3246BDF80610CE
:10EFD400E08A05F0C3FE05460028E9D1217E01F050
:10EFE4000101D4F81200FAF71FFF48B9BDF8040074
:10EFF4000FF078FC05460028DAD102F025F9D7E7AE
:10F004007846F8F74BF9F1E708B502F00DFE05F084
:10F01400ADF8FAF74DFC08BD00B583B001A805F0C2
:10F0240061F9BDF80400003018BF012003B05DF899
:10F0340004FB000070B582B0002831D004460D46B0
:10F04400FBF748FA064610B1304602B070BD05F031
:10F05400E9F802F0F1FD20690FF00CFC06460028E7
:10F06400F2D16369A269217F0191009259220021A2
:10F074000C480FF0B5FE06460028E5D1236A03B11B
:10F08400984704F0B1FF02F0FBFBFFF7C5FF04460D
:10F0940018B9002DD8D02C70D6E701F055FAF8E74E
:10F0A4000E26D1E73C59002008B5FFF7B5FF10B98B
:10F0B400FBF77EFA08BD01F0F3FAF9E708B5FEF7AD
:10F0C40013FC18B90348FBF7D9FA08BDFFF754FF3E
:10F0D400FBE700BF4433002076DF70477FDF7047D3
:10F0E4008FDF704790DF7047A8DF7047AADF704753
:10F0F400AEDF7047B1DF7047B5DF704710B431B988
:10F1040083B2934208D808465DF8044B7047401A0E
:10F11400904203DC0320F7E70120F5E70220F3E740
:10F12400002313B14FF6FF7070470A494FF4A672DB
:10F1340002FB0312918B4FF6FF72914201D001330F
:10F14400EFE704494FF4A67202FB0312908398B2CE
:10F15400704700BF98590020002313B14FF6FF7089
:10F16400704706494FF4A67202FB0312928B824247
:10F1740001D00133F1E798B2704700BF98590020DD
:10F1840090F83201003018BF0120704790F8EC006D
:10F194000B79013B984214BF0020012070470329DA
:10F1A40007D890F831318B4205D0FF2B05D00020D1
:10F1B400704700207047012070470120704708B550
:10F1C40008881321FFF788FF20B1082802D0784669
:10F1D400F8F764F808BD000070B504468688304628
:10F1E400FFF7BAFF4FF6FF73984216D00546E4883E
:10F1F400162C05D9442C11D8452C28BF452400E0F1
:10F20400172421463046FFF777FF48B9033C064BE5
:10F214004FF4A67202FB0535EC8370BD4524F0E77C
:10F224007846F8F73BF8F1E79859002030B585B0F7
:10F234008088FFF775FF4FF6FF73984219D0044694
:10F244000D4D4FF4A67000FB04F000F12001294499
:10F2540018302844D8220C310830F9F7B9FC0323BC
:10F264008DF800308DF80140AB69D5F86811684617
:10F27400984705B030BD00BF98590020D0F8E81079
:10F2840051B110B504460430F9F7CAFD0023C4F89F
:10F29400E83084F8EC3010BD704710B5044600F532
:10F2A4009A70FBF7C7FC002384F83231FF2384F8FB
:10F2B400313110BDF8B50646B8B90E4C4FF4A675F9
:10F2C40005FB06F505F118062644371D3846FFF7F9
:10F2D400E4FF3846FFF7D2FF06F10800F9F7CFFC48
:10F2E4002C444FF6FF73A383F8BD7846F7F7D6FF97
:10F2F400E3E700BF9859002010B584B08088FFF779
:10F304002BFF4FF6FF7398420DD00446FFF7D2FF50
:10F3140004238DF800308DF80140044B9A69D3F82A
:10F3240068116846904704B010BD00BF985900208A
:10F3340010B50446FBF74AFD0349014404F59A70ED
:10F34400FBF7A8FC10BD00BF002D31012DE9F047EB
:10F354008EB0894616460546002867D0002965D038
:10F364000027002F66D04F4A28681060AB8893802E
:10F37400C2F818902B88ADF8343001208DF836008F
:10F3840006320DA9FFF7B0FE00287ED1AB88ADF898
:10F394003430002306930793089309930A930B933D
:10F3A4000C9304228DF818200122114662F30711F0
:10F3B4008DF81410114662F307118DF81510924060
:10F3C40042F001028DF816200293039304930DABCF
:10F3D400009305AB01934223ADF80C30314800F1A2
:10F3E40010036A4606A9C088FFF780FE002850D1A2
:10F3F4006B88ADF834300023069307930893099380
:10F404000A930B930C9310238DF81830254800F1C0
:10F4140008036A4606A9C088FFF768FE00283CD1A5
:10F42400204BC3F868610EB0BDE8F0877846F7F763
:10F4340035FF95E71B4B4FF4A67404FB07F41A1928
:10F444001421D183FF2182F84D111749C2F85811B4
:10F4540004F11808984408F10401C2F860114FF649
:10F46400FF7191832034234403F10C044FF0D80A34
:10F474005246002120460FF05EFF5246214608F115
:10F484000800F9F7A5FB01376BE77846F7F706FFA5
:10F494007CE77846F7F702FFAAE77846F7F7FEFE1F
:10F4A400BEE700BF98590020C3F10200F0B583B055
:10F4B4000D4614461E46074610BB032D24D8422C85
:10F4C40026D81E4A4FF4A67303FB07239A8B4FF6E4
:10F4D400FF739A4230D0A21D02A9002341F8043DD3
:10F4E4004FF4A67000FB07F01830144B184492B286
:10F4F4000830F9F7EDFB78B1042818D1002014E0A6
:10F504007846F7F7CBFED8E77846F7F7C7FED6E795
:10F514007846F7F7C3FED4E70198466001340472D5
:10F52400437A65F3050343720A3003B0F0BD7846AD
:10F53400F7F7B4FE0020F8E70020F6E7985900201A
:10F5440038B504460D46B1B1CCB9114A4FF4A6738F
:10F5540003FB04239A8B4FF6FF739A4213D04FF4A4
:10F56400A67000FB04F01830094B1844691F0830DA
:10F57400F9F756FC38BD7846F7F790FEE4E778468D
:10F58400F7F78CFEE1E77846F7F788FEE7E700BF78
:10F594009859002070B5064680B90A4C4FF4A675F8
:10F5A40005FB06F505F5A47020440830FBF742FB83
:10F5B4002C441321A08BFFF78FFD70BD7846F7F71D
:10F5C4006DFEEAE7985900202DE9F04786B005461C
:10F5D400474A4FF4A67303FB0023D3F8046116B320
:10F5E400434A4FF4A67303FB052393F80821337AA7
:10F5F4009A421CD2347A3E4A4FF4A67303FB052385
:10F6040093F808A1B3F81E904A4651462046FFF7E6
:10F6140075FD8046471EFFB2012F59D958B1032802
:10F6240009D000240AE07846F7F738FED8E7784690
:10F63400F7F734FEDEE7A4EB0A04A4B2A14549D3EC
:10F644002B494FF4A67202FB051292F80801331DF0
:10F65400034403F1050C587968F3871058710023AB
:10F66400CDF80A30ADF80E30ADF806400B89ADF890
:10F674000830CDF814C00DF10603049301238DF86E
:10F684000A3002A9908BFFF733FD082826D01328EF
:10F694001BD018B9BDF80630A34202D07846F7F75C
:10F6A400FDFD134A4FF4A67303FB052393F80831B9
:10F6B4001C44E4B2013CE4B2012F13D90C4B4FF4C7
:10F6C400A67202FB053585F8084106B0BDE8F0874F
:10F6D4004C46B3E77846F7F7E1FDB1E72846FFF774
:10F6E40059FFF2E733445B7A26447372E6E700BFBE
:10F6F4009859002070B505460E4601B31DBB254A36
:10F704004FF4A67303FB05239A8B4FF6FF739A42BB
:10F714003ED04FF4A67404FB05F404F118031D4C09
:10F724001C44083436F80A2CA6F10A012046F9F7DD
:10F73400FEFA2046F9F74DFB48B9002070BD784623
:10F74400F7F7ACFDDAE77846F7F7A8FDD7E74FF40B
:10F75400A67101FB05F1F8310E4B19440C3120461A
:10F76400F9F716FB60B90B4A4FF4A67303FB0523A4
:10F77400D3F8043143B12846FFF726FF0020DDE724
:10F784007846F7F78BFDEEE77846F7F787FDF2E763
:10F794000820D3E79859002070B584B0FFF7DCFC4B
:10F7A4004FF6FF7398425BD005462E4B4FF4A6727A
:10F7B40002FB00F202F118041C4404341344D3F88D
:10F7C4000461002E3DD0311D2046FFF7DFFC0028E8
:10F7D40043D02046FFF752FD01238DF800308DF809
:10F7E4000150737AC3F305038DF8083073680193ED
:10F7F4001C4CA369D4F86811684698474FF4A67363
:10F8040003FB05F318331C4408342046F9F7E1FAE6
:10F8140030B34FF4A67101FB05F1F831114B1944D3
:10F824000C312046F9F7B4FA78B90E4A4FF4A673AE
:10F8340003FB0523D3F804315BB12846FFF7C4FE6C
:10F844000EE07846F7F72AFDBDE77846F7F726FD80
:10F85400EBE77846F7F722FDEFE72846FFF7B4FE1B
:10F8640004B070BD985900202DE9F04784B00446D7
:10F874000D464FF4A67303FB00F318332C490B44D5
:10F884001E1D013A97B22B789B09022B04D0032B3F
:10F894001ED0FFF77FFE18E03046FFF749FD2448ED
:10F8A4004FF4A67303FB04F4061996F84E311C4476
:10F8B40004F5847420443A46691C04300FF012FDA8
:10F8C40096F84E21174486F84E7104B0BDE8F087CF
:10F8D400DFF85C904FF4A67808FB00F809EB080AFF
:10F8E4009AF84E01404400F5847048443A46691C35
:10F8F40004300FF0F7FC00238DF800308DF8014040
:10F904009AF84D318DF8043008F584734B44043370
:10F9140002939AF84E211744ADF80C70D9F81830B8
:10F92400D9F86811684698473046FFF7B6FCCCE72B
:10F9340098590020F0B585B005460C464FF4A670E2
:10F9440000FB05F018301E4B1844013A96B20B78B0
:10F954009B0906D00430012B19D02846FFF71AFE64
:10F9640013E000238DF800308DF8015014F8013BAA
:10F97400C3F305038DF804300294ADF80C60104B0A
:10F984009A69D3F868116846904705B0F0BDFFF74F
:10F99400CFFC0B4F4FF4A67303FB05F505F58470FC
:10F9A40038443246611C04300FF09CFC2378C3F3C6
:10F9B40005032F4487F84D3187F84E61E5E700BF12
:10F9C40098590020F0B585B004468088FFF7C4FB41
:10F9D4004FF6FF73984209D00546E3882B4A928973
:10F9E400934205D0294A128A934214D005B0F0BD3F
:10F9F400228A022AF6D1A37C13F0010FF6D0052344
:10FA04008DF800308DF80100204B9A69D3F8681105
:10FA140068469047EAE7278A012F0CD91B4A4FF41E
:10FA2400A67303FB052393F84E31C3F142039F42AF
:10FA34001ED9002300E000231BB34FF4A67606FB77
:10FA440005F606F11803114E1E440436A17C01F09C
:10FA54003F013046FFF7A3FB98B13046FFF790FB18
:10FA640040B13A4604F112012846FFF7FDFEBDE716
:10FA74000123E1E73A4604F112012846FFF75AFF51
:10FA8400B4E72846FFF786FDB0E700BF9859002089
:10FA940000B585B00388103B472B27D8DFE803F077
:10FAA4002429265F262626262626262626262626B8
:10FAB400266B265226262C2626262626262626266B
:10FAC40026262626262626262626262626262626D2
:10FAD40026262626262626262626262626262626C2
:10FAE4003C264626267A263FFFF7A0FB05B05DF8A4
:10FAF40004FBFFF701FCF9E7037A012BF6D102239B
:10FB04008DF8003083888DF80130244B9A69D3F83E
:10FB1400681168469047E9E7FFF754FFE6E78088F5
:10FB2400FFF73AFE1E4B01221A70DFE700231A4644
:10FB340019468088FFF7DEFA0028D7D07846F7F711
:10FB4400ADFBD3E700220092019269468088FFF75B
:10FB5400C9FA0028CAD07846F7F7A0FBC6E7002305
:10FB64001A4685218088FFF7B9FA0028BED0784666
:10FB7400F7F794FBBAE700238DF800308DF80130D5
:10FB840069468088FFF7ACFA0028AFD07846F7F7CB
:10FB940085FBABE7FFF720FBA8E700BF98590020DF
:10FBA400045B00201130704710B50446C36C63B188
:10FBB4000848201A8010084B03FB00F0E16C80B267
:10FBC400FFF7BEFC0023E36410BD7846F7F766FB3D
:10FBD400EEE700BF8C5B0020A737BDE910B50446F3
:10FBE40020B1A4F15000FFF7DFFF10BD7846F7F70E
:10FBF40055FBF6E738B50546C36C73B10B4C2C1BAB
:10FC0400A3100B4C04FB03F4A4B2E96C2046FFF7E9
:10FC140071FD30B90023EB6438BD7846F7F73EFB3D
:10FC2400ECE7E96C2046FFF78BFCF3E78C5B0020E4
:10FC3400A737BDE9F8B50D461746044678B171B14A
:10FC4400A4F1500654F8043C6BB13A46294654F8E2
:10FC5400040C0FF047FB3046FFF7CCFFF8BD7846A5
:10FC6400F7F71CFBECE77846F7F718FBEDE7000025
:10FC7400F8B504460D4616461F46C36C13B17846C4
:10FC8400F7F70CFB0848201A8010084B03FB00F020
:10FC94003B46B2B2294680B2FFF708FCE06408B1E3
:10FCA4000020F8BD0420FCE78C5B0020A737BDE9E9
:10FCB40070B50D46044638B131B1A4F1500614F8BC
:10FCC4000C3C2BB9012070BD7846F7F7E7FAF4E74E
:10FCD400AB685988304600F006FE08B90120F2E707
:10FCE400EB686A6800213046FFF7C2FF0028EAD0BB
:10FCF4000220E8E710B582B00C4C0DF1070204F1C4
:10FD04001C01002005F076FBE3690BB102B010BDC5
:10FD14000DF1070204F11C01002005F06BFBE369FF
:10FD2400002BF3D17846F7F7B9FAEFE7085B002028
:10FD340008B500F1450200F14801002005F05AFB26
:10FD440008BD00B587B006A9002301F8143D026878
:10FD54004368CDF80520CDF80930092241F6280082
:10FD6400F7F750F907B05DF804FB30B58FB00546DE
:10FD74000C4600230A93ADF82C3008210DF12E0017
:10FD8400FBF776F9210A41EA0421ADF8361006AAF8
:10FD94000AA92846FBF7F4FD01238DF8043008ABCB
:10FDA40003CBCDF80500CDF80910DDF82E20DDF8E1
:10FDB4003230CDF80D20CDF81130112201A941F6D1
:10FDC4002800F7F71FF90FB030BD000010B582B05E
:10FDD400114BDC6993F8203054B13BB908340E4B15
:10FDE4005B783BB1012B0AD002B010BD3034F6E78A
:10FDF4000024F4E704F11000FFF7A3FFF4E70DF18A
:10FE0400060101A805F0C0FBBDF8041004F11800B8
:10FE1400FFF7ABFFE8E700BF085B002008B5FFF77A
:10FE240069FFFFF7D3FF08BD2DE9F04182B0054615
:10FE34000E4617469846002316220121FFF718FFA5
:10FE4400A8B90446EB6C00939DF82030424639462D
:10FE54003046FEF74FFD30B92846FFF7CBFE20466B
:10FE640002B0BDE8F0817846F7F718FAF4E7042405
:10FE7400F5E700002DE9F04383B081468846174634
:10FE84001E46002425461CB1284603B0BDE8F08375
:10FE94000B4A5C2303FB042393F844300BB901346D
:10FEA400F1E700963B464246494605484FF05C0C54
:10FEB4000CFB0400FFF7B8FF0028F0D00425EEE7A0
:10FEC4008C5B00200378042B00D07047C3681B7838
:10FED400012BFAD010B5044601690948FCF788FCE7
:10FEE40000B110BD637E227E6169A068FFF7C2FF86
:10FEF4000028F6D121690248FCF7A4FCF1E700BF11
:10FF04002C5B002010B5034C201DFAF793FE002350
:10FF1400237010BD085B002010B5044600F06DFC92
:10FF24000023A36410BD70B582B0044619E03035D7
:10FF3400F9F754FF0646F9F771FF94F8453000339A
:10FF440018BF012300930346324629462046FFF793
:10FF54006BFF70B904F1450204F14801002005F07B
:10FF640049FAA56C2DB194F84530002BDFD1083542
:10FF7400DEE702B070BD10B504460846FFF712FE76
:10FF84000023024602212046FFF772FE18B9E06CF6
:10FF9400FCF70FF910BD0020FCE730B583B005462F
:10FFA4001446012200920A462146FCF71DFA58B96C
:10FFB400EB7A2BB1AB7A2BB96B8833B9012004E00F
:10FFC400002002E0002000E0002003B030BD012A40
:10FFD40001D00920704708B5097800F01BFC08BD62
:10FFE40070B590B0402A18D812F0010617D1520803
:0CFFF40033460AE031F813502C0A44EAAE
:020000023000CC
:10000000052410AD05EB430525F8404C0133934220
:10001000F2D3694600F013FC304610B070BD0926DB
:10002000FAE70926F8E770B590B0402A18D812F020
:10003000010617D1520833460AE031F813502C0A52
:1000400044EA052410AD05EB430525F8404C013387
:100050009342F2D3694600F01FFC304610B070BDE9
:100060000926FAE70926F8E770B588B004460D4678
:10007000164600230193029303930493059306937A
:1000800001238DF80F30F9F7B1FE059006950DF1BB
:100090001E0103A805F07AFA04A8F9F739FE80B921
:1000A000054601A9E06CFCF71CF80123E26C31461F
:1000B00001A8FCF7DCF92046FFF79EFD284608B0B2
:1000C00070BD2046FFF772FD1125F7E738B50446ED
:1000D0000D460421FFF751FF80B10322027094F80E
:1000E00042204270B4F840100A0A42EA01224280DB
:1000F000042229462046FFF7B7FF38BD0420FCE75D
:1001000070B59AB01446531E412B16D92A4B1B6862
:1001100013F0010F0FD0294B1B68012B0BDD284B6F
:10012000D3F804350192274A00924FF4057226490C
:100130000220FCF767FC1AB070BD054609AB03A8A6
:10014000FFF72DFFA0B91C4B1B6813F0010FF2D075
:100150001A4B1B68032BEEDD194BD3F804351B4AF1
:10016000009240F20F2218490420FCF74BFCE2E712
:1001700009A8FCF720F80646214603A8FCF70FF86B
:10018000421E3378012B12D033B1022BD3D1711C14
:100190002846FFF748FF03E0711C2846FFF719FFC8
:1001A0000028C8D108992846FFF790FFC3E7711CC3
:1001B0002846FFF717FFF3E73833002034330020D9
:1001C00000B0004054FC030037FC030040FC030077
:1001D000F0B58BB005460C4617461E460023049327
:1001E0000593069307930893099301238DF8103024
:1001F000FAF7EEFD05901D4BEB1A9B101C4A02FB13
:1002000003F3ADF818301B4B1B6813F0010F03D03C
:10021000194B1B68032B09DC184B01221A709442FE
:1002200018D08CB1022C1BD00BB0F0BD144BD3F8FE
:10023000043502960194134A009240F22522124995
:100240000420FCF7DFFBE7E704AA31463846FBF75A
:10025000E9FEE9E704AAF1B23846FEF783FBE3E7DB
:10026000324639462846FFF74BFFDDE78C5B00201E
:10027000A737BDE93833002034330020F85B002075
:1002800000B00040FCFC030037FC030038B50D460D
:100290000246A8B90024134B5A701B789BB9ADB91C
:1002A0001148FAF7C9FC4FF448612046F6F722FFDF
:1002B000FFF78EFDF6F728FF0A4B01221A7038BDB2
:1002C0004EF66024E7E7F6F72FFFE8E7FFF714FDA7
:1002D000FAF77EFD034B19690144181DFAF7DCFC9F
:1002E000E1E700BF085B00200C5B002070B582B026
:1002F00004464678864D5C2000FB06552278052A88
:1003000000F2EE80DFE812F083009F00CB000600D1
:10031000400069007F4B1B6813F0010F03D07E4B38
:100320001B68032B1ADCFFF7EFFD794A5C2303FB04
:100330000626012386F84430784A13702846FFF7D2
:10034000EDFD2846FFF7F6FC0023194693B100297E
:100350004FD101210020FFF799FF4AE0704BD3F8FD
:100360000435704A009240F23F226F490420FCF7A6
:1003700049FBD8E766485C2202FB030292F844205E
:1003800002B101310133E1E7624B1B6813F0010F49
:1003900003D0614B1B68032B13DC5D4A5C2303FB1A
:1003A0000626002386F844305C4A13705F4B1B78A6
:1003B000FBB15F4B1B78E3B901210020FFF766FF1B
:1003C00017E0574BD3F804355A4A00924FF4147291
:1003D00055490420FCF716FBDFE74E4B1B6813F072
:1003E000010F03D04C4B1B68032B04DC2846FFF79E
:1003F0009CFD02B070BD4A4BD3F804354E4A0092C2
:1004000040F25B2248490420FCF7FCFAEEE7414B3E
:100410001B6813F0010F03D03F4B1B68032B06DC56
:10042000A389A26821792846FFF7D2FEE1E73C4B79
:10043000D3F80435414A00924FF418723A49042027
:10044000FCF7E0FAECE7334B1B6813F0010F03D025
:10045000314B1B68032B16DC237A002BC9D165684E
:10046000B5F1FF3F14BF00250125FAF7B1FC5C236D
:1004700003FB06F65036636802462946244830449A
:10048000FDF7FCFDB5E7264BD3F804352C4A009266
:100490004FF41A7224490420FCF7B4FADCE71D4B30
:1004A0001B6813F0010F03D01B4B1B68032B0BDCE5
:1004B0001F4B00221A701D4B1B78002B99D0012175
:1004C0001046FFF7E3FE94E7154BD3F804351D4AB9
:1004D000009240F2772214490420FCF793FAE7E7F0
:1004E0000C4B1B6813F0010F83D00B4B1B68012BC7
:1004F0007FF77FAF0A4BD3F804350192124A00927E
:1005000040F2812208490220FCF77CFA71E700BF23
:100510008C5B00203833002034330020885B0020BF
:1005200000B0004084FC030037FC0300E85B0020BF
:10053000085B002090FC0300A0FC0300ACFC03005F
:10054000B0FC0300C0FC0300D0FC030070B582B017
:1005500000241A4B1C701A4B93E803000090ADF86E
:100560000410224617496846FEF7F2FE1648174B5C
:100570000360FAF785F8164808238360154B03607B
:1005800004234360FCF727F9134B144ADA60144A3A
:100590001A611C700CB102B070BD124D5C2606FBD6
:1005A00004F606F1500002220F492844FDF77EFDB3
:1005B0003544002385F844300134EBE7E85B002044
:1005C00008FC0300ED020300EC5B0020C9FE020002
:1005D0002C5B0020485B0020085B002021FE02000D
:1005E000809698008C5B0020F0FC030030B583B04F
:1005F0000C4609B3002301930DF1030201A9204623
:1006000004F0FAFE019BDBB1019C9DF80330ECB1D4
:10061000D3B13034F9F7E4FB0546F9F701FC9DF856
:100620000330022B14BF0023012302462946204633
:10063000FFF722FC03B030BD7846F6F731FED9E76C
:100640007846F6F72DFEDFE70834E3E70024E1E71C
:100650000B78012B00D0704710B50C89104A5C2331
:1006600003FB042393F8443073B15C2303FB04239E
:1006700093F842304BB1012200F10801084B5C2095
:1006800000FB043000F008F910BD012200F1080160
:10069000034B5C2000FB043000F0D1F8F4E700BF0E
:1006A0008C5B0020084B1B785BB910B50024074B0E
:1006B000DC610121044B19702046FFF7E7FD20465D
:1006C00010BD0820704700BFE85B0020085B0020D9
:1006D00010B50F4BD86183F820100E4B01221A7011
:1006E00000231C4643B18CB9B0FA80F149090120BE
:1006F000FFF7CCFD204610BD07495C2202FB031228
:1007000092F8442002B101340133EBE71124F1E700
:10071000085B0020E85B00208C5B00200D4B1B7801
:100720007BB10D4B1B7873B10B4B5B78012B01D068
:100730000020704748B1084BDB69834207D0002096
:10074000704700207047002070470120704701204B
:10075000704700BFE85B0020085B002008B5002060
:10076000FFF7DCFF28B101210020FFF78FFD0020FB
:1007700008BD0820FCE70000134B1B7813B310B52D
:10078000114B00221A70114B1B7813B900242CB1A5
:1007900010BDF6F7C9FCFFF7B7FBF7E70C4A5C237F
:1007A00003FB042393F844300BB90134EFE7A0B204
:1007B000FEF7F2FE064A5C2303FB0423002283F8C3
:1007C0004420F2E7704700BFE85B0020085B002090
:1007D0008C5B0020014B1878704700BFE85B00205D
:1007E0000023B0F840209A4205D930F813208A42FD
:1007F00003D00133F5E7002070470120704710B5A2
:10080000044628B1002384F84230A4F8403010BDDB
:100810007846F6F745FDF5E738B50C46054618B1BC
:10082000012C05D90B2038BD7846F6F739FDF7E7DE
:100830002846FFF7E4FF85F842400020F3E72DE962
:10084000F8430F469046064610B12FB1002408E049
:100850007846F6F725FDF8E77846F6F721FDF5E747
:100860000134444516D2B6F840501F2D12D84FEA35
:10087000440937F814100029F2D03046FFF7B0FFD2
:100880000028EDD16B1CA6F8403037F8093026F867
:100890001530E5E7BDE8F883F8B50D461646044681
:1008A00010B12DB1002710E07846F6F7F9FCF8E713
:1008B0007846F6F7F5FCF5E7013A92B2A4F8402045
:1008C00034F8122024F813200137B7420CD2002349
:1008D000B4F840209A42F7D935F8170034F81310CD
:1008E0008842E9D00133F3E7F8BD38B50D46044638
:1008F00050B129462046FFF773FF94F8423013B1F8
:1009000080F00100C0B238BD7846F6F7C9FCF0E7C8
:1009100010B50446837803F00303032B21D8DFE8E6
:1009200003F0020C131981788B081A4A11681944D4
:10093000A160194B1B6800201AE083789B0803EB29
:10094000830359000B46F0E783789B08642101FB81
:1009500003F3EAE783789B0841F2707101FB03F32C
:10096000E3E77846F6F79CFC0023DEE71846DB68F1
:100970001BB19A688A1A002AF8DA18B133B1C46038
:10098000E36010BDE360044B1C60FAE7C460002321
:10099000E360F6E7145C00201C5C002010B56F4B90
:1009A00019688B7803F003036D4A1278934240F381
:1009B000B0808C686B4B1B68E41A6B4B03FB04F430
:1009C000032A09D8DFE802F0020D0406664B09E0AD
:1009D000664B07E0664B05E07846F6F761FC0023BE
:1009E00000E0644BB4FBF3F35C4A1268927802F0C7
:1009F0000302022A19D03AD8012A6AD102F1CC3274
:100A0000A2FB0312D20802EB820251008B4202D0F9
:100A1000002213465FE0FAF7DBF900F5742303F5D3
:100A2000107301224E490A7055E04D4A117839B9C8
:100A3000514AA2FB03025209642000FB12326AB140
:100A4000012902D00022134645E04C4AA2FB0312C2
:100A5000D20802EB820251008B4249D1FAF7B8F971
:100A6000424B03443E4A02211170012233E03C4ACA
:100A7000117841B9424AA2FB0302D20941F27070D7
:100A800000FB123282B1012904D0022915D00022C4
:100A9000134620E03B4AA2FB030292094FF4167072
:100AA00000FB1232002AF0D1FAF792F9304B0344DE
:100AB0002B4A0321117001220DE0334AA2FB0312DD
:100AC0005209C2EB021291008B42EDD00022134674
:100AD00001E000221346002A3DD1FAF779F90446D5
:100AE0001F4B1B78032B0CD8DFE803F00510070918
:100AF00000221346EFE71C4B09E01C4B07E01C4BA0
:100B000005E07846F6F7CCFB002300E0194B2344C0
:100B100021E0FAF75DF90446104B1B689B7803F05F
:100B20000303032B09D8DFE803F0020D04060E4B84
:100B300009E00E4B07E00E4B05E07846F6F7B0FBF8
:100B4000002300E00B4B2344044A12689278C2F35E
:100B5000010203490A70184610BD00BF1C5C00204A
:100B6000195C0020145C0020A0860100809698008B
:100B70000046C32340420F001F85EB51CDCCCCCCA7
:100B8000F1197605B5814E1B8988888810B5294BE7
:100B90001B7873B9284B1B68002B42D0FFF7FEFE71
:100BA0000146244B1B78002B33D02448FAF774F805
:100BB0003AE0224B5C68FAF70BF9241A204B1B78B9
:100BC000032B09D8DFE803F0020D04061D4809E0F5
:100BD0001D4807E01D4805E07846F6F761FB002058
:100BE00000E01B48001B164B1B7843B94CF25033F6
:100BF000984204D9174A136801331360CAE74009C1
:100C0000154BA3FB0030134A136803EBD0101060A0
:100C1000C0E7084B01221A7008484160F9F7DAFF73
:100C200002E0044B1B7803B910BD0448FAF704F83E
:100C3000FAE700BF185C00201C5C0020FC5B002071
:100C4000195C0020A0860100809698000046C3230E
:100C500040420F00145C0020C55A7C0A30B583B0B6
:100C600006E063680199284698472046FFF750FE42
:100C7000104B1C68D4B1A3680F4A1268934204D089
:100C80000D4A12689B1A002B10DA2588E268094B7E
:100C90001A6002A9002341F8043D284601F026FD10
:100CA0000028DED07846F6F7FBFADAE7FFF76EFFAA
:100CB00003B030BD1C5C0020145C002008B5134B51
:100CC0001B78032B1ED8DFE803F0020C1116104A24
:100CD0001368013313600F4B00221A70FFF7BEFF39
:100CE00008BD0B4A13680A331360F4E7084A136817
:100CF00064331360EFE7064A136803F5BB53103300
:100D00001360E8E77846F6F7CBFAE4E7195C0020D1
:100D1000145C0020185C002010B50446FFF7F8FDB5
:100D2000034B1B68A34200D010BDFFF72FFFFBE76A
:100D30001C5C0020074A002313605360D3601361DA
:100D4000536105499160054A1360054A1360054ADD
:100D500013707047FC5B0020BD0C0300145C002086
:100D60001C5C0020185C002070B50E461546044639
:100D700028B1FAF7CFFC144B1B68002205E0784637
:100D8000F6F78EFAF5E71A46DB680BB1A342FAD103
:100D9000A17866F3010165F38701A17013B13AB13F
:100DA000D968D16045B903B152B1FAF7D3FC70BD2F
:100DB000D86805490860F5E72046FFF7ADFFF4E77E
:100DC000FFF7E4FEF1E700BF1C5C002070B50E46A3
:100DD0001546044640B1A378C3F301033370A378EA
:100DE000C3F385032B7070BD7846F6F759FAF2E726
:100DF00010B44FF6FF7399420CD00C4A43001C18F4
:100E000061000C461144C97822444B1CD3705DF834
:100E1000044B7047054A43001C1861000C461144FE
:100E2000897822444B1C9370F1E700BF205C0020BE
:100E300030B482B001911A4943001D186C000C4473
:100E4000A57803445C002144CB78DD4201D0002327
:100E500003E0002020E001339BB2052B1BD81D4688
:100E6000104C342101FB034189898142F3D13421A3
:100E700001FB03414C88BDF806108C42EBD13421B4
:100E800001FB05F507494C5BBDF804108C42E2D12B
:100E90001380012000E0002002B030BC704700BF8A
:100EA000205C0020745C002082B000230093027854
:100EB00002F0C003402B0ED00CD9802B1BD0C02BCE
:100EC0000FD1ADF800204278837843EA0223ADF8D1
:100ED000023006E02BB9ADF800204FF6FF73ADF8F5
:100EE0000230009B00209AB262F30F001B0C63F3E8
:100EF0001F4002B07047437843EA0222ADF8002059
:100F00004FF6FF73ADF80230EBE782B00190000CB2
:100F10004FF6FF73984207D0BDF804300B70030AF8
:100F20004B70887002B07047BDF8043013F47F4FE7
:100F300001D10B70F6E71A0A0A704B70F2E782B023
:100F400001904FF6FF73B3EB104F0AD0BDF80400C9
:100F500020F03F0080B2C02814BF0020012002B062
:100F60007047BDF8040010F47F4F07D120F07F03D5
:100F70009BB26BB97F2809D00120F0E700F4404014
:100F8000B0F5004F14BF00200120E8E70020E6E79D
:100F90000020E4E770B506460D460024AC4207D2B7
:100FA00056F83400FFF7CBFF034610B10134F5E7E4
:100FB0000123184670BD30B482B00191002300E0D7
:100FC0000133018D994210D9416A01EBC30531F813
:100FD0003340BDF804108C42F2D16C88BDF8061085
:100FE0008C42EDD11360012000E0002002B030BC43
:100FF00070470000C289052A11D80A4B03EBC203CF
:1010000004334A0953F8223001F01F0123FA01F199
:1010100011F0010F01D1002070470120704700201E
:10102000704700BFAC5D002008B5804708BD0000D8
:101030004388C3F30B03052B19D830B41C460D4964
:1010400011F8332042F0010201F83320002313B1DC
:10105000012030BC704700EB83025168C94303EBA9
:101060004405044A02EB850251600133EFE700209A
:10107000704700BFAC5D00204388C3F30B03042B13
:1010800007D8818803EB43035A00034B9952012090
:1010900070470020704700BF205C0020F0B583B08F
:1010A0000F4616464FF47043ADF80430ADF8060015
:1010B00000252C46224601A90A48FCF702FA0446FC
:1010C00010B1B04740B10135002CF3D1AF4205DA81
:1010D0007846F6F7E5F801E04FF0FF35284603B013
:1010E000F0BD00BF4C5C002008B57846F6F7D8F894
:1010F00008BD0000F8B505460E4617461C4683B1EC
:101100003389B3F5BE7F10D2052D15D8204A34237C
:1011100003FB052393F8303013F0010F1DD100239A
:101120000BE07846F6F7BCF8EAE70923236020686D
:10113000B0FA80F04009F8BD002383B1144A34238B
:1011400003FB05239B89042B09D85FB13068FFF7A7
:10115000F6FEC8B100232360E9E70123EDE705238C
:101160002360E4E70A4A342303FB05239A884FF6F9
:10117000FF739A4208D0064B342202FB0535EA88F9
:101180004FF6FF739A42E1D107232360CFE700BFF8
:10119000745C0020F8B54388C3F30B03052B36D8E5
:1011A000021D018A042934D81C4C342101FB03415F
:1011B000C98905290AD8448AA14201D0002027E024
:1011C000174911F8341011F0010F24D0418A052974
:1011D00006D8134D15F8314044F0040405F83140A9
:1011E0000E4D342101FB03F3E9181468D2F804C052
:1011F0009768D668EC50C1F804C08F60CE6014695F
:101200000C618188008AFFF7F3FD012000E00020D7
:10121000F8BD0020FCE70020FAE700BF745C002066
:10122000AC5D002008B5064B01221A700548FCF79A
:10123000F7F800B908BD0448FCF740FBFAE700BF27
:10124000705C00204C5C0020603300202DE9F041F0
:10125000FAF760FA5D4B1B78002B48D15C4B1B788A
:101260000BB1002544E0062201215A48FCF7CFF9D2
:1012700058B10522C280062202818280FCF700FA62
:10128000534B01221A70002532E0112530E003EBA8
:101290004400514A02EB80025268D24301EB8300C2
:1012A0004260013316E011250134A4B2052C4BD85D
:1012B00005BB494B13F8343003F00303032BF3D180
:1012C000042244F440514348FCF7A1F901460028A8
:1012D000E9D02B46002BDAD00846FCF7D1F93E4A7C
:1012E00012F8343023F0020302F83430DCE708252A
:1012F0000024DBE7002402E011250134A4B2042C11
:1013000059D81DBB04EB44035A00344B13445B799A
:1013100013F0020FF1D0022244F480512D48FCF763
:1013200076F90028E8D02D4E670039194B0006EBFE
:101330000308F35A8380FCF7A3F998F8053023F0EB
:10134000020388F80530D8E70024D8E7002402E03B
:101350001125631C9CB2052C2FD875BB204A342361
:1013600003FB042393F8303003F00303032BF0D185
:10137000142244F400511748FCF749F902460028AA
:10138000E6D01749342606FB04163168D6F804C0A7
:10139000B768F0685160C2F808C0D7601061316961
:1013A00051611046FCF76CF996F8303023F00203D7
:1013B00086F83030CDE70024CDE71DB9FAF7CAF939
:1013C000BDE8F0810748FCF779FAF7E7705C002088
:1013D000715C00204C5C0020AC5D0020205C002093
:1013E000745C0020703300200378012B08D0438800
:1013F00004339BB2032B12D800230B8001207047CB
:1014000030B583B00D46044601A802F06DFF638835
:10141000BDF804209B1A2B80012003B030BD0020B2
:101420007047000008B54FF49C7200210F480DF082
:1014300084FF1E2200210E480DF07FFF3022002184
:101440000C480DF07AFF00220CE00849342303FB1E
:1014500002134FF6FF71D98099800620D8819981B7
:10146000013292B2052AF0D908BD00BF745C002099
:10147000205C0020AC5D002000B587B00F4B0393CB
:101480000F4B04930F4B05930423029302F02AFEA3
:10149000A0F580500090012301930B4A1370694618
:1014A0000A48FCF7C5F928B9074B00221A7007B0A3
:1014B0005DF804FB0648FCF701FAF8E76D15030038
:1014C000E9100300D5140300705C00204C5C002080
:1014D0005033002010B5002301E001339BB2052BEF
:1014E0000BD81F4A12F8332012F0010FF5D042F04A
:1014F00002021B4901F83320EFE7002301E001332A
:101500009BB2042B10D803EB43014A0015498A5AB9
:10151000002AF4D008465A00D418610001444A79E0
:1015200042F002024A71EAE7002301E001339BB274
:10153000052B11D80C49342202FB031292F83020FB
:1015400012F0010FF2D00846342101FB030142F0F2
:10155000020281F83020E9E7FFF78EFF10BD00BFDF
:10156000AC5D0020205C0020745C002070B58CB065
:1015700005460E461446012A05D0022C07D0032C3E
:1015800009D00CB070BD7846F5F78AFEF5E77846CD
:10159000F5F786FEF3E72C22002101A80DF0CDFE21
:1015A00010238DF8043002238DF808300396EB6881
:1015B00005932B69069301A8F7F72EFAE1E70000DF
:1015C0002DE9F04F95B004AF82460C46154607F161
:1015D0003C03FFF78FFD20B9F86B4437BD46BDE8EB
:1015E000F08F07F1380002F07FFE9C4A342303FBA2
:1015F0000A239E897B8F9E4280F029813B8F1E4467
:10160000B6B2002D00F0A180B5F81E80B5F8249088
:1016100007F130030C3595E8030083E803008F4B96
:10162000342202FB0A3A9AF81050FF2D00F0A080F5
:1016300007F1300001F032FC8246002840F09B8028
:10164000BAF1000F04D097F83030012B00F0FD8084
:10165000EB462422002107F10C000DF06EFE2389D9
:1016600022683A604FF6FF71B1EB124F00F0A08094
:1016700003221344073323F00703ADEB030D0DF1F1
:10168000100A07F124024146484603F041FDF86381
:10169000002840F0948007F10C0307F1300292E833
:1016A000030083E80300BE82BD75A37AFB75E37A6D
:1016B0003B76C7F81CA023892268BA604FF6FF71F9
:1016C000B1EB124F7DD0032213443B84E368FB62ED
:1016D00051462068FFF719FC23687B604FF6FF72C4
:1016E000B2EB134F74D003202289616850440DF08F
:1016F000FBFD002107F10C00F8F794FFF8630028C8
:1017000040F0A280564B1B6813F4005F03D0554B8A
:101710001B68042B63DC524B1B6813F4005F00F062
:101720009380504B1B68042B40F38E80E846B4F83E
:1017300008C04FEA4C030833DB08A8EBC3039D46FF
:101740000DF1100E7646002369E0444A342303FB72
:101750000A23B3F8048007F13001D88802F0B2FE02
:10176000002876D17B8E002B75D04FF6FF7956E797
:101770003D4B1D785CE7E368FB6023683B61636871
:101780007B6123893B837E8307F11C0307F13002D1
:1017900092E8030083E8030087F82450A7F8268026
:1017A000A7F8289007F10C0001F088FBF86347E7E1
:1017B0003A88FF2A01D902225BE7012259E7DD4678
:1017C0000BE73A89FF2A01D902227DE701227BE754
:1017D000BB88FF2B01D9022086E7012084E7234B39
:1017E000D3F8043522880192214A00924FF4CC723A
:1017F00020490520FBF706F98DE76268D25C4FEAC5
:10180000121959001C4D286810F8090006F8130039
:1018100002F00F0201312868825C72540133634583
:10182000EBD300230EF81C30104BD3F80435CDF861
:1018300008E0124A0192124A009240F299120D49B0
:101840000520FBF7DFF8C546DD46F86BC5E610203E
:10185000C3E60520C1E61020BFE600BF745C00208F
:1018600038330020343300208033002000B00040A3
:1018700084FD030079FD03003C33002098FD030044
:1018800094F60300F8B5FCF731F828B9FAF70CF82C
:101890000028F8D020BFF6E75F4B00221A70012124
:1018A0005E48FBF7E7FD002800F0B480C288052AF7
:1018B00040F0A8800289062A01D00024A3E0838892
:1018C000062B01D000249EE0534B01221A70544A8B
:1018D00006214FF44050FFF7E1FB002820DA0023F7
:1018E0001C46002B00F08F8092E04E4C5A001A44A8
:1018F0005100621800209070D0706052517921F030
:10190000020151710133042BEFDD474A05214FF4E9
:101910008050FFF7C3FBC743FF0F1FB90023DFE76A
:101920000023F0E7414A06214FF40050FFF7B6FBD1
:10193000002861DD002634E07846F5F7B1FC48E088
:1019400008240FE07846F5F7ABFC12E051420A405C
:10195000374901FB02F2D20E36498C5C04EB43148A
:1019600000E00824082C1AD0A0B202F065FD00287F
:10197000E8D10134072CF4D8630955F8232004F08A
:101980001F04012101FA04F461420A40002ADDD15A
:10199000013302D155F82320F8E70824E2E70136A5
:1019A000B6B2052E29D8244A342303FB06239A898C
:1019B0004FF6FF739A42F2D01F4B342404FB0634D7
:1019C000E0884FF6FF73984203D002F0A1FC002894
:1019D000B2D1E289062AE2D0184B03EBC2031D1DE7
:1019E0005B68002BACD05A421A40114B03FB02F348
:1019F000DB0E104AD45CB5E700270FB101236FE777
:101A000000236DE70024044B00221A70FFF70AFC44
:101A10002046F8BD0024FBE7715C00204C5C0020F0
:101A200031100300205C00207910030095110300A1
:101A300031B57C0730FD0300745C0020AC5D0020F4
:101A4000F0B583B0064600F11404204603F074FD9F
:101A500008B903B0F0BD4FF6FF73ADF80230694628
:101A60002046FFF7C1FC074608B100241EE00DF137
:101A70000201204602F0CCFD0028F6D07846F5F7AA
:101A80000FFCF2E7BDF802102846FFF7B3FA1CE09E
:101A9000254A342303FB04235A6A019902EBC1024D
:101AA0005568DA6A3146A0B2A8470134052CD0DC6B
:101AB0001D4B342505FB0435002FE3D0AB89BDF861
:101AC0000000984214BF00200120174A342303FB72
:101AD000042393F8303013F0010FE6D00028E4D04F
:101AE000342303FB04F308331344F28B510953F8F6
:101AF000213002F01F0223FA02F212F0010FD4D0BB
:101B000001AA31682846FFF756FA0028CDD0337D68
:101B1000012BBDD1044A342303FB0423DA6A314686
:101B2000A0B201F0A3F8B3E7745C002070B590B0E8
:101B3000044600284BD02068FFF7B6F90F9085B215
:101B40007F2D42D0304B1B6813F4005F03D02F4B26
:101B50001B68042B3FDCE06902F0DDFD0646A0694E
:101B600002F0C2FD0F9A059223684FF6FF71B1EBA8
:101B7000124F3CD0032213440693A388BDF83E10B5
:101B80004FF6FF72914238D003229B1AADF81C30F9
:101B9000237A8DF820306389ADF82230E368099309
:101BA000237C8DF82830638AADF82A3063690B9363
:101BB00094F820308DF83030ADF83260636A0D93C0
:101BC000ADF8380005A8FFF73BFF10B070BD7846B0
:101BD000F5F766FBAFE70E4BD3F8043501950D4AD8
:101BE0000092F1220C490520FAF70CFFB3E7FF2D14
:101BF00001D90222BFE70122BDE7FF2D01D8012252
:101C0000C3E70222C1E700BF38330020343300208D
:101C100000B000401CFD030079FD030008B5037807
:101C200003B108BD0430FFF781FFFAE708B5FFF7FD
:101C3000F9FB01F065F8FFF7F5FA08BD08B5FFF705
:101C4000F1FB0748074B0360F8F71AFD01F048F86D
:101C5000FFF770F801F026F9FFF70EFC08BD00BF92
:101C6000405C00201D1C0300002800F09580F8B5A2
:101C700004468268002A00F09180002900F09080DC
:101C80004FF6FF720A80C268002A00F08B808088BD
:101C9000042800F289800D460A462168FFF7C8F83B
:101CA00048B12B88444A342101FB032393F8303098
:101CB00013F0010F7AD1E168A068FFF76BF90028F3
:101CC00076D029884FF6FF73994257D0298820692A
:101CD000394B342202FB0131C8622988A06802FB1B
:101CE00001314862E068298802FB013108852988B2
:101CF000606902FB01318861298802FB0130818221
:101D0000298802FB013393F8302042F0010283F866
:101D10003020002049E099B229804FF6FF739942A4
:101D200048D0254E342707FB01611A46CB802B880B
:101D300007FB03639A802B88A28807FB03639A81C1
:101D40002B88628807FB03635A802B88228807FB55
:101D500003F3F2522B8807FB0363184A12781A74B4
:101D60002188A088FFF744F82B8807FB036696F8C4
:101D7000303043F0020386F83030A7E70023052B0C
:101D8000CAD80D48342202FB030292F8302012F028
:101D9000010FC0D00133F2E70E2070470E2004E09F
:101DA0000E2002E0092000E00520F8BD0F20FCE72E
:101DB0000720FAE70420F8E7745C00208033002055
:101DC00021B108B50022FFF7FBFB08BD0E207047CC
:101DD00039B108B50B4632B111461A46FFF7F0FB90
:101DE00008BD0E2070470E20FAE7000005280AD82B
:101DF000154A342303FB002393F8303013F0010F0E
:101E000019D1002300E00023BBB1072917D80E4ADF
:101E1000342303FB0023DB888B4212D01346342289
:101E200002FB0030C18090F8303043F0020380F8AC
:101E30003030002070470123E6E705207047072077
:101E400070470020704700BF745C00200A46C1B193
:101E500005280AD80D49342303FB001393F83030CA
:101E600013F0010F0BD1002300E000235BB1074BFF
:101E7000342101FB0030C388138000207047012308
:101E8000F4E70E2070470520704700BF745C002007
:101E900005282BD8174A342303FB002393F830304E
:101EA00013F0010F24D0342303FB00239B7C03F0A9
:101EB000070301F0070293420CD00E4B342202FBC1
:101EC0000030817490F8303043F0020380F83030F5
:101ED00000207047074A342303FB00239A7CC1F398
:101EE000C403B3EBD20FE8D1002070470520704740
:101EF00005207047745C00200A4691B1052812D86D
:101F00000B49342303FB001393F8303013F0010F17
:101F10000BD00B46342101FB0030837C1370002072
:101F200070470E207047052070470520704700BF9E
:101F3000745C0020052839D870B5224C342303FB8B
:101F4000004393F8303013F0010F31D0342303FBFA
:101F500000439B6973B33F2A2ED803292ED834231C
:101F600003FB00435B7CB2EB930F07D1342303FBED
:101F700000435B7C03F003038B4221D0114C3423DC
:101F800003FB00F025186B7C62F3870361F3010308
:101F90006B74103020440430FEF7E6FE95F83030C4
:101FA00043F0020385F83030002002E0052070473E
:101FB000052070BD0620FCE70720FAE70720F8E7B8
:101FC0000020F6E7745C002021B30B4622B310B565
:101FD00005280AD8134C342101FB004191F8301038
:101FE00011F0010F14D1002100E00021B1B10D4C1E
:101FF000342101FB0041896991B11946342303FB67
:1020000000F0103020440430FEF7E0FE002010BD48
:102010000121EBE70E2070470E2070470520F6E700
:102020000620F4E7745C002005280AD8194A3423F6
:1020300003FB002393F8303013F0010F0CD1002381
:1020400000E000231BB3134A342303FB0023DB8986
:10205000062B03D0002070470123F3E70023052B54
:1020600013D80D4A12F8332012F0010F01D00133BA
:10207000F5E742F00102084901F83320054A34210E
:1020800001FB0020C3810020704704207047052019
:10209000704700BF745C0020AC5D002005280AD8A2
:1020A000214A342303FB002393F8303013F0010F4F
:1020B00030D1002300E0002373B31B4A342303FB19
:1020C0000023DA89062A29D0072929D830B4174BEA
:1020D00003EBC20304334C0953F8242001F01F0121
:1020E00022FA01F515F0010F1CD1012505FA01F1C5
:1020F0000A4343F824200C4B342202FB0030C189F0
:102100000A4A12F8313043F0020302F8313000205D
:1021100030BC70470123CFE7052070470620704789
:10212000072070470020F3E7745C0020AC5D0020BE
:1021300005280AD8224A342303FB002393F83030C1
:1021400013F0010F31D1002300E000237BB31C4AC0
:10215000342303FB0023DA89062A2AD007292AD848
:1021600030B4184B03EBC20304334C0953F824205A
:1021700001F01F0122FA01F515F0010F1DD0012514
:1021800005FA01F122EA010243F824200C4B342223
:1021900002FB0030C1890B4A12F8313043F00203D0
:1021A00002F83130002030BC70470123CEE7052013
:1021B000704706207047072070470020F3E700BFF4
:1021C000745C0020AC5D002000293CD02DE9F84370
:1021D0000F46002A39D005280AD82049342303FBAA
:1021E000001393F8303013F0010F11D1002300E0F9
:1021F000002363B38046194B342101FB0030C389AF
:10220000062B26D01546B2F800900024148002E078
:102210000123EEE70134072C12D8A6B231460F4B4A
:10222000342000FB0830FEF7E5FE0028F2D02B88B2
:10223000994510D927F813602B8801332B80E9E7E3
:102240000020BDE8F8830E2070470E20F9E7052036
:10225000F7E70620F5E70920F3E700BF745C0020EC
:1022600005280AD81D4A342303FB002393F8303095
:1022700013F0010F29D1002300E000233BB3012913
:1022800027D830B4342303FB00F30833134A134434
:102290004C0953F8242001F01F0122FA01F515F032
:1022A000010F18D1012505FA01F10A4343F8242052
:1022B0000A4B342202FB003090F8303043F0020326
:1022C00080F83030002030BC70470123D6E705206D
:1022D0007047072070470020F5E700BF745C0020BE
:1022E00005280AD81D4A342303FB002393F8303015
:1022F00013F0010F2AD1002300E0002343B301298A
:1023000028D830B4342303FB00F30833134A1344B2
:102310004C0953F8242001F01F0122FA01F515F0B1
:10232000010F19D0012505FA01F122EA010243F853
:1023300024200A4B342202FB003090F8303043F066
:10234000020380F83030002030BC70470123D5E70D
:1023500005207047072070470020F5E7745C0020D7
:1023600099B370B40D4692B305280AD81B4934239B
:1023700003FB001393F8303013F0010F0AD1002350
:1023800000E000232BB316880023138023B1002024
:1023900070BC70470123F5E7342101FB00F10831DF
:1023A0000E4C21445C0951F8241003F01F04E14055
:1023B00011F0010F07D011888E420CD925F8113089
:1023C0001188013111800133E0E70E2070470E20A3
:1023D000DEE70520DCE70920DAE700BF745C0020B7
:1023E00005280AD8154A342303FB002393F830301C
:1023F00013F0010F19D1002300E00023BBB1012924
:1024000017D80E4A342303FB00239B888B4212D03B
:102410001346342202FB0030818090F8303043F0C4
:10242000020380F83030002070470123E6E70520E2
:102430007047072070470020704700BF745C002081
:102440000A46C1B105280AD80D49342303FB0013FD
:1024500093F8303013F0010F0BD1002300E000237C
:102460005BB1074B342101FB0030838813800020CF
:1024700070470123F4E70E2070470520704700BF26
:10248000745C002010F0800F05D1012805D0044BAA
:10249000187000207047072070470720704700BF62
:1024A00080330020014B1878704700BF8033002034
:1024B00005280AD8164A342303FB002393F830304A
:1024C00013F0010F1BD1002300E00023CBB181F0FA
:1024D00080037E2B17D90E4A342303FB00231B7C79
:1024E0008B4212D01346342202FB0030017490F864
:1024F000303043F0020380F8303000207047012371
:10250000E4E705207047072070470020704700BFB0
:10251000745C00200A46C1B105280AD80D4934234D
:1025200003FB001393F8303013F0010F0BD100239D
:1025300000E000235BB1074B342101FB0030037C3A
:102540001370002070470123F4E70E207047052028
:10255000704700BF745C00200A4649B1042809D8BE
:1025600000EB400043000449CB5A13800020704721
:102570000E20704705207047205C002069B110B420
:1025800004280CD800EB40004200064B13449B7813
:102590000B7000205DF8044B70470E20704705203B
:1025A000F8E700BF205C002069B110B404280CD803
:1025B00000EB40004200064B1344DB780B70002018
:1025C0005DF8044B70470E2070470520F8E700BF08
:1025D000205C00200A46D9B105280AD80E493423C8
:1025E00003FB001393F8303013F0010F0ED10023DA
:1025F00000E0002373B10849342303FB00F00B18FB
:102600005B8853800B5A1380002070470123F1E749
:102610000E20704705207047745C002030B482B0F3
:1026200001915AB3154604282AD84FF6FF73138038
:10263000002301E001339BB2052B1BD81C46114936
:10264000342202FB031292898242F3D1342202FB2C
:1026500003125188BDF806209142EBD1342202FBCF
:1026600004F4084A115BBDF804209142E2D12B80AA
:10267000002000E0052002B030BC70470E20FAE7D1
:102680000520F8E7745C002031B3F0B40F462AB39C
:10269000042825D816880023138000E00133052B79
:1026A00017D81488B4421DD20F4D342101FB0351B9
:1026B00091F8301011F0010FF0D0342101FB0351DB
:1026C00089898142EAD127F81430118801311180BB
:1026D000E4E70020F0BC70470E2070470E20F9E7B9
:1026E0000520F7E70920F5E7745C00200A46C1B130
:1026F00005280AD80D49342303FB001393F8303022
:1027000013F0010F0BD1002300E000235BB1074B56
:10271000342101FB0030C36A13600020704701239D
:10272000F4E70E2070470520704700BF745C00205E
:1027300005280AD8204A342303FB002393F83030BD
:1027400013F0010F34D1002300E0002393B370B5E0
:102750000546194C342303FB00F606F11000204413
:10276000002211460430FEF7FFFA284600F004FB71
:10277000A3194FF6FF72DA809A80997C01F0F80174
:102780006FF3C701997400201874597C01F003019C
:1027900060F301015974997D01F0030160F30101B7
:1027A000997593F8302042F0020283F8302070BD12
:1027B0000123CBE705207047745C002001281AD85C
:1027C00030B583B00546002401E00134A4B2052CE5
:1027D0000ED80DF106012046FFF732FE0028F4D195
:1027E000BDF80630AB42F0D12046FFF7A1FFECE781
:1027F000002003B030BD0720704700004FF6FF7384
:102800000B800023052B18D810B402E00133052BF0
:102810000DD80C4C2C2202FB034292F84020002AD7
:10282000F4D02C2202FB0342128B8242EED106230B
:102830000B8001205DF8044B704706230B800120BC
:10284000704700BFDC5D00200B4BB3F8203173B143
:10285000094AB2F822312C2101FB03239B6B01FBB7
:102860000020826B9B1A002B03DB012070470120A4
:1028700070470020704700BFDC5D002010B4124A92
:102880002C2303FB0020836B104C1C4400234FF6C9
:10289000FF7001E001339BB2052B11D80A492C22AD
:1028A00002FB031292F84020002AF3D02C2202FBF4
:1028B0000312926B111B0029ECDA18461446E9E763
:1028C0005DF8044B704700BFDC5D00200087930378
:1028D00070B506460C4615464FF6FF730B80042371
:1028E0001360F8F717FF164BB3F82031062B1FD8EB
:1028F000002308E012492C2202FB0312118B3288BC
:10290000914213D00133052B12D80D492C2202FB22
:10291000031292F84020002AECD121884FF6FF7272
:102920009142EFD100222A602380EBE708232B603D
:10293000F8F710FF2868B0FA80F0400970BD00BFBA
:10294000DC5D002010B50446204A2C2303FB002345
:1029500093F84030B3B11D4BB3F82031B3B11B4AEB
:102960002C2303FB0423002183F84010B2F820310C
:10297000013B9BB2A2F8203123B3B2F82231A3422B
:1029800008D010BD7846F4F78BFCE4E77846F4F7FE
:1029900087FCE4E72046FFF771FF0C4BA3F8220108
:1029A0004FF6FF73984209D00848B0F822312C2224
:1029B00002FB0303996BF8F76FF9E2E77846F4F747
:1029C0006FFCF1E70148F8F737F9DAE7DC5D002042
:1029D000F0B583B00546594BB3F8203143B105F546
:1029E0007A76564B4FF6FF72A3F82221002471E04D
:1029F0007846F4F755FCF2E72C2303FB042300216F
:102A000083F84010B2F820110139A2F8201101A971
:102A1000188BFFF76BFE48B9484A2C2303FB0423AD
:102A20005F6B01220199188BB84752E07846F4F7A2
:102A300037FCF1E7414F2C2101FB04F17B181831E1
:102A400039440431188BFFF7BBF9A7F82241B8B914
:102A50002C2303FB0473DA6B996B114499635200C6
:102A6000DA63364A2C2303FB04231A6B9B6BD31ABD
:102A7000002B2EDA31492C2303FB04139A6328E040
:102A8000042803D07846F4F70BFCEAE72B4B2C2202
:102A900002FB0434A36B03F51C434033A363274BB1
:102AA000B3F82031002B44D0244BB3F82231052B4E
:102AB00039D8224AB2F822312C2101FB03239B6B27
:102AC0005A1B34D41D4BDA6003B0F0BD1B4BA3F886
:102AD00022410134052CE2D8184A2C2303FB04239D
:102AE00093F84030002BF4D02C2303FB04231B6B02
:102AF0009B1B002B80DB114A2C2303FB04239B6BC5
:102B00009A1B002A96DB0D4AB2F822214FF6FF717C
:102B10008A42DBD009492C2000FB0212926B9B1ADF
:102B2000002BD6DAD2E77846F4F7BAFBC1E7EA1A07
:102B3000C8E7024B0022DA60C6E700BFDC5D002078
:102B400010B582B004460DF107010088FFF7E2FCE2
:102B500008BB636800934FF6FF72B2EB134F1ED0B1
:102B60000322A38913449BB29DF8072044F62060FA
:102B700000FB02F000F5433000F5A0700B2B08D9E4
:102B80000B330B4A82FB03235B1044F6206202FBEB
:102B9000030002B010BD7846F4F782FBD9E7BDF818
:102BA0000030FF2B01D90222DBE70122D9E700BF69
:102BB000ABAAAA2A2DE9F04106460C462A4A2C2344
:102BC00003FB002393F84030002B3ED1F8F700F9C7
:102BD0008046254D2C2303FB06F707F1180E05EB65
:102BE0000E03D4F800C06068A168E26845F80EC022
:102BF00058609960DA60D4F810C06069A169E26930
:102C0000C3F810C058619961DA612046FFF798FF58
:102C1000EB19D8631A6B42441A6340449863F8F77F
:102C200079FD3046FFF710FE98B90F4B2C2202FBBE
:102C30000636012286F84020B3F820210132A3F89D
:102C40002021F8F787FDBDE8F0817846F4F728FBEE
:102C5000BCE72C2303FB0653996B2846F8F71CF8B6
:102C6000A5F82261E1E700BFDC5D002070B582B00D
:102C700004460D461646052815D8F8F74BFD0DF10C
:102C800006012046FFF7BAFD48B1BDF80600134A19
:102C90002C2303FB00239A8D2B889A4207D0F8F748
:102CA00059FD02B070BD7846F4F7FAFAE5E70B4A31
:102CB0002C2303FB0023DA8D6B889A42EFD1FFF7B8
:102CC00041FEBDF80630054A2C2101FB03235B6B56
:102CD0000022314620469847E1E700BFDC5D002036
:102CE00010B5054C4FF49272002120460CF025FBE4
:102CF000024BA36010BD00BFDC5D0020D1290300A2
:102D000070B582B0F8F706FD1A4BB3F820310BB955
:102D100000240BE017480023A0F82031F7F78CFFC0
:102D2000F6E7022201992846B0470134052C1DD848
:102D3000104A2C2303FB042393F84030002BF4D0DB
:102D400010462C2202FB04F3C1180D8B4E6B183376
:102D5000002118440CF0F1FA01A92846FFF7C6FC3F
:102D60000028DED07846F4F79BFADAE7F8F7F2FCB1
:102D700002B070BDDC5D002010B582B0052828D8F7
:102D80000446F8F7C7FC0DF102012046FFF736FDB7
:102D900028B90524F8F7DEFC204602B010BDBDF8C6
:102DA0000200FFF7CFFD01A92046FFF79FFC60B9A5
:102DB000BDF80230084A2C2101FB03235B6B022281
:102DC0000199204698470024E4E77846F4F768FA2A
:102DD000EEE70524E0E700BFDC5D002030B585B0FC
:102DE000002836D00446C269002A34D00288052A59
:102DF00033D881691C4A0A441C498A422FD803AA45
:102E00000DF10A01FFF764FD08B9039D28E0211DBB
:102E10002088FEF7D5FF0546039008B104281FD18E
:102E200002A92088FFF712F805460390C0B9694649
:102E3000BDF8080001F046FB0546039080B99DF8F7
:102E40000030012B0CD12146BDF80A00FFF7B2FE7D
:102E500006E00E2504E00E2502E0052500E007252A
:102E6000284605B030BD00BF803C36FE80C3C90196
:102E700010B50AE004F11C00FEF7E2FD0648016807
:102E8000F9F729FD20460CF095F9034B1C68002C3E
:102E9000F0D1012010BD00BF045F002008B502F092
:102EA0004BFB08BD08B50348F8F776FC024B1860E9
:102EB00008BD00BF712E0300005F002070B50546FD
:102EC000808944300CF02CF900282FD004460523CB
:102ED00003712B6883606B68C36100F14403036274
:102EE000AA898284012180F82810E989418500F1AE
:102EF000300605F1100103C986E80300297E84F835
:102F00003810698B6187211DE163A98BA4F84010FB
:102F1000A96818460CF0E8F921460548F9F7B0FC15
:102F2000044B1868F8F758FC002070BD0420FCE73B
:102F3000045F0020005F002002460E4B1B6813F068
:102F4000010F0AD00C4B1B8898420FD30A484088C7
:102F500003449A420CDB002300E00023184623B10F
:102F60004A8001230B7000234B6070470023F5E774
:102F70000123F3E7105F0020C85F00204FF6FF73C6
:102F80000B800023062B26D810B40DE05A09134CF1
:102F900054F8222003F01F04E24012F0010F08D180
:102FA0000B800133062B12D80C884FF6FF72944227
:102FB000ECD00B4A32F823208242F2D1084A02EBCD
:102FC0008302D278002AECD00B80012000E00020A0
:102FD0005DF8044B70470020704700BF085F002079
:102FE000205F00200B880BB9013300E000234FF66F
:102FF000FF720A80EBB910B408E003EB8304A2006F
:103000000D4CA25A82420DD0013373B95A090B4CB0
:1030100054F8222003F01F04E24012F0010FECD11B
:103020000B80F1E70B80012000E000205DF8044BED
:1030300070470020704700BFA8600020185F002084
:103040004FF6FF730B800023062B21D810B407E046
:103050000C884FF6FF72944214D00133062B13D81C
:103060005A090C4C54F8222003F01F04E24012F0DD
:10307000010FEDD0084A32F823208242EDD10B80B7
:10308000012002E00B80E8E700205DF8044B704768
:1030900000207047085F0020205F00204FF6FF737C
:1030A0000B8000236BB10020704701330B8001209F
:1030B0001DE00C884FF6FF72944214D15A1C0A800E
:1030C00011E010B45A090B4C54F8222003F01F04ED
:1030D000E24012F0010FECD0162202FB03F2064C84
:1030E000A25A8242E1D00133002BEBD000205DF8E0
:1030F000044B7047705F0020785F00204FF6FF732D
:103100000B8000235BB1002070470B8001201CE086
:103110000C884FF6FF72944213D10B8011E010B46B
:103120005A090B4C54F8222003F01F04E24012F01D
:10313000010FEDD02A2202FB03F2064CA25A824272
:10314000E3D00133002BEBD000205DF8044B704737
:103150003C5F0020445F0020F0B416680023136039
:1031600013B10120F0BC70475C09114D55F82440A3
:1031700003F01F05EC4014F0010F06D00D4D2A247A
:1031800004FB03546488844201D00133E8E71568E6
:10319000B5420AD02A2404FB03F4064F3C5B21F815
:1031A0001540146801341460EFE70020DAE700BF2F
:1031B0003C5F0020445F002070B40D6800230B606A
:1031C00013B1012070BC70475A090D4C54F82220ED
:1031D00003F01F04E24012F0010F0CD00C68AC4267
:1031E0000BD0C82202FB03F2064EB25A20F814207C
:1031F0000A6801320A600133E2E70020E2E700BF1B
:10320000D85F0020E05F0020014688B100230BB1A9
:1032100000207047162202FB03F20648825A8A42B7
:1032200001D00133F3E7162202FB0303181D704798
:1032300000207047785F00200D4B23F8210003EB3E
:1032400081030022DA709A704B090A4801F01F01CD
:10325000012202FA01F150F823200A4340F823200A
:10326000054850F82320114340F82310704700BF51
:10327000205F0020085F00200C5F00200A68014BDF
:103280001A607047C85F002008B50B8881B21846E5
:10329000FFF7D2FF08BD0000014B1B680B607047B1
:1032A000C85F0020024B33F820300B80704700BF0E
:1032B000205F00202DE9F041013B164F162505FB4C
:1032C00003F57C19D2F80080D2F804E0D2F808C0E7
:1032D000D268C4F80680C4F80AE0C4F80EC0C4F886
:1032E00012200022627101222271618078535909F3
:1032F000094803F01F039A4050F82130134340F867
:103300002130064850F821301A4340F82120BDE80A
:10331000F08100BF785F0020705F0020745F0020A4
:1033200010B50C46431C9BB20A1D49882088FFF744
:10333000C1FF10BDF0B40B4D162303FB00F02C1899
:10334000234653F806CF5F689E68DB68C1F804C067
:103350008F60CE600B612B5A0B8063884B80F0BC72
:10336000704700BF785F002010B400EB800082003F
:10337000064B134453F8044F58689A68DB680C6096
:1033800048608A60CB605DF8044B7047A8600020FD
:1033900010B5044608B1A04710BD7846F3F780FF8A
:1033A000F9E700002DE9F84307460C469046994698
:1033B00005281AD80F4EFD00EA1B930033449B6981
:1033C0004A46414620469847ED1BAB001E447268B2
:1033D000610904F01F04012303FA04F452F82130B8
:1033E000234342F82130BDE8F8837846F3F758FFCD
:1033F000E0E700BFA0FD030010B5044650B10A4B42
:103400009C420BD30DD8E01A084CA4FB0030C0F34B
:103410008F1010BD7846F3F743FFF0E74FF6FF70CB
:10342000F7E74FF6FF70F4E7506000201F85EB517F
:1034300038B5044620B1002030B14FF6FF7038BDDA
:103440007846F3F72DFFF6E71449C82303FB001372
:1034500093F86410A1B1C82303FB00F303F1200229
:103460000E4B13440233A342E9D0C82303FB00F3FD
:1034700003F14002094B13440333A3420AD1DEE7B0
:10348000C82303FB00F303F12002044B134402336F
:10349000A342D4D0013080B2CEE700BFE05F00206D
:1034A00010B5044678B1114B9C4200D30FD9104B94
:1034B0009C4214D316D8E01A0E4CA4FB003000092D
:1034C000013080B210BD7846F3F7EAFEEBE7E01A70
:1034D0004008094CA4FB0030C0F38F00F2E74FF620
:1034E000FF70EFE74FF6FF70ECE700BF485F00208A
:1034F0007C5F0020A38B2EBA310CC33070B504461C
:103500000E461546106820B3FFF7CAFF013000E0F1
:10351000013000BB4309114A52F8233000F01F026A
:10352000D34013F0010FF3D00D4A2A2303FB0023ED
:103530005B88A342ECD12A2303FB00235B79734011
:1035400013F03F0FE4D12A2303FB002304332B6045
:1035500003E00020DDE700232B6070BD3C5F00200E
:10356000445F00202DE9F84306460D461C462348DB
:103570002A2303FB04F3C118D2F80090D2F8048088
:10358000D2F808E0D2F80CC0C1F80690C1F80A8061
:10359000C1F80EE0C1F812C0103303440020C3F894
:1035A0000900C3F80D00C3F81100C3F81500053178
:1035B0001046F9F763F8E8B910492A2303FB04F32E
:1035C000CA18002010719075CE52558063090C49BD
:1035D00004F01F04012202FA04F451F823202243CC
:1035E00041F82320074951F82320144341F8234090
:1035F000BDE8F8837846F3F753FEDDE7445F00202B
:103600003C5F0020405F0020F8B505460C4616469A
:1036100083B20A1D49882088FFF7A4FF242E05D015
:10362000142E02D07846F3F73BFEF8BD12492A2348
:1036300003FB05F3CA180120907510331944204686
:1036400050F8147F46688468C268C1F80970C1F8F0
:103650000D60C1F81140C1F815200831F9F70EF8D6
:1036600030B9054B2A2202FB05352B79EB75DCE7D7
:103670007846F3F715FEF4E7445F00202DE9F041AA
:1036800006460C4615462422002120460BF055FE26
:10369000174F2A2202FB06F2B9180B4653F8068F81
:1036A000D3F804E0D3F808C0DB68C4F80480C4F899
:1036B00008E0C4F80CC02361BB5A23804B886380A8
:1036C0008B7D23B92B88043B2B80BDE8F0812A2316
:1036D00003FB06F606F110033E461E4456F8095F4A
:1036E0007068B168F3686561A061E1612362ECE72D
:1036F000445F0020F8B506460C46154624220021FA
:1037000020460BF01AFE1A49C82303FB06F3CA1819
:10371000CB5A238092F86430A370134653F802CF3B
:103720005F689868DB68C4F803C0C4F80770C4F821
:103730000B00C4F80F3092F864301BB92B88043B9F
:103740002B80F8BDC82303FB06F606F11003084ED4
:103750001E4456F8025F7068B168F368C4F81350ED
:10376000C4F81700C4F81B10C4F81F30E9E700BF05
:10377000E05F00202DE9F0410D461446394BC82288
:1037800002FB04F202F1680119441344596706462A
:1037900010B9354B01221A70C82101FB04F1203108
:1037A000304B194402312846F8F773FF00284CD1FA
:1037B000C82303FB04F378332A4919442846F8F751
:1037C0007BFF002845D1C82303FB04F39033254930
:1037D00019442846F8F79AFF00283ED1214FC82205
:1037E00002FB04F2B818D5F80080D5F804E0D5F84B
:1037F00008C0E968C0F80280C0F806E0C0F80AC056
:10380000C0F80E1002F1100139440023C1F8023053
:10381000C1F80630C1F80A30C1F80E30BE5280F847
:1038200064306309114904F01F04012202FA04F410
:1038300051F82320224341F823200D4951F8232039
:10384000144341F82340BDE8F0817846F3F728FDA2
:10385000AEE77846F3F724FDB5E77846F3F720FDA9
:10386000BCE700BFE05F0020C45F0020D85F0020FD
:10387000DC5F0020F8B505460C46164682B20331DF
:103880002088FFF777FFA2781949C82303FB0513A7
:1038900083F864202AB3242E1BD11549C82303FBC7
:1038A00005F303F110020A44204650F813CF47688D
:1038B0008668C468C2F802C0C2F80670C2F80A601E
:1038C000C2F80E40403319440331F8F7E2FE20B944
:1038D000F8BD7846F3F7E4FCDFE77846F3F7E0FC61
:1038E000F6E7142EF4D07846F3F7DAFCF0E700BFE1
:1038F000E05F0020F8B5CC1FA200224495001249D9
:103900002944076846688568C3684F608E60CD604B
:103910000B61F8F723FF90B963090C4904F01F0409
:10392000012202FA04F451F82320224341F8232013
:10393000074951F82320144341F82340F8BD784645
:10394000F3F7AEFCE8E700BFA8600020185F002096
:103950001C5F002008B50B46C11D89B21846FFF751
:10396000C9FF08BD08B5064B00221A700548F9F7D3
:1039700057FD00B908BD0448F9F7A0FFFAE700BFFA
:103980008E5F0020905F002084330020F8B504464D
:103990000D46F7F7BFFE052C1ED81E4B1E78FEB154
:1039A000E200121B91001C4B0B44998929441A69AF
:1039B00089B21A48F9F72BFE074688B1C4EBC40454
:1039C000A200154B13445B690246011D2846984727
:1039D0003846F9F755FE18E07846F3F761FCDCE766
:1039E000C4EBC404A2000C4B13449A68690905F0A7
:1039F0001F05012303FA05F552F821302B4342F845
:103A000021300748F9F75AFF0026F7F7A3FE3046A2
:103A1000F8BD00BF8E5F0020A0FD0300905F002076
:103A2000B45F002010B50A2201210948F9F7EFFD23
:103A3000002814BF0124002408D007234381012358
:103A400083818380C3800381F9F71AFE204610BD6D
:103A5000905F002070B504460E46F7F75BFE052C1C
:103A600029D8174B1D7875B1C4EBC4039A00154BC8
:103A700013449989314489B21348F9F729FEB0FA01
:103A800080F56D099DB9C4EBC404A2000D4B13442D
:103A90009A68710906F01F06012303FA06F652F828
:103AA0002130334342F821300848F9F707FFF7F790
:103AB00051FE284670BD7846F3F7F2FBD1E700BF10
:103AC0008E5F0020A0FD0300905F0020B45F002007
:103AD0002DE9F84F00264FF0010818E0A4EB421141
:103AE00001238B40013B55F8221019421ED10132AF
:103AF00004F11F035B099A4205D2013B9A42EDD0C3
:103B00004FF0FF33EFE7434693B10136F6B2052E8F
:103B100042D8B8F1000F3FD037462049F3009B1B35
:103B20009A008B189D688C580022E1E70023EBE790
:103B30004FF000090FE049463046FFF78BFF48B3CE
:103B4000012303FA0BFB55F82A3023EA0B0345F84F
:103B50002A3009F101094C45D7D94FEA591A55F8CD
:103B60002A3009F01F0B23FA0BF313F0010FF0D0EA
:103B7000C7EBC7039A00094B13445B6853F82A301C
:103B800023FA0BF313F0010FD5D049463046FFF767
:103B9000FDFED4E78046B8E7BDE8F88FA0FD03003E
:103BA00038B5062828D84409314951F8243000F0A6
:103BB0001F0223FA02F515F0010F1DD02D4D05EB64
:103BC0008005AD78002D4BD12A4D05EB8005ED78B1
:103BD0000DB1002047E0012505FA02F223EA0203B5
:103BE00041F824300024234B23F820400146284686
:103BF000FFF730FF204636E0C31F9BB293BB590945
:103C00001D4A52F8212003F01F0322FA03F313F098
:103C1000010F29D0C11F01EB81039A00174B1344F8
:103C20009B781BBB154B1344DB780BB100201AE0CB
:103C30004C09114801F01F02012303FA02F250F867
:103C4000243023EA020340F8243001EB8102930080
:103C500000240A4AD4520220FFF7FCFE204602E06C
:103C6000002000E0052038BD0520FCE70020FAE731
:103C7000085F0020205F0020185F0020A86000205F
:103C800030B58DB005460C46012905D0022C07D071
:103C9000032C09D00DB030BD7846F3F701FBF5E7F2
:103CA0007846F3F7FDFAF3E72C22002101A80BF088
:103CB00044FB10238DF8043002238DF8083003955F
:103CC000044BDA6805921B69069301A8F4F7A4FE79
:103CD000E0E700BF905F002008B511460020FFF725
:103CE000CFFF08BD08B508461146FFF7C9FF08BD5C
:103CF00070B505460C4616464FF6FF730B80F6F777
:103D000005FB3070022822D0032841D0012841D081
:103D1000002020E021884FF6FF72914208D003EB8B
:103D200083018A001D498A5AAA420DD001330FE04F
:103D30005A091B4951F8222003F01F01CA4012F012
:103D4000010FECD12380F1E72380012003E0002361
:103D5000002BDFD0002070BD124A32F82320AA4287
:103D600013D00133062B17D821884FF6FF729142EA
:103D7000F2D15A090C4951F8222003F01F01CA4020
:103D800012F0010FE8D12380EBE723800120E2E766
:103D90000023E7E70023E5E70020DCE7A860002038
:103DA000185F0020205F0020085F002000293CD021
:103DB00070B582B00E46144605460DF1070201A902
:103DC000FFF796FF1CB99DF80730032B2FD1012C6C
:103DD0001BD068B9BDF804104FF6FF73994228D084
:103DE0002846FFF729FABDF804100120FFF7CEFDA1
:103DF000BDF80430338084B10F4A02EB83039A7814
:103E000001329A70002002B070BD9DF80730032B7C
:103E1000DFD0012BDDD01020F5E7074A02EB83034A
:103E2000DA780132DA700020EDE70E2070471020BA
:103E3000E9E70420E7E700BF205F002070B50646F1
:103E40000D464FF6FF730B8000240CB1002070BDAF
:103E50006309104A52F8233004F01F02D34013F0D4
:103E6000010F06D12A884FF6FF739A420CD12C809D
:103E70000AE004EB840293000748184410223146FC
:103E800004300BF0FBF908B10134DEE72C8001208F
:103E9000DDE700BF185F0020A8600020F0B583B008
:103EA0004FF6FF73ADF80630C0B30746C1B31546F1
:103EB0000C460DF10601FFF7C1FFBDF80630DE1D0F
:103EC000B6B260B94FF6FF7293422BD031463846F6
:103ED000FFF710FDBDF806100220FFF757FD268002
:103EE00075B1BDF80600104A83001C18A1000C46ED
:103EF0001144897822444B1C9370002003B0F0BD1C
:103F0000BDF80600084A83001C18A1000C461144A5
:103F1000C97822444B1CD3700020EFE70E20EDE758
:103F20000E20EBE70420E9E7A860002030B583B05D
:103F300005460C46486820B10DF10601FFF77EFFEB
:103F400018B94FF6FF73ADF806300DF1060128469B
:103F5000FFF748F80246A8B1BDF8063003EB83032B
:103F600099000B4B0B44DB787BB1658002232370F7
:103F7000BDF8061001EB810101FA03F0044B034484
:103F800004336360104603B030BD0022FAE700BF7F
:103F9000A860002000B583B0488003230B70002385
:103FA0004B60A0F57F43FC3B032B17D8DFE803F001
:103FB0000402071A002016E0FCF70CFC13E0694627
:103FC0004FF4C870F7F7B1F820B90198003018BF66
:103FD000012008E07846F3F763F9F6E76946FEF753
:103FE000CDFF00E0012003B05DF804FB70B5F9F7E8
:103FF0007DFC28B9F7F758FC0028F8D020BFF6E779
:10400000344B187800B970BD01213348F9F732FA02
:10401000044600285BD04389072B02D18389012BFA
:1040200003D0FFF79FFC0020EDE7C388012BF8D1F8
:104030000389012BF5D18388012BF2D1002519E0EA
:10404000002B36D0B3F5805F2ED1012000E0032095
:104050006988C0EBC0039A00204B13449E892B88CB
:1040600003F57F533F339B009BB22A1D891BFFF74B
:1040700099F93DB32A4600211748F9F722FA054677
:104080000028F6D08442F4D0428802F47043B3F59D
:10409000005F13D0D4D9B3F5804F11D0B3F5A04F42
:1040A0000AD0B3F5405FD2D07846F3F7F9F8002094
:1040B000CEE7023AD0B2CBE70520C9E70220C7E736
:1040C0000420C5E7064B186800F001009BE70020BC
:1040D00099E700BF8E5F0020905F0020A0FD0300E5
:1040E000105F002008B5F5F791FCA0F5805008BDE1
:1040F00010B586B0164B0393164B0493164B0593DD
:1041000000230293FFF7EEFF009001230193F7F7DE
:1041100001FB69461148F9F78BFB50B90F4B1B782F
:10412000012B0CD0F7F716FB0D4B01221A7006B0CD
:1041300010BDF7F70FFB0B48F9F7C0FBF7E7FFF7E8
:1041400071FC0446F7F706FB002CF4D0ECE700BF47
:10415000E53C0300D93C030069410300905F002067
:104160008E5F00209433002008B5FFF7C1FF08BD23
:1041700070B5002513E02149EB005B1B9A008E18F7
:104180008C581F346409A4002246002170680BF08B
:10419000D4F822460021B0680BF0CFF80135052D88
:1041A000E9D9002206E0164B03EB82030021D97007
:1041B00099700132062AF6D90023A3B10023114ACF
:1041C0001360114A1360114A1360114A1360114AB7
:1041D0001360114A1360114A13805380104A137000
:1041E000FFF7C0FB70BD9900194488000D4A0244D6
:1041F0000021D17091700133DFE700BFA0FD030003
:10420000205F0020105F0020085F0020185F002062
:10421000D85F00203C5F0020705F0020C85F002056
:10422000C45F0020A860002008B50848084B036060
:10423000F6F726FA074B084A9A60084ADA60084BF4
:1042400000221A70FFF754FF08BD00BFCC5F0020AA
:104250001D4D0300B45F002091330300D13A0300E9
:104260008E5F002010B5044680B11C4B1B6813F014
:10427000010F2ED1208863880344013B98422ADC39
:10428000F6F744F8012805D00B2025E07846F3F72F
:1042900007F8EAE720886388184480B2013880B2C2
:1042A000F6F734F8012801D00B2015E022680C4BFA
:1042B0001A600A4A136843F001031360002108469C
:1042C000FFF764FB074A136843F001031360002003
:1042D00002E00F2000E00B2010BD00BF105F0020A7
:1042E000C85F0020145F002010B5044618B1044BCD
:1042F0001B68236010BD7846F2F7D2FFF7E700BFD6
:10430000C85F002008B50122FFF750FD08BD00007E
:10431000062809D843091D4A52F8233000F01F022D
:10432000D34013F0010F11D1C31F9BB283B95909B8
:10433000174A52F8212003F01F0322FA03F313F067
:10434000010F01D0012304E0002302E0012300E07B
:104350000023CBB1062807D80E4B03EB80008378EF
:10436000013383700020704710B407380A4A830075
:104370001C18A1000C461144897822444B1C9370F0
:1043800000205DF8044B704705207047085F00204F
:10439000185F0020205F0020A860002008B50122DF
:1043A000FFF77CFD08BD000038B5062809D8430991
:1043B000184A52F8233000F01F02D34013F0010FC7
:1043C0001BD1C31F9BB20BBB5909134A52F82120C2
:1043D00003F01F0322FA03F313F0010F18D0C41FD8
:1043E0000E4AA3001D19A9000D46114489782A44DC
:1043F0004B1E9370FFF7D4FB38BD094B03EB8003D2
:104400009A78013A9A70FFF7CBFBF5E70520F3E7BE
:104410000520F1E7085F0020185F0020A860002059
:10442000205F002008B50022FFF7C0FC08BD08B5DA
:104430000022FFF733FD08BD062809D843091D4AAD
:1044400052F8233000F01F02D34013F0010F11D1B6
:10445000C31F9BB283B95909174A52F8212003F0B0
:104460001F0322FA03F313F0010F01D0012304E02C
:10447000002302E0012300E00023CBB1062807D887
:104480000E4B03EB8000C3780133C37000207047EC
:1044900010B407380A4A83001C18A1000C461144C6
:1044A000C97822444B1CD37000205DF8044B704740
:1044B00005207047085F0020185F0020205F002063
:1044C000A8600020A9B338B50A46062809D84309D0
:1044D0001B4951F8233000F01F01CB4013F0010FAE
:1044E0001CD1C31F9BB233BB5C09164951F8241081
:1044F00003F01F0321FA03F313F0010F1DD0073857
:10450000114B81000D18AC0025461C5B54802B44D8
:104510000433536002231370002038BD14460B4B44
:1045200033F820005080F5F7F1FE20700020606025
:10453000F3E70E2070470520EFE70520EDE700BF09
:10454000085F0020185F0020A8600020205F002086
:10455000062809D843092A4A52F8233000F01F02DE
:10456000D34013F0010F11D1C31F9BB283B9590976
:10457000244A52F8212003F01F0322FA03F313F018
:10458000010F01D0012304E0002302E0012300E039
:1045900000239BB310B582B004466946FFF792FF33
:1045A00048BB9DF80030032B03D0022B11D00F2005
:1045B00022E0154B03EB8403DB780BB905201BE0ED
:1045C000114A02EB8402013BD3702046FFF7E8FA60
:1045D00012E0E31F03EB830291000C4A0A44D278F5
:1045E0000AB9052008E0094B0B44013ADA7020466D
:1045F000FFF7D6FA00E0002002B010BD052070479A
:10460000085F0020185F0020205F0020A8600020C5
:1046100068B330B583B0054659B30C464088F5F70A
:1046200075FE02280ED0032803D0012801D01020E7
:1046300020E021466888FEF703FD08B1002019E05C
:10464000052017E04FF6FF73ADF80630686850B1EB
:104650000DF10601FFF7F2FB38B1BDF80630073364
:104660002380002006E00E2004E0052002E00E205A
:1046700070470E2003B030BD4FF6FF71002393B199
:1046800000236BB10846704799B2012321E04FF631
:10469000FF72914219D199B217E04FF6FF711AE0FB
:1046A0004FF6FF71EEE710B45A090D4C54F8222072
:1046B00003F01F04E24012F0010FE8D0C82202FB11
:1046C00003F2084CA25A9042DED00133002BEBD00B
:1046D0000023002BE1D008465DF8044B704700BF73
:1046E000D85F0020E05F002018B108B5FEF7A0FEFB
:1046F00008BD4FF6FF70704700B583B00DF106019D
:10470000FEF7FCFC20B1BDF8060003B05DF804FB29
:104710004FF6FF70F9E718B108B5FEF7C1FE08BD06
:104720004FF6FF70704700000A4691B198B94309EF
:104730000B4951F8233000F01F01CB4013F0010F5B
:104740000BD02A2303FB00F0064B1B5A13800020DA
:1047500070470E207047052070470520704700BF46
:104760003C5F0020445F0020012866D8002966D005
:1047700038B50D46044678BB4309344A52F8233015
:1047800000F01F02D34013F0010F5AD0304A2A2301
:1047900003FB00235B88BBB92D4A2A2303FB0423B8
:1047A0005B8859092B4A52F8212003F01F0322FA93
:1047B00003F313F0010F0BD0254B2A2000FB04302C
:1047C00043882B80002038BD7846F2F769FDE3E787
:1047D0007846F2F765FDEFE7441E62091E4B53F879
:1047E000223004F01F02D34013F0010F2BD01B4ADC
:1047F000162303FB04235B88BBB9184A162303FB6B
:1048000004235B885909134A52F8212003F01F033F
:1048100022FA03F313F0010F0BD01048162303FB09
:10482000040463882B800020CDE77846F2F738FD3A
:10483000E3E77846F2F734FDEFE7052070470E20F6
:1048400070470520BFE70520BDE700BF3C5F0020A3
:10485000445F0020D85F0020705F0020785F002058
:10486000002951D038B50C46002A4FD0B0F5805FF2
:104870004ED24FF6FF73138000238BB100232146E5
:10488000144605464BB31088244BC82202FB003067
:10489000102202300AF0F2FC00283BD1032038E05D
:1048A00059091F4D55F8211003F01F05E94011F07B
:1048B000010F0BD0C82101FB03F1184D695A884242
:1048C00001D00133D9E713800123D8E715884FF6CB
:1048D000FF718D42F5D11380F3E712884FF6FF7315
:1048E0009A4219D0FEF746FF21880320FFF74EF8C1
:1048F0002188C82303FB01F388330849194428465B
:10490000F5F7C7FE002004E00E2070470E2000E0FF
:10491000072038BD0F20FCE70420FAE7E05F002005
:10492000D85F0020034690B942090B4850F8222076
:1049300003F01F00C24012F0010F0AD0074AC8203E
:1049400000FB032393F864300B70002070470520B0
:1049500070470520704700BFD85F0020E05F00204F
:10496000002900F083802DE9F8430F4600287FD10D
:104970004509434B53F8253000F01F06F34013F070
:10498000010F78D004463F4AC82303FB002393F865
:1049900064307BB1012B70D1C82000FB04F01030D3
:1049A0001044102202300AF069FC08B9002060E0CF
:1049B00008205EE03349C82303FB00F303F1100233
:1049C0000A4402F10208D7F80090D7F804E0D7F8BB
:1049D00008C0F868C2F80290C8F804E0C8F808C037
:1049E000C8F80C004033194403313846F7F751FE3C
:1049F00080BBC82303FB04F3A0332249194440467B
:104A0000F7F75AFE50BBC82303FB04F3B8331D4924
:104A100019443846F7F77AFE20BB1A48C82303FB2F
:104A200004F3C218012782F8647003F1B0013A461A
:104A30000144C05AF5F7C4F9134B07FA06F653F8C8
:104A400025703E4343F8256021460320FEF79EFF74
:104A500000200EE07846F2F723FCCAE77846F2F72A
:104A60001FFCD0E77846F2F71BFCD6E70E20704714
:104A70000520BDE8F8830520FBE70820F9E700BF23
:104A8000D85F0020E05F0020DC5F002090BB70B5A5
:104A900004464509194B53F8253000F01F06F34032
:104AA00013F0010F28D0164AC82303FB002393F804
:104AB0006430012B01D0082070BD1046C82303FBD1
:104AC00004F3D118022281F8642003F1B0010144FB
:104AD000C05AF5F775F90B4A012303FA06F652F8A6
:104AE0002530334342F8253021460320FEF74EFFA0
:104AF0000020E1E7052070470520DDE7D85F0020B2
:104B0000E05F0020DC5F0020002840F0CC802DE931
:104B1000F04701464409674B53F8243000F01F0565
:104B2000EB4013F0010F00F0C080634AC82303FB81
:104B3000002393F86430002B00F0B980C82000FBFC
:104B400001F0171800F11003134453F8028FD3F843
:104B500004E0D3F808C0DB68C7F80280C7F806E0B5
:104B6000C7F80AC0C7F80E3000F1200313444030E4
:104B70000244D01C02332332D0F800E0D0F804C045
:104B80008768C668C3F800E0C3F804C09F60DE60B1
:104B9000103010339042EFD102781A70464AC82381
:104BA00003FB01F303F17800A0331344024403F143
:104BB0002000D3F800E0D3F804C09F68DE68C2F894
:104BC00000E0C2F804C09760D66010331032834210
:104BD000EFD10F4619685B68116053603648C823EF
:104BE00003FB07F3C218002682F8646003F1880112
:104BF00032460144C05AF5F7E3F811E072092F4B31
:104C000053F8223006F01F01CB4013F0010F06D0FD
:104C10002B482A2303FB06035B88BB4212D00136D4
:104C2000002EEBD0274A012303FA05F552F8243071
:104C30002B4342F8243039460320FEF7A7FE00201C
:104C4000BDE8F0872A2303FB06039B7D002BE6D0FB
:104C500003462A2000FB06F003EB000E103003444D
:104C600053F807AFD3F80490D3F80880D868CEF88B
:104C700004A0CEF80890CEF80C80CEF810001B8A65
:104C8000AEF8143000238EF816300F48012303FAD3
:104C900001F150F822300B4340F822303146042015
:104CA000FEF774FEBBE7052070470520C8E7082023
:104CB000C6E700BFD85F0020E05F00203C5F002017
:104CC000445F0020DC5F0020405F002070B5044698
:104CD0000D469DF81060FEF78FFB4FF6FF7398426C
:104CE00002D03034AC4200D070BD56B10A4AC8235D
:104CF00003FB002393F86430012BF5D1FFF7C6FEC8
:104D0000F2E7054AC82303FB002393F86430002B25
:104D1000EAD0FFF7F9FEE7E7E05F00200378042B15
:104D200000D0704710B582B00446037E42698168A6
:104D30004068647E0094003318BF0123FFF7C6FF6C
:104D400002B010BD40B108B541B1FEF735FA08B167
:104D5000002008BD0920FCE70E2070470E20F8E770
:104D60008AB3F0B583B014467BB31F460E460546A2
:104D7000F5F7CCFA01282AD166BB7309194A52F813
:104D8000233006F01F02D34013F0010F24D00DF1A1
:104D900006012846FEF782F900BBBDF806304FF643
:104DA000FF7293421CD0224631462846FEF782FA13
:104DB000BDF8061001390520FEF7E8FDBDF8063004
:104DC0003B80002004E00E2070470E2000E0102001
:104DD00003B0F0BD0520FBE70520F9E70F20F7E75A
:104DE0000420F5E7D85F0020A2B3F8B517469BB3BF
:104DF000A1BB4C091E4A52F8244001F01F02D440C6
:104E000014F0010F2CD0B0F5805F2BD21D460C465C
:104E100006461946FEF772F960B12888154B2A221A
:104E200002FB00301022394606300AF027FAD8B9C2
:104E3000032014E02B884FF6FF72934216D03A46B7
:104E400021463046FEF78EFB29880420FEF79EFDA2
:104E5000002004E00E2070470E2000E00520F8BD81
:104E60000520FCE70720FAE70F20F8E70420F6E723
:104E7000D85F0020445F0020002965D0F8B50F46B8
:104E8000002863D14409344B53F8243000F01F0547
:104E9000EB4013F0010F5BD030492A2303FB0013D2
:104EA0005B882F49C82606FB031393F86430012B57
:104EB00050D10646294A2A2303FB00239B7D73B168
:104EC0002A2303FB00F310331046184410223946FE
:104ED00009300AF0D3F9002839D0082037E01F49FB
:104EE0002A2303FB00F3CA180120907510331944DC
:104EF000D7F800E0D7F804C0B868FA68C1F809E04C
:104F0000C1F80DC0C1F81100C1F8152008313846AC
:104F1000F7F7B4FBA0B9114A2A2303FB06231A7939
:104F2000DA75104A012303FA05F552F824302B43B1
:104F300042F8243031460420FEF728FD002006E028
:104F40007846F2F7ADF9E6E70E2070470520F8BD88
:104F50000520FCE70820FAE73C5F0020445F0020C2
:104F6000E05F0020405F0020C0B938B5014640092D
:104F70000C4A52F8203001F01F0423FA04F515F012
:104F8000010F0DD0012505FA04F423EA040342F8C9
:104F900020300420FEF75EFD002038BD052070475C
:104FA0000520FAE73C5F0020002879D12DE9F04187
:104FB000804645093E4C54F8253000F01F06F3406A
:104FC00013F0010F6ED0236813B90123002714E0FA
:104FD0005A421340374A02FB03F3DB0E364AD35CD6
:104FE000F4E750420240334800FB02F2D20E32484E
:104FF000825C02EB431300E00123012B18D0013740
:10500000581CF9D143092A4A52F8232000F01F0006
:105010004FF0010C0CFA00F040420240002AE0D1AF
:10502000013303D1224A52F82320F7E70123E4E7B2
:10503000012F3AD00027BFB1C82303FB08F31F4A52
:10504000D35A13B91E4B00221A70012303FA06F635
:1050500054F8253023EA060344F82530414603205E
:10506000FEF7F8FC00201EE07B09164A52F82330B8
:1050700007F01F02D34013F0010F06D0124A2A2373
:1050800003FB07235B88434501D00137D3E7B8B260
:10509000FFF76AFF0028F8D07846F2F701F9F4E745
:1050A000052070470520BDE8F0810F20FBE700BF19
:1050B000D85F002031B57C0748FE0300E05F002088
:1050C000C45F00203C5F0020445F0020A9B110B500
:1050D0000C46A2B1A8B943090C4951F8233000F09D
:1050E0001F01CB4013F0010F0DD02146FEF734F81D
:1050F00008B1002008E0092006E00E2070470E20CD
:1051000002E0052000E0052010BD00BFD85F0020B0
:10511000012974D8002A74D030B461BB3D4C61BB06
:105120000B465D0954F8254003F01F0324FA03F3EE
:1051300013F0010F67D04FF6FF7398421FD000287D
:1051400063D14309344C54F8233000F01F04E3408A
:1051500013F0010F5BD081BB304CC82303FB00432D
:1051600093F86430022B18D02D4C2A2303FB014105
:105170000431516028E02B4CD1E74B1ED1E729B90F
:1051800027482A2303FB01035888D8E74B1E2648EB
:10519000162404FB03035888D1E7214C2A2303FB80
:1051A00001439B7D002BDFD02A2303FB01F110314B
:1051B00023460B440733536006E001391A4B16248B
:1051C00004FB0131043151601449C82303FB00136F
:1051D00093F86430022B0AD0C82303FB00F0203080
:1051E0000E4B034402331360002030BC7047C823C9
:1051F00003FB00F040300B4603440333F3E7052084
:1052000070470E2070470520EFE70820EDE70820E3
:10521000EBE700BF3C5F0020D85F0020E05F00208C
:10522000445F0020705F0020785F00200A4699B13B
:10523000A0B943090B4951F8233000F01F01CB40BE
:1052400013F0010F0CD0C82303FB00F07030064BA5
:1052500018441060002070470E20704705207047EA
:1052600005207047D85F0020E05F002010B50C4695
:10527000FFF702FAACB1B0B943090D4A52F8233036
:1052800000F01F02D34013F0010F0ED0C82303FB20
:1052900000F000F12003074818440230206000208D
:1052A00010BD0E20FCE70520FAE70520F8E700BF57
:1052B000D85F0020E05F002070B5064615460C461A
:1052C00059B175B1206880B1FEF7B2F80130002302
:1052D00023602B6006F07F011BE07846F1F7E0FFCA
:1052E000EFE77846F1F7DCFFECE70020EFE73BB1B2
:1052F0002A4AC82303FB002393F843308B4239D05A
:10530000264AC82303FB002393F822308B423BD06C
:105310000130002840D14309214A52F8233000F0DF
:105320001F02D34013F0010FF2D01C4AC82303FB25
:10533000002393F86430002BD9D01646C82202FB14
:10534000006292F822208A42D1D1C82202FB006278
:1053500092F843208A42CAD13346C82202FB00F0A9
:1053600000F1200232440232226040300344033311
:105370002B6011E0C82303FB00F303F14002074B4D
:1053800013440333236007E0C82303FB00F02030FD
:10539000134603440233236070BD00BFE05F00206A
:1053A000D85F002070B504460E46154662B17CB148
:1053B0002046FEF73DF84FF6FF7398420CD02A4680
:1053C0003146FEF79BF870BD7846F1F769FFEEE7CE
:1053D0007846F1F765FFEBE700232B60F3E738B57C
:1053E00005460C4621B12846FDF70EFF206038BD6A
:1053F0007846F1F755FFF6E7F8B5054617460E462D
:1054000039B157B1306800286FD0FDF7F5FF441C63
:105410000DE07846F1F744FFF3E77846F1F740FFF7
:10542000F0E7012300E00023002B42D10134002CDF
:105430005DD163092F4A52F8233004F01F02D34094
:1054400013F0010FF2D02C4AC82303FB042393F876
:1054500064307BB9002DE4D0C82303FB04F3883308
:10546000082225491944284609F008FF0028DAD106
:105470000123D9E7BDB1C82303FB04F38833082215
:105480001D491944284609F0F9FE70B1C82303FBF1
:1054900004F3B033082218491944284609F0EEFEF7
:1054A00028B90123C0E70123BEE70123BCE700239D
:1054B000BAE7124B1B784BB1C82303FB04F30E4A27
:1054C000D35A0BB1002102E0012100E001210A4A78
:1054D000C82303FB04F4131983F8701070341444C8
:1054E000346093F864303B7003E000249FE70023AE
:1054F0003360F8BDD85F0020E05F0020C45F00206B
:1055000038B504460D46F4F701FF02280FD00328F2
:1055100008D0012801D0002003E029462046FDF7ED
:105520000BFD38BD29462046FEF734FDF9E7294634
:105530002046FEF7FBFCF4E700B583B00378022BAE
:105540000ED0032B03D0012B01D0002304E06946C9
:105550004088FFF7D5FF0346184603B05DF804FB0B
:1055600069464068FEF76AFC03460028F4D0BDF89F
:10557000003003EB83039A00034B1344DB780033C2
:1055800018BF0123E8E700BFA860002038B50C462B
:10559000054630B129B1054B1A882A805B882380E3
:1055A00038BD7846F1F77CFEF5E700BFC85F002004
:1055B000034643B1A3F1080013F8082C8A4203D034
:1055C00012B11B68F5E70020704750B1426852B134
:1055D0004378073BDBB2F72B01D900207047072047
:1055E00070470E2070470E20704710B5007848B9FC
:1055F000002404E0E0B200F099F80134A4B2FF2CDA
:10560000F8D910BD00F092F8FBE70000F8B50546A8
:10561000FFF7DBFF044608B12046F8BD094E3768A6
:105620002846FFF7E2FF05F108013046F7F728F9B1
:10563000002FF1D1002000F089F8012000F066F879
:10564000EAE700BFBC6000202DE9F8430646884623
:1056500091461F460C4616E05B6821783A460139B0
:10566000A01C984765B161782846FFF7A1FF034663
:1056700030B185684278B242EED0FF2AECD0F1E733
:10568000237801331C4408EB0903A34202D9024BDF
:105690001D68E7E7BDE8F883BC600020F0B41A4B52
:1056A0001E7BB6FA86F56D090021437D063BDBB211
:1056B0008B421ADD4218577F4A1C0244527F4FEA40
:1056C000521C114C04EB8C04246902F01F0224FAD2
:1056D00002F212F0010F02D101373944E5E75B1AFB
:1056E0009F420ADA351C18BF01251DB1064A536BCB
:1056F000013353632846F0BC7047034A136B0133F0
:1057000013630125F6E700BFC060002008B518B993
:10571000044800F021FE08BD0248034B036000F07E
:1057200005FEF8E7C06000209D5603004109064AC7
:1057300000F01F00012303FA00F052F82130034368
:1057400042F82130704700BFD060002010B50446F9
:10575000012802D97846F1F7A3FD014B1C7310BD57
:10576000C060002010B5044648B1E36F5BB1E36F41
:10577000D4F89820D4F894102046984710BD784665
:10578000F1F78EFDF1E77846F1F78AFDEFE710B506
:105790000446037813F0FE0301D0022B05D12378D1
:1057A00003F0FE03022B04D010BD7846F1F778FD1C
:1057B000F5E7A37963F03F03A371F5E710B582B075
:1057C000044628E0002002B010BD7846F1F768FDDD
:1057D00026E004F15C00F3F70EFB08B1012324E09E
:1057E000002322E0012300E0012333B3616831B1DB
:1057F000043904F15C00F3F715FB0023636001A991
:1058000004F15C00F3F7C6FA0028DBD1019B1A1DF6
:1058100062600C3363626368002BE7D0002BD4D046
:1058200063681B79FF2BD4D0002362681279002BA8
:10583000DAD1002AD6D00023D7E70120C3E7000041
:1058400070B5064643682BB106F174052B79DBB1C0
:10585000002405E07846F1F723FDF5E70134E4B2D2
:10586000EB789C4210D21348F5F7F0FBEA78B0FBD6
:10587000F2F302FB1300C3B2A342EFD02B5DC0B220
:105880002A5C2A552B54E9E77468237953B12379AC
:10589000FF2B01D0013B237106F1080000F00AFD47
:1058A00020B970BD7846F1F7FBFCF0E77846F1F7D8
:1058B000F7FCF6E7F86000200B78002B36D070B5C7
:1058C0000C4691F8403053B9CB6F33B101F18000F1
:1058D000F5F7E0FFE0B1012300E00023D3B104F1CC
:1058E0004405266F94F84430DBB2062B02D078468C
:1058F000F1F7D6FC0F48F5F7A9FB0F4BA3FB0023EC
:105900005B0B42F2107202FB13033344EB6070BD79
:105910000023E3E72046FFF751FF054610B9002DAD
:10592000F5D0DCE72046FFF78BFFF8E700230B6597
:10593000704700BFF86000205917B7D110B5044672
:1059400050F8202C1379013BDBB2FD2B08D9836D75
:1059500033B11368036741675C30F5F779FF20B90D
:1059600054F8201C0B7923B110BD7846F1F798FC50
:10597000F6E744F8203C043904F13800F3F752FA12
:10598000F2E7000008B50248F5F79AFB08BD00BF32
:10599000F86000200378E3B970B504460123037072
:1059A000436883B104F14406256F0A48F5F74EFBBE
:1059B000B0FBF5F405FB1404F5F70AFA211830469C
:1059C000F5F76AF970BD5C30F3F705FA0028E9D104
:1059D000F8E77047F860002030B583B00C46054604
:1059E00078B11F2C11D804F1110292B201A905F16E
:1059F0005C00F3F76FF960B1042826D1002003B0F2
:105A000030BD7846F1F74CFCEBE77846F1F748FCFF
:105A1000E9E7019B181DE4B206345C731A7B02218E
:105A200061F303021A7395F86820C2F34002197BF0
:105A300062F38611197355F8692FC3F80F20AA88ED
:105A4000A3F8132000225A60D9E77846F1F728FC22
:105A50000020D4E770B505460C4611B308B323798E
:105A60001BB3237A03F0CF036FF3C7132372002312
:105A7000A37234F8042C211F05F15C00F3F759F9E7
:105A80002B78D3B195F84430ABB195F84430DBB204
:105A9000042B13D095F84430DBB2052B09D0012339
:105AA0000AE07846F1F7FCFBD9E77846F1F7F8FB16
:105AB000D7E7002300E0002313B170BD0023FBE70C
:105AC00005F144062D6F0748F5F7C0FAB0FBF5F471
:105AD00005FB1404F5F77CF921183046F5F7DCF8DE
:105AE000EBE700BFF860002038B504460D4631B141
:105AF00028B1291F04F15C00F3F794F938BD78460A
:105B0000F1F7CEFBF5E7000038B50D460446C0B10D
:105B1000132D1AD9B5F5205F1BD84FF47A7000FB0E
:105B200005F5256794F84430CBB194F84430DBB2E6
:105B3000042B19D094F84430DBB2052B0DD001238F
:105B40000EE07846F1F7ACFBE2E77846F1F7A8FB08
:105B5000E0E77846F1F7A4FBDFE7002300E000234D
:105B60000BB1237813B938BD0023F9E74434074853
:105B7000F5F76CFAB0FBF5F305FB1305F5F728F91B
:105B800029182046F5F788F8EDE700BFF8600020F7
:105B900038B50D46044610B184F8285038BD784613
:105BA000F1F77EFBF8E710B504465C30F3F769F8CF
:105BB000EFF3108272B663680BB10021197102B95C
:105BC00062B610BD10B504464FF08053D3F8A03034
:105BD00013F0010304D093B97846F1F761FB03E0B9
:105BE00003786FF347030370084B1868C4F801008B
:105BF0009B88A4F805302046FFF7C9FD10BD037847
:105C0000012262F347030370EEE700BFA400001017
:105C1000F8B50D4617461E46044688B182B10A2ED5
:105C200012D9B2B2394604F15C00F2F7D3FF04F1A5
:105C30006800FFF7C7FF44F62063236700230EE0E8
:105C40007846F1F72DFBEAE77846F1F729FBE8E71C
:105C5000154AD15CE21882F874100133DBB2022BD2
:105C6000F6D984F87730002284F878200F49216330
:105C700025216185032184F82C1084F8282004F163
:105C80007401A16384F83C30094B63636262E56789
:105C9000084BE364646522702DB12246064904F185
:105CA0008000F5F7BBFDF8BD68FE0300D6BE898E07
:105CB0003D590300B958030065570300084B012202
:105CC0005A60DA604FF0FF32C3F808230022C3F8AD
:105CD0000022044B4FF48062C3F88021704700BF5C
:105CE00000A0004000E100E0044B4FF0FF32C3F899
:105CF0000823034B0222C3F88021704700100040A4
:105D000000E100E008B5054B1B7803B908BD00F0C1
:105D100029FE024B00221A70F8E700BF196100202B
:105D200010B5FFF7CBFF1A4B0022C3F84021012129
:105D3000C3F840150420C3F81005C3F80425C3F8C0
:105D40000825144A1448C2F86005A0F503503838F5
:105D5000C2F864054FF48060C2F8040519600C4B6A
:105D6000D3F84031002BFAD0094C0023C4F840315D
:105D7000084B4FF48062C3F80825F5F7EBFB074B9F
:105D8000D3F848351844D4F84035C01A10BD00BFC8
:105D900000A0004000F0014040A100400080004011
:105DA00008B5074B1B7803B108BDFFF79DFF044BF7
:105DB00001221A70FFF7B4FF00F0BEFDF4E700BF48
:105DC0001961002038B5F5F7AFFB00B138BD1248B6
:105DD000F4F7B0FC054668B10468F5F7C1FB1CB1E7
:105DE000E3686433834207D3B0F5FA7FEED9FFF757
:105DF000D7FFEBE70024F0E7FFF784FF0648F4F74E
:105E000084FC854202D07846F1F74AFA00236361A8
:105E1000204600F025F8D9E70C61002008B5F4F71A
:105E2000D7FF0C4B1B68C01A00280BDA0020F5F7CF
:105E3000E7FB094B00221A60084B1B7833B9FFF7C8
:105E4000C1FF08BD7846F1F72BFAEFE7F5F7C4FB81
:105E5000F7E700BF146100201C6100201A610020D8
:105E600070B505460120F5F7CBFB0D4C2560FFF71B
:105E70003BFFFFF755FF2368DA68024409490A60CF
:105E8000094C00262670094D01222A701A681969EA
:105E900090472E70237803B970BDFFF7BFFFFBE773
:105EA0001C6100201461002008610020186100209E
:105EB00010B5124B1B68B3B19B686BB1104C01233A
:105EC00023700E4B1B689A68186990470023237053
:105ED0000C4B1B7823B910BD7846F1F7E1F9EDE7DB
:105EE000FFF79CFFF7E7084B1B7813B100F058FD54
:105EF000F1E77846F1F7D4F9F8E700BF1C6100201C
:105F000018610020086100201961002008B50948C7
:105F1000F4F7D4FB0023084A1360084A1370084AB8
:105F200001211170074A1370074A1370074A82F85B
:105F30000A3308BD0C6100201C610020196100209B
:105F40001A610020186100200861002000E100E0D3
:105F5000064B1B783BB110B50024044B1C70F5F7C1
:105F600029FB204610BD0820704700BF1A610020A1
:105F700008B5064B1B7833B9044B01221A70F5F7AC
:105F800019FB002008BD0820FCE700BF1A610020B3
:105F900010B50446C0B12368D3B1E368E3B1E26849
:105FA000154B9A421CD86369A34221D0646104F165
:105FB00014011248F4F78DFB114B1B78D3B9114B28
:105FC0001B688BB1002016E07846F1F769F9E2E72B
:105FD0007846F1F765F9E0E77846F1F761F9DEE731
:105FE0007846F1F75DF9DEE7F5F7E4FA002002E024
:105FF000082000E0002010BDA08601000C610020F8
:106000001A6100201C61002008B50F4B1B6863B1AA
:10601000F5F7CAFA68B10D4B1B7873B90C4B1B78B6
:106020007BB10A4B01221A7008BD7846F1F738F9A6
:10603000EEE77846F1F734F9EDE77846F1F730F915
:10604000ECE7FFF7EBFEEFE71C61002008610020A2
:106050001861002010B5F5F7A7FA90B1134B1B6833
:10606000D3B15B688BB1124C012323700F4B1B68BB
:106070005A6818699047002323700E4B1B7843B968
:1060800010BD7846F1F70CF9E8E77846F1F708F922
:10609000E9E7FFF7C3FEF3E7074B1B7813B100F006
:1060A0006BFCEDE77846F1F7FBF8F8E71C610020A0
:1060B00018610020086100201961002008B5F5F77B
:1060C00073FA18B1054B1B6823B108BD7846F1F788
:1060D000E7F8F7E7FFF776FEF7E700BF1C6100205F
:1060E00008B5F5F761FA70B1094B1B6813B1784632
:1060F000F1F7D6F8074B4FF480621A6002221A605B
:10610000FFF760FE08BD7846F1F7CAF8ECE700BF7C
:106110001C61002000E100E008B5F5F745FA88B100
:106120000A4B1B6813B17846F1F7BAF8FFF7EAFD9E
:10613000FFF7C4FDFFF7D8FD054B4FF48062C3F8AD
:10614000802008BD7846F1F7ABF8E9E71C61002034
:1061500000E100E0064B074AC3F8602502F50F4254
:106160003C32C3F864254FF48062C3F804257047BD
:1061700000F001400411004070B50546254BD3F8EE
:106180001031CBB1234B0022C3F81021224C2378CD
:106190000133237000F0F2FD95F8342023789A4201
:1061A0000ED39A422AD92A6BD05C00F01FF9194B02
:1061B000D3F810314BBB70BD7846F1F771F8E1E7C9
:1061C000164BD3F84065164B1B681E44F4F700FECF
:1061D0000446EB6A314605F11C009847F4F7F8FDD8
:1061E000001B502802D47846F1F75AF800F000FE60
:1061F000FFF70AFF002385F83830DCE7054B032260
:10620000C3F8002200F0CAFDD1E77846F1F748F85C
:10621000D1E700BF001000402461002000A0004032
:106220002061002038B505460C46FFF793FF00F0CB
:10623000BDF804F1200000F0EDF80021A06A00F0A4
:1062400039F9236B187800F0D1F80121154B19703A
:10625000154B1D60E269154BC3F804250022C3F8F5
:1062600010211022C3F80423114A51641960D2F896
:106270004405084400F038FD94F83430012B0AD965
:106280000A4B0722C3F80022226B064B1B78D05C16
:1062900000F0ACF838BD054B0322C3F8002200F033
:1062A0007DFDF7E724610020206100200010004000
:1062B00000A0004010B50446C36A1BB394F8383000
:1062C0005BBB174B2360174B6360E36994F8341092
:1062D00094F824205B780C33042A17D01248825C8F
:1062E00003FB02F32E3303FB01F39833E3602461D5
:1062F000012384F838302046FFF74AFE034638B9B8
:10630000184610BD7846F0F7CBFFD7E70133E5E735
:106310007846F0F7C5FF0023F2E71123F0E700BF4E
:1063200025620300796103006CFE030010B504468A
:1063300038B123684BB104F108010648F6F7A0FA1A
:1063400010BD7846F0F7ACFFF3E77846F0F7A8FF0A
:10635000F1E700BF2C61002010B5044628B104F11C
:1063600008010448F6F7B7FA10BD7846F0F798FF31
:10637000F5E700BF2C61002038B50546094B1C68C5
:106380004CB154F8083C54F8041C2846984703467E
:1063900030B92468F4E7044A13680133136000231A
:1063A000184638BD2C610020286100200D4B0022CA
:1063B000C3F8FC2F0122C3F8FC2F40F25B62C3F844
:1063C000382540F20312C3F83425074AC3F83C25A8
:1063D0009622C3F84425D3F8502642F00102C3F8B0
:1063E00050267047001000405555550010B5044622
:1063F000272807D8054B1A5D054BC3F80825C3F8B5
:10640000544510BD7846F0F74BFFF3E774FE0300E8
:106410000010004010B5044688B32379052B32D80C
:106420006388002B33D063880233B3F5817F32D881
:1064300023781F4AC2F80C352379C2F81035A378A7
:1064400043F0007343F44033C2F818356388252BBA
:1064500025D90823C3F10802120402F47022134361
:1064600043F48073124AC2F81435D2F8143543F459
:106470008013C2F814352379042B12D010BD78464E
:10648000F0F70EFFC9E77846F0F70AFFC8E778464D
:10649000F0F706FFC7E77846F0F702FFC8E70623E4
:1064A000D8E7D2F8143543F08073C2F81435E5E725
:1064B0000010004038B504460D46124BD3F818358D
:1064C000C3F30243032B06D14DB1012D0FD0784603
:1064D000F0F7E6FE0AE07846F0F7E2FEF4E7220E77
:1064E000084BC3F824252402C3F81C4538BD230CEF
:1064F00003F47F43034AC2F824352402C2F820453E
:10650000F4E700BF00100040074B00221A71EFF3C0
:10651000108272B65B781BB1044B0221C3F80011E4
:1065200002B962B6704700BF3061002000E100E0B0
:106530000D4A53790133DBB2537192F82F20934205
:1065400002D3094B00225A71074B02221A71EFF352
:10655000108272B65B781BB1044B0221C3F80011A4
:1065600002B962B6704700BF3061002000E100E070
:1065700030B482B0114B1B68ADF804301B0C8DF8A1
:106580000630002203E000239BB10132D2B28A42DE
:106590000ED20023022BF6D8855C02AC1C4414F802
:1065A000044CA54202D00133DBB2F3E70123EBE751
:1065B0000123184602B030BC704700BF9CFE0300A8
:1065C00010B5FFF7F3FE1C48FFF724FF00241B4B18
:1065D000C3F8304500E00134072C13D804F10A0356
:1065E000174A02EB830398680028F4D02146FFF78E
:1065F00061FF1249D1F830350122A2401343C1F89E
:106600003035E8E70D4B0822C3F804231122C3F804
:1066100000220022C3F8042103F5F033094AC3F82D
:10662000602502F5DE424432C3F864254FF48062EF
:10663000C3F8042510BD00BF4C61002000100040CD
:10664000306100200411004008B5114B9B6813B164
:106650007846F0F725FE0E483C2200F10801843010
:10666000F2F738FB031E0CBF0120002009D00849B7
:106670008A6901328A61003318BF0123044A93708A
:1066800008BD034A926818320249C1F80425F2E7AE
:10669000306100200010004010B51B4BD3F850357E
:1066A0007BB91A4C6379234493F82C00FFF79EFEC4
:1066B000E37853B9FFF7C8FF60B9144B01221A7190
:1066C00010BD7846F0F7ECFDEBE7FFF779FF00220D
:1066D000E270EFE70E4C012161640B4B5960D4F876
:1066E0004405084400F024FB00F058FB0023C4F8E4
:1066F0004431084B4FF48062C3F880214FF40033DB
:10670000C4F80433D9E700BF001000403061002016
:1067100000A0004000E100E008B5064B1B791BB16A
:10672000022B02D8FFF7B8FF08BD7846F0F7B8FD96
:10673000FAE700BF3061002010B50C4B01221A614E
:106740000022C3F80C210A4B996831B11C4603F1B1
:106750008400F2F767FB0023A360044BD3F85035A5
:10676000002BFAD100F044FB10BD00BF0010004028
:106770003061002008B50D4B1B79012B07D073B198
:10678000022B0FD1FFF7D8FFFFF786FF08BDFFF7F9
:106790005BFF0028FAD0064B01229A60F6E7FFF76C
:1067A000CBFFF3E77846F0F77BFDEFE730610020A1
:1067B0000010004008B5094B1B79012B06D033B1FE
:1067C000022B07D1FFF7B8FFFFF766FF08BDFFF701
:1067D000B3FFFBE77846F0F763FDF7E73061002091
:1067E00008B5114B1B78012B05D0022B06D078463B
:1067F000F0F756FD01E0FFF79FFF08BD0B4BD3F804
:106800005035032B0CD8DFE803F002080508FFF72A
:1068100083FFF2E7FFF7AEFFEFE7FFF7CBFFECE711
:106820007846F0F73DFDE8E73061002000100040B9
:1068300070B52F4B9C682F4BD3F8003463B92C4AAA
:106840001369013313612A4881688430F2F7EAFA48
:10685000274B00229A6070BD251D627E244BDB8B86
:106860009A4204D9224A536901335361EBE7214A22
:10687000D2F848355B426373D2F808341C4E0A33B1
:1068800006EB83039B68A360D2F8543503F03F0303
:106890002373F4F75FFE184BD3F848351844606053
:1068A000234653F81B2FC4F80F209B88A4F81330FD
:1068B000237EC3F38011A27B61F34702A273C3F36B
:1068C00003036375F3680133F360D6F890320BB1BC
:1068D00028469847627E064C1732A16804F184006E
:1068E000F2F727FAD4F88000F4F776FFB0E700BF9C
:1068F00030610020001000400080004010B5F4F727
:1069000067FA0446094B9A6A596A8A4208D00144D8
:106910000748F4F7C1F921460648F4F7BDF910BD60
:1069200003F16800F4F788F9F5E700BF3061002053
:10693000986100208061002010B5094C012363702C
:106940000023E370C4F89402FFF73AFE2378022B89
:1069500000D010BD2379002BFBD0FFF79DFEF8E798
:106960003061002008B5034B00225A70FFF7E4FEA7
:1069700008BD00BF3061002008B5084BD3F80C31CA
:1069800013B9FFF72DFF08BD044B0022C3F80C21FB
:10699000D3F80C31FFF74CFFF3E700BF00100040C5
:1069A00008B50A4BD3F8443163B1084B4FF40032B9
:1069B000C3F808230022C3F84421D3F8443100F07F
:1069C000DDF908BD7846F0F76BFCEEE700A000406B
:1069D00008B5094B1B7823B1074B1B78012B04D05A
:1069E00008BD7846F0F75CFCF6E7FFF787FF024B3F
:1069F00002221A70F4E700BF3061002010B5124B7C
:106A00001B7823B1104B1B78022B04D010BD7846A5
:106A1000F0F746FCF6E70C4C04F16800F4F70CF9CB
:106A200004F15000F4F708F901232370EFF3108309
:106A300072B662781AB1054A0221C2F80011002B21
:106A4000E4D162B6E2E700BF3061002000E100E07F
:106A500038B5054698B10C4C291F04F18400F2F7B3
:106A6000E1F9A37853B1EFF3108372B662781AB1EB
:106A7000064A0221C2F8001103B962B638BD784651
:106A8000F0F70EFCE7E700BF3061002000E100E016
:106A900000B583B001A90A48F2F77CF960B9019802
:106AA0000430FFF769FC20B101980430FFF7D0FFF4
:106AB000F0E70198043000E0002003B05DF804FB2B
:106AC000B461002008B50248F2F785F908BD00BF9F
:106AD000B4610020024B83F820000122DA70704775
:106AE0003061002038B504460D4688420FD30F4B65
:106AF0009C4210D840F6B7339D4210D90C4B9C6293
:106B00005D625C67DC651B78022B0CD038BD784673
:106B1000F0F7C6FBEBE77846F0F7C2FBEAE778460A
:106B2000F0F7BEFBEAE7FFF7E9FEEFE700007102CE
:106B30003061002070B506460C464B1EDBB2022BBE
:106B400010D821463046FFF713FD78B1094D224693
:106B5000314605F12C0008F0C7FB00236B7185F866
:106B60002F4070BD7846F0F79BFBEAE77846F0F7D8
:106B700097FBEBE730610020F8B507460E464B1E49
:106B8000DBB2072B0FD80A4C04F13005202200217C
:106B9000284608F0D2FBB2003946284608F0A4FB8C
:106BA0000123E370F8BD7846F0F77AFBEBE700BF0E
:106BB0003061002000B583B00D4B1B68ADF8043088
:106BC0001B0C8DF80630032101A8FFF7B3FF02A8C4
:106BD000084B40F8083D0121FFF7CEFF0320FFF7E7
:106BE00079FF05480146FFF77DFF03B05DF804FB20
:106BF0009CFE0300D6BE898E80841E0038B50546F3
:106C0000104C4FF426720021204608F096FB4FF4FA
:106C1000007204F1900104F18400F1F7DBFFFFF74B
:106C2000C9FF002323772523E383074B2367074B03
:106C3000A3650123237023712846F4F7ADFDC4F842
:106C4000800038BD30610020096503003165030014
:106C5000037813F0020F0BD04FF003130278920861
:106C600043EA022301F5A271024A42F8213070473B
:106C7000014BF3E7006000400300130010B4002351
:106C80000B600B4B9C780B4804F1A20240F83210C9
:106C90001B799B0003F1804303F5C04300EBC20264
:106CA00053600123A340C0F804355DF8044B7047DE
:106CB000C863002000F00140037813F0010F0AD0F0
:106CC00013F0020F08D103789A08012393404FF084
:106CD000A042C2F8083570479A08012393404FF04C
:106CE000A042C2F80C3570470E4B5B7923B10D4BB7
:106CF0001B7813F0010F00D1704770B50C460546A4
:106D0000084EB1783046FFF7A3FF074901EB840135
:106D10003046FFF7B3FF163504F5A871034B43F86F
:106D2000215070BDC863002040A1004000A0004079
:106D30000F4B5B7923B10E4B5B7813F0010F00D141
:106D4000704770B50C460546094B5E1C9978304675
:106D5000FFF77EFF074901EB84013046FFF78EFF06
:106D6000163504F5A871044B43F8215070BD00BFDF
:106D7000C863002040A1004000A00040054B5B79A3
:106D800033B1044B9A7801239340034AC2F8083583
:106D9000704700BFC863002000F00140104B5B79D2
:106DA000E3B110B40F4B0022C3F810210C4BD8787C
:106DB0000D4900F1A2020D4C41F832401B799B00B5
:106DC00003F1804303F5C04301EBC202536001238A
:106DD0008340C1F804355DF8044B7047704700BF2D
:106DE000C86300200010004000F001401011004076
:106DF0000F4B5B7903B9704710B50D4CA378012296
:106E000002FA03F3E1788A4013430A4AC2F80835CC
:106E1000237903F5A273A2F5C832002142F82310AA
:106E20002046FFF749FF601CFFF746FF10BD00BF7B
:106E3000C863002000F001400369C268934202D990
:106E40009B1A581E70478068801A0344581E70476A
:106E50002DE9F041054688461646C7688468E41B5C
:106E600094420ED840682246384408F03DFA361B5A
:106E7000324608EB0401686808F036FAEE60BDE8B7
:106E8000F0814068384408F02FFA3E44EE60F6E79F
:106E90002DE9F843064688461746C5684FF00009B5
:106EA0001AE0B268641B1444621EB3685C1B94420F
:106EB00028BF1446BC4228BF3C4670682246414663
:106EC000284408F011FAA144A0443F1B2544B368AC
:106ED000AB4207D0F5603FB13469A542E1D2641BF3
:106EE000621EE2E70025F5E74846BDE8F8830000AA
:106EF000114B02221A615A6110499961104ADA61F4
:106F00004FF480621A6200229A625A62DA629964CD
:106F10000C49D964802119659A655A65DA650A4A6F
:106F20001068C3F80700094A92E8030018609980C6
:106F300020229A71704700BFD0630020A0FE03009A
:106F4000C864002048640020ACFE0300B0FE0300CB
:106F50002DE9F047054688469146234B1B78C3B17F
:106F60006A002A44D100204B0B449F6D5C6DA74200
:106F700012D80026E41B4C4528BF4C4634BB2EB12A
:106F800005EB4500C200184B13449F653046BDE831
:106F9000F087FFF7ADFFE3E7134B03EB010ADAF8E5
:106FA0005060F61B4E4528BF4E46DAF84C1032466C
:106FB0003944404608F098F9B044A9EB0609374433
:106FC000DAF85030BB42D5D10027D3E705EB4503B3
:106FD000DA00054B1344D96C22463944404608F088
:106FE00083F926442744CAE7D063002010B50B4636
:106FF000EFF311844FF0800181F311881946FFF7F8
:10700000A7FF84F3118810BDF8B50F461646194A3C
:10701000431C03EB4303DD00154400EB4000C300B9
:107020001A44D46A012C10D01CB1022C1BD00024AD
:1070300017E02846FFF700FF864212D8324639464D
:107040002846FFF705FF34460BE02846FFF7F4FE1D
:107050003446864228BF0446224639462846FFF772
:10706000F7FE2046F8BD32462846FFF711FF0446DA
:10707000F7E700BFD0630020F8B505460E46174677
:10708000094B1B786BB1EFF311844FF0800181F352
:1070900011883A4631462846FFF7B6FF84F3118837
:1070A000F8BDFFF725FFEEE7D063002000B583B001
:1070B00001220DF107010020FFF798FF012804D1FC
:1070C0009DF8070003B05DF804FB4FF0FF30F9E7CF
:1070D00010B58268531C4468A34205D80468A154C3
:1070E0008360C3680133C360826843689A4200D0FA
:1070F00010BD044601680069FFF7BEFFA36898420F
:1071000003D04FF0FF33E360F2E70023A360EFE723
:107110002DE9F84F80460F4615461E46DDF828A09B
:107120000B9A0B464FF0010903E0B3FBF5F309F1AD
:107130000109AB42F9D2B14500D2B14612F0010BC0
:1071400018D1BAF1000F15D012F0020F02D0BEB163
:10715000202400E02024BAF1000F0BD0CA4509D941
:107160000AF1FF3A21464046FFF7B2FFD8F80C304B
:10717000002BF0DAD8F80C30002B33DB012407E0C9
:107180003024E8E7B7FBF4F39D4205D805FB04F48F
:10719000012EF7D9013EF9E7B7FBF4F304FB1377AF
:1071A000114AD15C4046FFF793FFD8F80C30002B12
:1071B00003DBB4FBF5F4002CEED1BBF1000F11D0D2
:1071C000BAF1000F0ED0BAF1000F0BD0CA4509D9A1
:1071D0000AF1FF3A20214046FFF77AFFD8F80C3039
:1071E000002BF0DABDE8F88FB8FE03002DE9F04778
:1071F00082B00746894615469A460A9EDDF82C80DD
:1072000081EAE173A3EBE173012402E093FBF5F360
:1072100001349D42FADD544500D2544636B1B9F1ED
:10722000000F02DB18F0040F00D0013E18F0020F2F
:1072300002D0BAF1000F03D018F0010F00D1F6B957
:10724000FB68002B18DBB9F1000F25DB18F0040FE9
:1072500029D1FB68002B0FDB08F00303022B27D09A
:10726000FB68002B08DBCDF80480009653462A46C5
:1072700049463846FFF74CFF02B0BDE8F087002EC4
:10728000DED0A642DCD9013E20213846FFF720FFA0
:10729000FB68002BF3DAD3E7C9F100092D2138464A
:1072A000FFF716FFD5E72B213846FFF711FFD0E790
:1072B000BAF1000FD4D1002ED2D0002ED0D0A642E9
:1072C000CED9013E30213846FFF702FFFB68002B84
:1072D000F3DAC5E7F0B599B006460C46154603ABA0
:1072E0001393402314930023159317901693A5E04E
:1072F0000027012203E047F00107013482B323781D
:10730000233B0D2B2AD801A151F823F0557303001C
:107310005D7303005D7303005D7303005D73030021
:107320005D7303005D7303005D7303004D73030021
:107330005D730300F77203005D7303005D73030068
:107340004573030047F002070134D7E747F004070D
:107350000134D3E747F008070134CFE70022CDE737
:107360002078A0F13001C9B2092906D8013402EB16
:10737000820253001A18303AF2E72E2802D0002376
:10738000217812E00134002394F800C0ACF1300001
:10739000C0B20928F4D8013403EB8303590001EB90
:1073A0000C03303BF0E714F8011B6C29FBD0682973
:1073B000F9D064294CD00FD9732954D017D9752925
:1073C00024D12968081D28600968019700920A22C3
:1073D00013A8FFF79DFE2DE0582919D0632922D06C
:1073E000252927D1252113A8FFF772FE22E0702955
:1073F00020D12B681A1D2A601968002301930823E5
:107400000093102213A8FFF783FE13E0782911D10F
:107410002968081D2860096801970092102213A8A6
:10742000FFF776FE06E02B681A1D2A60197813A86C
:10743000FFF74EFE0134169B002B23DB14F8011BD3
:1074400001B325293FF454AF13A8FFF741FEF2E73B
:107450002968081D28600968019700920A2213A86C
:10746000FFF7C4FEE6E72B681A1D2A601F6817F8AD
:10747000011B0029DED013A8FFF72AFE169B002B64
:10748000F5DAD7E7169B002B05DD159A32B9159A68
:10749000169B13441693169819B0F0BD03A93046F5
:1074A000FFF7EAFDF3E700BF0EB400B582B003AB0F
:1074B00053F8041B02AA42F8043DFFF70BFF02B089
:1074C0005DF804EB03B0704730B40346002010C9E8
:1074D00020CA641910C310C920CA6C4110C310C956
:1074E00020CA6C4110C310C920CA6C4110C310C916
:1074F00020CA6C4110C310C920CA6C4110C310C906
:1075000020CA6C4110C310C920CA6C4110C340414D
:1075100030BC704730B4002310C920CA641B10C0AF
:1075200010C920CAAC4110C010C920CAAC4110C05B
:1075300010C920CAAC4110C010C920CAAC4110C04B
:1075400010C920CAAC4110C010C920CAAC4110C03B
:1075500010C920CAAC4110C05B41B3FA83F04009A6
:1075600030BC70472DE9F041013B9B0000242546CB
:107570002646A4465FF0000E03E05FEA0C0EBEEB69
:10758000030EBCEB0E0752F8078051F80E70A7FBF4
:107590000878E41955EB080556F100061EF1040EB3
:1075A0009E4501DCE645ECDD40F80C402C463546B6
:1075B00000261CF1040C9C45DCDDBCEB430FDCDD3C
:1075C00040F80C40BDE8F081002304E0002240F8C0
:1075D000232001335BB28B42F8DB704700231A464D
:1075E0008B420DDA10B450F82340224301335BB2D2
:1075F0008B42F8DBB2FA82F040095DF8044B704729
:10760000B3FA83F0400970474B1150F8230001F0A2
:107610001F01012303FA01F108407047013949B203
:1076200001E0013949B2002903DB50F82130002B79
:10763000F7D0013148B2704710B50446FFF7EEFFAE
:1076400090B1024600F18043013B54F82330002101
:1076500001E05B080131002BFBD1501E80B24001DC
:1076600080B2084400B210BD0020FCE70023934222
:107670000BDA10B451F8234040F8234001335BB2D9
:107680009342F7DB5DF8044B70477047013A52B202
:10769000002A14DB10B450F8224051F822309C42EA
:1076A00008D809D3013A52B2002AF4DA00205DF872
:1076B000044B70470120FAE74FF0FF30F7E7002056
:1076C000704730B4013A52B2002407E050F822303B
:1076D00051F822506B401C43013A52B2002AF5DAAD
:1076E000B4FA84F0400930BC704730B589B0154613
:1076F00013460A4601466846FFF70CFF041C18BFF4
:10770000012429466846FFF769FF6400002814BF7A
:107710006042C4F1010009B030BD10B400EB81013A
:10772000002307E051F8042C43EA520341F8043CDB
:10773000D30721460C1F8142F4D85DF8044B7047F3
:1077400070B505461E469DF910402346FFF7BCFE66
:1077500030B9224629463046FFF798FF012805D068
:107760002346324629462846FFF7D4FE70BD70B541
:1077700005461E469DF910402346FFF7CBFE00B993
:1077800070BD2346324629462846FFF79DFEF7E79F
:1077900030B591B005461C4693F900306846FFF7B6
:1077A000E1FED4F8AC3069462846984711B030BDA8
:1077B00008B513460A46FFF7EBFF08BD70B506464D
:1077C0001446006810F001050ED121463046FFF73F
:1077D000A4FF45B104F18044013C56F8243043F045
:1077E000004346F8243070BD13460A463146304601
:1077F000FFF76AFE0546E8E7F0B5A1B007460E467A
:1078000015461C4619463046FFF7E8FEA0B9224649
:10781000314618A8FFF72AFF2246294610A8FFF78D
:1078200025FF214608A8FFF7CFFE01230893214634
:107830006846FFF7C9FE0DE021463846FFF7C4FE53
:1078400071E0214618A8FFF768FF2246294608A8DC
:10785000FFF7B4FF224610A918A8FFF717FF02464A
:1078600000285BD0189B13F0010FEAD0109B13F097
:10787000010F1ED0002A2DDD234610AA18A90846A4
:10788000FFF748FE214618A8FFF747FF2246694642
:1078900008A8FFF7FBFE002815DB23466A4608A967
:1078A0000846FFF737FE2246294608A8FFF786FF5D
:1078B000D0E7214610A8FFF730FF22462946684648
:1078C000FFF77CFFC6E723462A4608A90846FFF7CC
:1078D000FBFDE2E7234618AA10A90846FFF71AFEA7
:1078E000214610A8FFF719FF224608A96846FFF7AE
:1078F000CDFE00280BDB234608AA69466846FFF741
:1079000009FE224629466846FFF758FFA2E72346AC
:107910002A4669466846FFF7D7FDECE7224608A9E4
:107920003846FFF7A3FE21B0F0BD2DE9F04792B035
:107930000546894614461F4693F9006031461046B5
:10794000FFF74CFE10B112B0BDE8F0873A46494649
:107950000AA8FFF72DFF3B460AAA294602A8FFF70F
:1079600017FF3A460AA90846FFF722FF3B46224680
:1079700049464846FFF70CFF3A4621462046FFF7A6
:1079800017FF07F104080096434622462946284679
:10799000FFF7D6FE00964346224621462046FFF7D3
:1079A000CFFE00964346224629462046FFF7DFFEDB
:1079B0003B46224629462846FFF7EAFE0096434604
:1079C0002A4629462046FFF7BBFE0096434622463C
:1079D00029462846FFF7B4FE00212846FFF714FE8B
:1079E00000284AD03346424629462846FFF76CFD18
:1079F000824631462846FFF790FE06F18043013B60
:107A000055F8232042EACA7245F823203A4629460F
:107A10002046FFF7CDFE0096434602AA21462046A7
:107A2000FFF7A5FE0096434602AA21462046FFF72F
:107A30009EFE00964346224602A90846FFF797FE9F
:107A40003B4602AA29462846FFF7A2FE0096434677
:107A50000AAA29461046FFF78AFE324621462846E2
:107A6000FFF704FE324649462046FFF7FFFD324647
:107A70000AA94846FFF7FAFD65E731462846FFF7B1
:107A80004CFEC3E72DE9F0438BB004468946164609
:107A90000023039304930593069307930893099394
:107AA0000AAF032347F8203D154615F9048BFFF76D
:107AB0007FFECDF800802B463A4621462046FFF750
:107AC00056FE33464A4621462046FFF761FECDF872
:107AD00000802B4606F1840221462046FFF730FE47
:107AE0000BB0BDE8F0830000F0B589B006460C4647
:107AF0000822FFF7BBFD0027029701970097E36A72
:107B00000393236B0493636B0593A36B0693E36B5F
:107B1000079308236A4669466846FFF7D5FC054681
:107B200008236A4631463046FFF7CEFC0544236BF6
:107B30000393636B0493A36B0593E36B069307971F
:107B400008236A4669466846FFF7BEFC05440823D9
:107B50006A4631463046FFF7B7FC0544236A009376
:107B6000636A0193A36A0293059704970397A36B33
:107B70000693E36B079308236A4631463046FFF7C6
:107B8000A3FC0544636A0093A36A0193E36A02932A
:107B9000636B0393A26B0492E26B05920693236AD4
:107BA000079308236A4631463046FFF78DFC0544AB
:107BB000E36A0093236B0193636B02930597049729
:107BC0000397236A0693A36A079308236A463146FC
:107BD0003046FFF79FFC2D1A236B0093636B0193D4
:107BE000A36B0293E36B039305970497636A069371
:107BF000E36A079308236A4631463046FFF78AFC5A
